:020000040800F2
:20000000E8120020DD1B0008F91B0008FD1B0008011C0008051C0008091C0008000000000F
:200020000000000000000000000000000D1C0008111C000800000000151C0008191C0008E4
:200040001D1C0008211C0008251C0008291C00082D1C0008311C0008351C0008391C000828
:200060003D1C0008411C0008451C0008491C00084D1C0008511C0008551C0008591C000808
:200080005D1C0008611C0008651C0008691C00086D1C0008711C0008751C0008791C0008E8
:2000A0007D1C0008811C0008851C0008891C0008A11A0008BD1A000800000000951C000849
:2000C000991C000800000000000000009D1C000800000000370F00088D0F0008A91C0008E3
:2000E000AD1C0008B11C0008B51C000800B587B0012141F2040000F04FFCE020ADF800005C
:2001000003208DF8020018208DF8030000A9DFF88C0700F073FC1020ADF8000003208DF886
:20012000020010208DF8030000A9DFF8700700F065FC1021DFF8640700F0C6FC0020ADF8D3
:2001400004004FF48270ADF806000020ADF808000220ADF80A000120ADF80C004FF4007098
:20016000ADF80E000020ADF810000020ADF812000720ADF8140001A9DFF8240700F0EEFCBA
:200180000121DFF81C0700F009FD4FF6FF7007B000BD00B587B00121082000F0FDFB0121E5
:2001A0004FF4804000F008FC4FF42040ADF8000003208DF802001C208DF8030000A9DFF812
:2001C000E40600F01BFC4FF48040ADF8000003208DF8020004208DF8030000A9DFF8C406E6
:2001E00000F00CFC4FF48050ADF8000003208DF8020014208DF8030000A9DFF8A80600F0CB
:20020000FDFB4FF48051DFF89C0600F05DFC0020ADF804004FF48270ADF806000020ADF8A2
:2002200008000020ADF80A000120ADF80C004FF40070ADF80E003820ADF810000020ADF8DD
:2002400012000720ADF8140001A9DFF85C0600F085FC0121DFF8500600F0A0FC4FF6FF70C9
:2002600007B000BD00B587B00121012000F094FB0121DFF8380600F02DFC01210C2000F0CE
:200280008BFB01214FF4004000F096FB3820ADF8000003208DF8020018208DF8030000A9A2
:2002A000DFF8000600F0AAFB4FF40040ADF8000003208DF8020010208DF8030000A9DFF8C2
:2002C000DC0500F09BFB4FF40041DFF8D00500F0FBFB0020ADF804004FF48270ADF80600F8
:2002E0000020ADF808000220ADF80A000120ADF80C004FF40070ADF80E000020ADF8100053
:200300000020ADF812000720ADF8140001A9DFF8A00500F023FC0121DFF8940500F03EFC35
:200320004FF6FF7007B000BD80B51021DFF86C0500F0CDFB062000F05CFA1021DFF85C055A
:2003400000F0C2FB01BD80B54FF40041DFF84C0500F0BDFB062000F088FA4FF40041DFF8B6
:200360003C0500F0B1FB01BD80B51021DFF82C0500F0ADFB042000F03CFA1021DFF81C0569
:2003800000F0A2FB00F05AF801BD80B54FF40041DFF8080500F09BFB042000F066FA4FF4F6
:2003A0000041DFF8F80400F08FFB00F057F801BD80B51021DFF8E40400F089FB502000F0B9
:2003C00018FA1021DFF8D40400F07EFB1021DFF8CC0400F07CFB012000F00BFA002000F05D
:2003E00008FA1021DFF8B40400F06EFB00F026F801BD80B54FF40041DFF8A00400F067FB90
:20040000502000F032FA4FF40041DFF8900400F05BFB4FF40041DFF8840400F058FB0120D4
:2004200000F023FA002000F020FA4FF40041DFF86C0400F049FB00F011F801BD10B50120E9
:20044000002401E000F01AF8C0B2C00705D52000441C42F210718842F4D310BD10B5012009
:20046000002401E000F01EF8C0B2C00705D52000441C42F210718842F4D310BD10B51021D5
:20048000DFF8180400F023FB052000F0B2F900F0ABF904001021DFF8040400F015FB2000D3
:2004A000C0B210BD10B54FF40041DFF8F00300F00EFB052000F0D9F900F0D2F904004FF408
:2004C0000041DFF8D80300F0FFFA2000C0B210BDF8B504000D00160000271021DFF8BC031F
:2004E00000F0F5FA0B2000F084F9200CC0B200F080F9200AC0B200F07CF92000C0B200F0FB
:2005000078F9002000F075F904E000F06DF9BFB278557F1CBFB2B6B2B742F6D31021DFF836
:200520007C0300F0D1FA4FF6FF70F2BD70B504000D0000264FF48051DFF8680300F0C7FABB
:2005400014F07F0000F073F904E000F06BF9B6B27055761CB6B2032EF7D34FF48051DFF877
:20056000440300F0B1FA4FF6FF7070BDF8B504000D00160000274FF40041C84800F0A7FA98
:200580000B2000F072F9200CC0B200F06EF9200AC0B200F06AF92000C0B200F066F90020F0
:2005A00000F063F904E000F05BF9BFB278557F1CBFB2B6B2B742F6D34FF40041B74800F0E0
:2005C00083FA4FF6FF70F2BDF8B504000D0016000027200000F0C6F8FFF7EAFEFFF7A4FEFC
:2005E0001021AE4800F073FAAD2000F002F9200CC0B200F0FEF8200AC0B200F0FAF820009D
:20060000C0B200F0F6F8287800F0F3F8687800F0F0F81021A14800F057FA0220070015E0DE
:20062000401E0028FCD110219C4800F050FAAD2000F0DFF8785D00F0DCF87F1C785D00F08B
:20064000D8F87F1C1021954800F03EFAB6B2B74201D27820E5E7642000E0401E0028FCD1AA
:20066000FFF782FE10218D4800F031FAFFF7E6FE4FF6FF70F2BD38B504000D004FF4805194
:20068000884800F024FA54F08000C0B200F0CFF8287800F0CCF8687800F0C9F8A87800F09A
:2006A000C6F84FF480517F4800F00EFA4FF6FF7032BDF8B504000D0016000027FFF799FE7E
:2006C000FFF741FE4FF40041744800F000FAAD2000F0CBF8200CC0B200F0C7F8200AC0B252
:2006E00000F0C3F82000C0B200F0BFF8287800F0BCF8687800F0B9F84FF40041674800F02E
:20070000E3F90220070017E0401E0028FCD14FF40041624800F0DBF9AD2000F0A6F8785D68
:2007200000F0A3F87F1C785D00F09FF87F1C4FF400415A4800F0C8F9B6B2B74201D27820F9
:20074000E3E7642000E0401E0028FCD1FFF71DFE4FF40041514800F0BAF9FFF77FFE4FF68F
:20076000FF70F2BD10B50400FFF722FEFFF7DCFD10214A4800F0ABF9202000F03AF8200CC8
:20078000C0B200F036F8200AC0B200F032F82000C0B200F02EF81021404800F095F9FFF73E
:2007A0004DFE10BD10B50400FFF723FEFFF7CBFD4FF40041394800F08AF9202000F055F88E
:2007C000200CC0B200F051F8200AC0B200F04DF82000C0B200F049F84FF400412F4800F0C3
:2007E00073F9FFF73BFE10BD80B5002000F001F802BD10B504000221294800F0E1F9002845
:20080000F9D0E4B2210089B2254800F0D5F90121234800F0D5F90028F9D0214800F0CEF996
:20082000C0B210BD80B5002000F001F802BD10B5040002211C4800F0C3F90028F9D0E4B2F9
:20084000210089B2184800F0B7F90121164800F0B7F90028F9D0144800F0B0F9C0B210BDF7
:2008600080B5002000F001F802BD10B5040002210F4800F0A5F90028F9D0E4B2210089B2C7
:200880000B4800F099F90121094800F099F90028F9D0074800F092F9C0B210BD000801404B
:2008A00000300140000C01400038004000023000003C0040ED000008D1040008C9050008AC
:2008C000930100082D05000877060008650200086D050008B306000830B4002200210023C9
:2008E00000243D4D2D6815F00C052A00002A04D0042A05D0082A06D021E03849016020E089
:20090000374901601DE03449096811F47011324A126812F48033890C891C002B03D1314A22
:20092000514301600AE02C4A1268920303D52E4A5143016002E02A4A5143016001E0274972
:2009400001602549096811F0F00212092749545C0168E14041602049096811F4E062120AC1
:200960002249545C4168E14081601B49096811F46052D20A1D49545C4168E140C1601649E9
:20098000096811F44042920B1949545CC168B1FBF4F1016130BC7047C9B2002905D015491A
:2009A000096808431349086005E01249096831EA0000104908607047C9B2002905D00E49A3
:2009C000096808430C49086005E00B49096831EA00000949086070470410024000127A0086
:2009E000001BB70000093D00808D5B004800002060000020181002401C100240F0B40022F1
:200A00000026002400250023002791F803C01CF00F0C624691F803C05FEACC6C01D58B785C
:200A20001A430B781B0621D00368002406E0CD78482D02D10125A5400561641C082C14D2B7
:200A40000125A5400E882E40AE42F6D1A5000F2616FA05F7BB4312FA05F52B43CD78282DDE
:200A6000E5D10125A5404561E7E703600B884FF48074A34226D34368002420E0012514F13C
:200A80000806B5400E882E40AE4217D1A5000F2616FA05F7BB4312FA05F52B43CD78282D85
:200AA00004D1012514F10806B5404561CD78482D04D1012514F10806B5400561641C082CB6
:200AC000DCD34360F0BC704789B20161704789B24161704770B4002200240023002500289F
:200AE00002D51C4A136801E01B4A1368C0F3034582B210F44014B4F5401F08D133F070631F
:200B0000154C246834F07064134D2C600FE0C40205D50324AC40A34353F0706307E0440D2E
:200B2000E4B2240112FA04F4A34353F07063C9B2002905D0410DC9B2090112FA01F10B4362
:200B4000002802D50348036001E00348036070BC704700001C0001400400014010B40022EE
:200B600003881A0012F441520B884C8823438C882343CC8823430C8923434C8923438C89EB
:200B80002343CC8923431A430280828B4FF2FF731A408283098A018210BC7047C9B20029F9
:200BA00004D0018851F04001018004E001884FF6BF721140018070478181704780897047F0
:200BC00000220089084201D0012200E000221000C0B2704770477047704710B4019CDBB2DE
:200BE000012B03D14FF48063038108E0DBB2022B03D14FF4C063038101E000230381E4B2CD
:200C0000012C02D10023C38016E0E4B2022C03D14FF40053C3800FE0E4B2032C03D14FF43C
:200C20008053C38008E0E4B2042C03D14FF44053C38001E00023C380D2B2082A09D10289A1
:200C4000002A02D10022828013E04FF4805282800FE0D2B2092A03D14FF48052828008E0F0
:200C60000289002A02D10022828002E04FF480528280B1F5966F15D0B1F5166F16D0B1F588
:200C8000965F17D0B1F5165F18D0B1F5964F19D0B1F5164F1AD0B1F5614F1BD0B1F5E13F05
:200CA0001CD01FE04FF4966101601EE04FF4166101601AE04FF49651016016E04FF4165170
:200CC000016012E04FF4964101600EE04FF4164101600AE04FF46141016006E05FF4E131E2
:200CE000016002E04FF41651016010BC7047F0B589B004000D0016001F00012144F20400A3
:200D0000FFF74AFE4FF40070ADF8040003208DF8060018208DF8070001A9B248FFF76EFEC1
:200D20004FF48060ADF8040004208DF8070001A9AC48FFF763FEFFB200973300DBB22A0010
:200D4000D2B2210005A8FFF748FF0020ADF820000C20ADF81E0005A9A34800F053F900203B
:200D6000ADF80C000020ADF80E004FF40070ADF810000020ADF8120003A99B4800F0A4F994
:200D8000012240F22551984800F0BEF90121964800F0ACF925208DF8080000208DF80900EC
:200DA00000208DF80A0001208DF80B0002A800F000FA4FF6FF7009B0F0BDF0B589B0040043
:200DC0000D0016001F0001210420FFF7E5FD01215FF40030FFF7F0FD0420ADF80400182026
:200DE0008DF8070003208DF8060001A97D48FFF705FE0820ADF8040004208DF8070001A926
:200E00007848FFF7FBFDFFB200973300DBB22A00D2B2210005A8FFF7E0FE0020ADF82000E7
:200E20000C20ADF81E0005A9704800F0EBF80020ADF80C000020ADF80E004FF40070ADF88E
:200E400010000020ADF8120003A9684800F03CF9012240F22551654800F056F901216348A6
:200E600000F044F926208DF8080000208DF8090000208DF80A0001208DF80B0002A800F0CA
:200E800098F94FF6FF7009B0F0BD10B5040040F22661554800F077F9E4B2210089B252489C
:200EA00000F05BF9012240F226614F4800F02CF94F480078AA28FBD14D485521017000221B
:200EC00040F22661484800F01FF94FF6FF7010BD10B5040040F22661444800F054F9E4B25F
:200EE000210089B2414800F038F9012240F226613E4800F009F93F480078AA28FBD13D4876
:200F000055210170002240F22661384800F0FCF84FF6FF7010BD384A127802700120088003
:200F20004FF6FF707047354A12780270012008804FF6FF70704780B520212B4800F015F9D0
:200F4000C0B201280CD1284800F00BF92A49087040F22551244800F016F929480069804716
:200F60004021214800F001F9C0B201280DD1002240F226611C4800F0C7F840F226611A483B
:200F800000F001F91A48AA21017001BD80B52021164800F0EAF8C0B201280CD1134800F0A2
:200FA000E0F81649087040F22551104800F0EBF81348806A804740210C4800F0D6F8C0B2BE
:200FC00001280DD1002240F22661084800F09CF840F22661054800F0D6F80648AA2101700D
:200FE00001BD00000008014000380140004400406400002065000020E0100020E1100020C3
:2010000000000020F0B585B004000D0000200021002200230026AF89002F2600208A4CF6A0
:20102000FF710840E98808432082A0894EF6F3110840A9882A8911436A8911430843A081F6
:20104000A08A4FF6FF410840A9890843A08200A8FFF742FC1B48864201D1039900E002990A
:20106000A089000407D5192000FB01F029684900B0FBF1F206E0192000FB01F029688900B5
:20108000B0FBF1F26420B2FBF0F000010109642303FB1123A189090408D5D9003231642217
:2010A000B1FBF2F111F00701084307E0190132316422B1FBF2F111F00F010843208105B022
:2010C000F0BD00000038014010B40022038A1A004FF2FF031A400B884C8823438C88234379
:2010E000C98819430A43028210BC7047C9B2002904D0818951F40051818104E081894DF6A4
:20110000FF72114081817047F0B4002300240025002640F66A1789B2B94206000800C0B2B1
:201120004309DBB289B211F01F04012010FA04F5012B01D10C3604E0022B01D1103600E00A
:201140001436D2B2002A03D030682843306002E03068A8433060F0BC7047C905C90D818034
:2011600070478088C005C00D704700224FF4007389B299420088084201D0012200E00022B1
:201180001000C0B2704710B40022002340F66A1489B2A14289B20A0A012111FA02F39BB27D
:2011A000D943018010BC70471E4908431E490860704710B4002100220F23C478002C1ED048
:2011C0001949096811F4E061D1F5E061090AD1F10402CB404178914082781A4011430901CD
:2011E0000278124BD15401784911114A0123007810F01F0013FA00F042F821000AE001784F
:2012000049110C4A0123007810F01F0013FA00F042F8210010BC7047074A1140084307494B
:20122000086070470000FA050CED00E000E400E000E100E080E100E080FFFF1F08ED00E07F
:2012400080B501214020FFF7A7FB0220ADF8000010208DF8030002208DF8020000A97F48A7
:20126000FFF7CCFB02217D48FFF72EFC01BD000080B500F003F900F025F900F044F902206D
:2012800000F054F9FFF7DCFF1423754A0021022000F061F973480021016004E0714800687B
:2012A000401C704908606F480068042805D26D4800686B49405C5A28F0D06A48006804289A
:2012C00040F0B4806648007965494979090451EA00606349897950EA01206149C97908432B
:2012E0006149086060480068B0F5483F03D25E485FF4962101605A4800795949097A08185A
:2013000080B2FF2840F09280554840795449497A081880B2FF2840F089805148807950499F
:20132000897A081880B2FF2840F080804C48C0794B49C97A081880B2FF2877D100F028F98B
:201340004948006810F50051484800F006FA02214248FFF7BCFB43480021016023E04FF411
:201360008052FF213E4800F02EFA4FF480533C4A3C480068401C4FF4805101FB00F10220D6
:2013800000F0E9F84FF48052364800684FF48051364B01FB0031324800F0B8F931480068C3
:2013A000401C304908602F4800682F490968B0EB113FD4D32B4800684FF4805148432A49A9
:2013C000096888422BD24FF48052FF21244800F0FAF925480068234909684FF4805202FB8D
:2013E00011039BB21E4A1F480068401C4FF4805101FB00F1022000F0AEF81B480068194913
:2014000009684FF4805202FB1102164800684FF48051164B01FB0031114800F077F90020F5
:20142000FFF7C0F902210D48FFF74EFB4FF400515FF00060FFF7F0FE4FF4005080F3088889
:20144000DDF800D00A480B49096801600A4808490968016008480068804701BD0018014064
:2014600068000020D8100020D410002000200008D010002004200008CC10002080B500F063
:20148000C3F94FF4C060FFF78FFE01BD80B5214A2148008821494118012000F099FA1E488E
:2014A0000088642804D21C480088401C1A49088019480088642802D117480021018001BD08
:2014C0007047704780B514480021018011480021018001200090002308225FF4E1310120EC
:2014E00000F052FA002801D100200BE00C4B0D4A0D49012000F07EFA002801D1002001E023
:201500004FF6FF7002BD0348002101800248002101807047DE100020DC1000206810002016
:20152000C3140008C11400088D14000810B50024C0B203280CD2C0B20C21144A01FB0020C9
:20154000006880474FF6FF71884201D14FF6FF74200080B210BD70B50400080011001A00D8
:201560000025E4B2032C0DD292B2E4B20C23074E03FB04635B6898474FF6FF71884201D1EC
:201580004FF6FF75280080B270BD0000B4080008DFF83401DFF834110160DFF82C01DFF8E3
:2015A000301101607047DFF82C01006850F08000DFF820110860704738B5040004255FF412
:2015C000302000F08DF80500EDB2042D20D1DFF80401006850F00200DFF8F8100860DFF8DC
:2015E000F8000460DFF8EC00006850F04000DFF8E41008605FF4302000F072F80500DFF8D8
:20160000D400006841F6FD710840DFF8C81008602800C0B232BD70B582B005000C0004266F
:20162000002000904FF4005000F05AF80600F6B2042E2DD1DFF89C00006850F00100DFF854
:20164000941008602C804FF4005000F049F80600F6B2042E13D1A81C0090200C00990880A9
:201660004FF4005000F03CF80600DFF86800006841F6FE710840DFF85C10086008E0DFF8AE
:201680005400006841F6FE710840DFF8481008603000C0B276BD11490860704704200F493F
:2016A0000968C90701D501200CE00C480068400701D5022006E009480068C00601D50320AD
:2016C00000E00420C0B270470420024023016745AB89EFCD10200240142002400C20024061
:2016E00038B504000425FFF7D9FF050003E0FFF7D5FF0500641EEDB2012D01D1002CF6D137
:20170000002C00D105252800C0B232BDF8B505000C00170004208DF80000FFF739FFBE08A7
:201720000420B7FBF0F101FB1071002909D0761C07E029682000FFF76EFF8DF80000241D20
:201740002D1D3000461E80B2002803D09DF800000428EED0FFF727FFF1BD70B582B00400DA
:201760000D0004208DF800004FF48060B4FBF0F101FB1041002901D0002023E0FFF708FF99
:20178000AE0A4FF48060B5FBF0F101FB1051002900D0761C3520FFF77EFF002508E04FF4DD
:2017A000806000FB0540FFF707FF8DF800006D1CB54203D29DF800000428F0D0FFF7F3FECB
:2017C0004FF6FF7076BD10B5040010000A000100200000F031F9200010BD10B450F8041BEC
:2017E00081B102681218001D50F8043BDC0744BFA9F10104E31852F8044B43F8044B091FB4
:20180000F9D1EBE710BC704780B54F48006850F001004D4908604D4800684D4908404B49C7
:201820000860494800684B490840474908604648006830F48020444908604448006830F4AC
:20184000FE004249086044485FF41F01016000F005F842485FF00061016001BD80B500F0CC
:2018600001F801BD82B000200190002000903648006850F48030344908603348006810F478
:20188000003000900198401C01900098002803D10198B0F5A06FF0D12B480068800302D52B
:2018A0000120009001E0002000900098012847D12B48006850F01000294908602848006830
:2018C00080088000264908602548006850F00200234908601D481D49096801601B481B49DA
:2018E000096801601948006850F48060174908601648006830F47C10144908601348006863
:2019000050F48810114908600F48006850F080700D4908600C4800688001FBD50B480068B4
:2019200080088000094908600848006850F00200064908600548006810F00C000828F9D179
:2019400002B070470000000000100240041002400000FFF8FFFFF6FE0810024008ED00E05E
:20196000002002400749002201E01831521C0B78FF2B01D1002004E00B78C0B28342F4D1F9
:2019800008007047000000202DE9F0410E0017009846069CC0B2FFF7E5FF0500002D01D12C
:2019A000002013E02300DBB24246D2B23900C9B230006C682468A047002129724FF6FF71BC
:2019C00080B2884201D10121297280B2BDE8F08138B50C001500C0B2FFF7C4FF0200002ACF
:2019E00001D1002005E02900200052689268904780B232BD70B50C0015001E00C0B2FFF74F
:201A0000B1FF002801D1002004E004614661C5604FF6FF7070BD50F8041B61B150F8042B16
:201A2000D30744BFA9F101039A18002342F8043B091FFAD1EFE7704762F30F2262F31F4221
:201A4000401810F0030308D0C91A1FD3DB0748BF00F8012D28BF20F8022D130030B41446ED
:201A60001546103928BF20E93C00FAD8490728BF20E90C0048BF40F8042D890028BF20F880
:201A8000022D48BF00F8012D30BC7047C91818BF00F8012DCB0728BF00F8012D70470000D3
:201AA00080B501215FF0804000F016F8002804D001215FF0804000F026F801BD80B5012172
:201AC000044800F009F8002803D00121014800F01AF801BD0004004030B400220023002412
:201AE000058A0D402B008089084004009BB2002B04D0A4B2002C01D0012200E000221000B6
:201B0000C0B230BC704789B2C94301827047000080B500F015F802000023DB431068984268
:201B200004D011000220ABBE002010605068984204D0111D0220ABBE0020506001BD0000F8
:201B4000004870475800002010B5084979441C31074C7C441A34A14206D0081D0A685118D4
:201B600088470146A142F8D110BD00BF0800000028000000A3FEFFFF7C1000006800002034
:201B80000000000057FCFFFF680000002C010000000000200000000000F009F8002801D055
:201BA000FFF7D2FF0020FFF763FB00F002F80120704780B500F002B800BF000007463846BF
:201BC00000F002F8FBE7000080B5FFF7A1FF024A11001820ABBEFBE7260002000148804756
:201BE0000148004709180008ED1B0008C046C046C046C046FFF7D0FFFFF7FEBFFFF7FEBFD9
:201C0000FFF7FEBFFFF7FEBFFFF7FEBFFFF7FEBFFFF7FEBFFFF7FEBFFFF7FEBFFFF7FEBF2C
:201C2000FFF7FEBFFFF7FEBFFFF7FEBFFFF7FEBFFFF7FEBFFFF7FEBFFFF7FEBFFFF7FEBF0C
:201C4000FFF7FEBFFFF7FEBFFFF7FEBFFFF7FEBFFFF7FEBFFFF7FEBFFFF7FEBFFFF7FEBFEC
:201C6000FFF7FEBFFFF7FEBFFFF7FEBFFFF7FEBFFFF7FEBFFFF7FEBFFFF7FEBFFFF7FEBFCC
:201C8000FFF7FEBFFFF7FEBFFFF7FEBFFFF708BFFFF714BFFFF7FEBFFFF7FEBFFFF7FEBF8C
:201CA000FFF749B9FFF772B9FFF7FEBFFFF7FEBFFFF7FEBFFFF7FEBF0000000030000020EF
:201CC00000000000D70B0008D50B0008D90B0008010000003C00002000000000D70B0008FF
:201CE000D50B0008D90B0008EF0C00088B0E0008170F0008BB0D0008D10E0008270F000849
:201D000000000000010203040102030406070809FFFFFFFFFFFFFFFF02040608AAAA000031
:201D2000FFFFFFFFFFFFFFFFFFFFFFFFFFFFFFFFFFFFFFFFFFFFFFFFFFFFFFFFFFFFFFFFC3
:201D4000FFFFFFFFFFFFFFFFFFFFFFFFFFFFFFFFFFFFFFFFFFFFFFFFFFFFFFFFFFFFFFFFA3
:201D6000FFFFFFFFFFFFFFFFFFFFFFFFFFFFFFFFFFFFFFFFFFFFFFFFFFFFFFFFFFFFFFFF83
:201D8000FFFFFFFFFFFFFFFFFFFFFFFFFFFFFFFFFFFFFFFFFFFFFFFFFFFFFFFFFFFFFFFF63
:201DA000FFFFFFFFFFFFFFFFFFFFFFFFFFFFFFFFFFFFFFFFFFFFFFFFFFFFFFFFFFFFFFFF43
:201DC000FFFFFFFFFFFFFFFFFFFFFFFFFFFFFFFFFFFFFFFFFFFFFFFFFFFFFFFFFFFFFFFF23
:201DE000FFFFFFFFFFFFFFFFFFFFFFFFFFFFFFFFFFFFFFFFFFFFFFFFFFFFFFFFFFFFFFFF03
:201E0000FFFFFFFFFFFFFFFFFFFFFFFFFFFFFFFFFFFFFFFFFFFFFFFFFFFFFFFFFFFFFFFFE2
:201E2000FFFFFFFFFFFFFFFFFFFFFFFFFFFFFFFFFFFFFFFFFFFFFFFFFFFFFFFFFFFFFFFFC2
:201E4000FFFFFFFFFFFFFFFFFFFFFFFFFFFFFFFFFFFFFFFFFFFFFFFFFFFFFFFFFFFFFFFFA2
:201E6000FFFFFFFFFFFFFFFFFFFFFFFFFFFFFFFFFFFFFFFFFFFFFFFFFFFFFFFFFFFFFFFF82
:201E8000FFFFFFFFFFFFFFFFFFFFFFFFFFFFFFFFFFFFFFFFFFFFFFFFFFFFFFFFFFFFFFFF62
:201EA000FFFFFFFFFFFFFFFFFFFFFFFFFFFFFFFFFFFFFFFFFFFFFFFFFFFFFFFFFFFFFFFF42
:201EC000FFFFFFFFFFFFFFFFFFFFFFFFFFFFFFFFFFFFFFFFFFFFFFFFFFFFFFFFFFFFFFFF22
:201EE000FFFFFFFFFFFFFFFFFFFFFFFFFFFFFFFFFFFFFFFFFFFFFFFFFFFFFFFFFFFFFFFF02
:201F0000FFFFFFFFFFFFFFFFFFFFFFFFFFFFFFFFFFFFFFFFFFFFFFFFFFFFFFFFFFFFFFFFE1
:201F2000FFFFFFFFFFFFFFFFFFFFFFFFFFFFFFFFFFFFFFFFFFFFFFFFFFFFFFFFFFFFFFFFC1
:201F4000FFFFFFFFFFFFFFFFFFFFFFFFFFFFFFFFFFFFFFFFFFFFFFFFFFFFFFFFFFFFFFFFA1
:201F6000FFFFFFFFFFFFFFFFFFFFFFFFFFFFFFFFFFFFFFFFFFFFFFFFFFFFFFFFFFFFFFFF81
:201F8000FFFFFFFFFFFFFFFFFFFFFFFFFFFFFFFFFFFFFFFFFFFFFFFFFFFFFFFFFFFFFFFF61
:201FA000FFFFFFFFFFFFFFFFFFFFFFFFFFFFFFFFFFFFFFFFFFFFFFFFFFFFFFFFFFFFFFFF41
:201FC000FFFFFFFFFFFFFFFFFFFFFFFFFFFFFFFFFFFFFFFFFFFFFFFFFFFFFFFFFFFFFFFF21
:201FE000FFFFFFFFFFFFFFFFFFFFFFFFFFFFFFFFFFFFFFFFFFFFFFFFFFFFFFFFFFFFFFFF01
:2020000040A900202D070408D3C10008D5C10008DBC10008D7C10008D9C10008DDC10008B1
:20202000DDC10008DDC10008DDC10008DDC10008DDC10008DDC1000837330108D72D01083C
:2020400077480108814801088B480108954801089F480108A9480108B3480108BD48010828
:20206000C7480108D1480108DB480108E5480108EF480108F9480108034901080D49010886
:2020800017490108214901082B490108354901083F49010849490108534901085D490108E0
:2020A00067490108714901087B490108854901088F49010899490108A3490108AD49010840
:2020C000B7490108C1490108CB490108D5490108DF490108E9490108F3490108FD490108A0
:2020E000074A0108114A01081B4A0108DFC10008DFC10008DFC10008DFC10008DFC100086C
:20210000DFC10008DFC10008254A01082F4A0108394A0108434A01084D4A0108574A010809
:20212000614A01086B4A0108754A01087F4A0108894A0108934A01089D4A0108A74A0108E7
:20214000B14A0108BB4A0108C54A0108CF4A01080000000000000000000000000000000033
:2021600000000000000000000000000000000000000000000000000000000000000000005F
:2021800000000000000000000000000000000000000000000000000000000000000000003F
:2021A00000000000000000000000000000000000000000000000000000000000000000001F
:2021C0000000000000000000000000000000000000000000000000000000000000000000FF
:2021E0000000000000000000000000000000000000000000000000000000000000000000DF
:2022000058444A32322D424759542D442D56312E3030370000B587B04FF4FA6005F0F2F9BE
:2022200005F004FD66E00422DFF8541A2B2006F098FA0222DFF84C1A1F2006F092FA0122DF
:20224000DFF8DC161B2006F08CFADFF8D816002006F0CEFC0422DFF8281A2B2006F081FA5E
:202260000322DFF8C416222006F07BFA0222DFF8BC16212006F075FA0222DFF8B416232060
:2022800006F06FFA0022DFF8AC16382006F069FA0022DFF8A416392006F063FA0022DFF81B
:2022A0009C163A2006F05DFA0022DFF894163B2006F057FADFF88C060088052190FBF1F2FB
:2022C00001FB1200002801D100F017FA00200090042200A92B2006F044FA0098C00407D5BF
:2022E000DFF8940D00210180DFF8900D0021018000F06AFB642005F085F9DFF848060088B5
:20230000401CDFF840160880DFF8380600880A2190FBF1F201FB1200002806D105208DF8BF
:20232000100004A9022005F0BFF805F0C5FA002804D005F0C1FA01287FF475AF01A806F053
:202340005EFDDFF80406008800287FF46CAF9DF8080002287FF467AF9DF8090002287FF478
:2023600062AF9DF80A0000287FF45DAF9DF80B00002808D09DF80B00012804D09DF80B0029
:2023800002287FF450AFFEE730B400230022002810D000230AE092B2DBB21C5CA4184FF436
:2023A000807594FBF5F202FB15425B1CDBB2C9B28B42F0D3100080B230BC704710B4002383
:2023C000002200280AD00278012303E09BB21C5C62405B1C9BB289B28B42F7D3D2B21000C7
:2023E00080B210BC704770B40023002200280FD0022309E0DBB21C5C4FF4807594FBF5F6F3
:2024000006FB1546B2185B1CDBB2C9B28B42F1D31000C0B270BC70470FB410B40021002059
:202420000022110018E0C9B201AA8A1852780A2392FBF3F403FB14223032C0B2DFF80C351E
:20244000C254401CC9B2032905D2C0B2DFF8FC242E238354401C491CC9B2042957D2C9B2EE
:2024600001AA8A185278642A2ED3C9B201AA8A185278642392FBF3F23032C0B2DFF8CC3480
:20248000C254401CC9B201AA8A1852780A2392FBF3F20A2392FBF3F403FB14223032C0B2F0
:2024A000DFF8A834C254401CC9B201AA8A1852780A2392FBF3F403FB14223032C0B2DFF8E5
:2024C0008C34C254401CBDE7C9B201AA8A1852780A2AA8D3C9B201AA8A1852780A2392FB99
:2024E000F3F23032C0B2DFF86434C254401CC9B201AA8A1852780A2392FBF3F403FB1422DB
:202500003032C0B2DFF84434C254401C9AE7C0B2DFF8381422224254401CC0B2DFF82C1451
:202520002C224254401CC0B2DFF8201420224254401CBDF80A1042F2107291424AD3BDF880
:202540000A1042F2107291FBF2F13031C0B2DFF8FC238154401CBDF80A104FF47A7291FBB8
:20256000F2F10A2291FBF2F302FB13113031C0B2DFF8D8238154401CBDF80A10642291FB03
:20258000F2F10A2291FBF2F302FB13113031C0B2DFF8B8238154401CBDF80A100A2291FB5D
:2025A000F2F10A2291FBF2F302FB13113031C0B2DFF898238154401CBDF80A100A2291FB5D
:2025C000F2F302FB13113031C0B2DFF880238154401C8EE0BDF80A104FF47A72914237D32E
:2025E000BDF80A104FF47A7291FBF2F13031C0B2DFF858238154401CBDF80A10642291FB37
:20260000F2F10A2291FBF2F302FB13113031C0B2DFF838238154401CBDF80A100A2291FB5C
:20262000F2F10A2291FBF2F302FB13113031C0B2C64A8154401CBDF80A100A2291FBF2F379
:2026400002FB13113031C0B2C04A8154401C50E0BDF80A10642925D3BDF80A10642291FBE6
:20266000F2F13031C0B2B94A8154401CBDF80A100A2291FBF2F10A2291FBF2F302FB131148
:202680003031C0B2B14A8154401CBDF80A100A2291FBF2F302FB13113031C0B2AB4A815411
:2026A000401C26E0BDF80A100A2916D3BDF80A100A2291FBF2F13031C0B2A44A8154401C71
:2026C000BDF80A100A2291FBF2F302FB13113031C0B29E4A8154401C0BE0BDF80A100A229B
:2026E00091FBF2F302FB13113031C0B2974A8154401CC0B210BC04B0704780B59448007831
:20270000102805D292480078401C9149087002E08F48002101708F4800788F4909788842ED
:2027200009D08C488C49097801708948002101708A480021018005F0BFF8212800F0C08029
:20274000DFF83C05006843F2F501084203D184480078AA282ED105F08AFADFF824050078AA
:20276000C00703D57C480121017014E0DFF810050078800603D57848022101700BE0DFF897
:2027800000050078400603D573480321017002E071480721017072480078AA2802D16E488D
:2027A000052101706F480078AA280ED16A48062101700AE005F060FA654800210170664832
:2027C0000021017065480021018067480078012803D1022007F081F81BE06348007802281A
:2027E00014D1624800884FF6FF71884206D1022007F073F85D48002101800AE0022007F09E
:2028000084F85A484FF6FF71018002E0022007F07CF857480078012803D056480078AA28FA
:2028200003D1012007F059F81BE051480078022814D1514800884FF6FF71884206D10120A8
:2028400007F04BF84C48002101800AE0012007F05CF849484FF6FF71018002E0012007F0F1
:2028600054F846480078012803D1002007F035F826E04248007802281FD13548007836492F
:202880000978B0EB410F14DA344800884FF6FF71884206D1002007F020F83048002101803B
:2028A0000EE0002007F031F82C484FF6FF71018006E0002007F011F802E0002007F025F824
:2028C00001BD2F48002101802E484FF6FF7101802D48002101802D48002101802C480021B2
:2028E00001802C48002101802B48002101802B48002101802A48002101802A4800210180EF
:202900002948002101802948002101802848002101602848002101802748002101707047D5
:2029200078870020F07C0020368700201A8800201B880020388600203C86002040860020E4
:2029400044860020768700204E870020387E00203288002031880020308800207E870020F5
:20296000E8090020EA090020158800207A87002016880020E90900207C87002017880020A3
:202980009E870020C80900208E870020908700209287002094870020968700209C870020A1
:2029A000988700205487002056870020A08700207C860020508700203688002080B506F077
:2029C000DFFF07F00BF801BD2DE9F04FADF2AC4D5FF0000A00245FF00009002252A9002062
:2029E00005F0BFFE002251A9152005F0BAFE002250A9162005F0B5FE00224FA9052005F0FA
:202A0000B0FE0322DFF80C1E5D2005F0AAFEA6A9002006F0EDF85298DFF8FC1D07F00AF8AB
:202A200007F074F880465198DFF8EC1D07F002F807F06CF806005098DFF8E01D06F0FAFFA7
:202A400007F064F807004F98DFF8D01D06F0F2FF07F05CF805008B480078012802D15FF0A4
:202A600001080FE087480078022802D15FF0020808E084480078002802D15FF0000801E062
:202A80005FF00308DFF8980D0078012803D10120ADF8040002E00020ADF80400DFF8840D0E
:202AA000002101709DF89902002802D15FF0020935E09DF89902062828D1DFF86C0D0078CB
:202AC000022802D15FF0100929E0DFF85C0D0078032802D15FF0110921E0DFF84C0D0078C0
:202AE000042802D15FF0120919E05FF001096448006843F2F501084211D1DFF8280D00782C
:202B000050F08000DFF81C1D087008E09DF89902052802D15FF0040901E05FF0030958481D
:202B20000078800707D5DFF8FC0C007850F00100DFF8F01C087052480078400707D5DFF8BB
:202B4000E40C007850F00200DFF8D81C08704C480078C00707D5DFF8CC0C007850F004006E
:202B6000DFF8C01C087046480078400607D5DFF8B40C007850F00800DFF8A81C0870404810
:202B80000078800607D5DFF89C0C007850F01000DFF8901C08703A480078000607D5DFF866
:202BA000840C007850F02000DFF8781C087034480068C00407D5DFF86C0C007850F08000BF
:202BC000DFF8601C0870DFF8640C008840F22621884208D3DFF8540C008840F22621401AAB
:202BE000DFF8481C0880DFF8480C0088DFF83C1C098880B2884204D3DFF8301C0988441ABA
:202C000005E000F22620DFF8241C0988441AA4B2062CC2F0C284DFF8140CB0F800A01FFAB9
:202C20008AFADFF8100C1AF80000682842F014811AF1010A40F226201FFA8AFA824503D3EC
:202C400040F22620BAEB000A1FFA8AFADFF8E40B1AF800B0BBF1040080B2FA2882F0AC8086
:202C6000A4B21FFA8BFB1BF102008442C2F29C804FF48C72002155A806F05AFF002422E0E7
:202C8000708600202E8800201AF1010A40F226201FFA8AFA824503D340F22620BAEB000A59
:202CA000A4B255A81FFA8AFADFF8881B1AF801102154A4B2042C05D2A4B200A8A4B255A963
:202CC000615C2154641CA4B21FFA8BFB5C45DBD30021002006F044FF1AF1010A40F22620F6
:202CE0001FFA8AFA824503D340F22620BAEB000ADFF8380BA0F800A09DF8000007282DD15F
:202D00009DF80100002829D19DF80200002825D19DF80300002821D14FF48072002104A892
:202D200006F006FF68208DF8100004208DF811000B208DF8120000208DF8130000208DF8A2
:202D4000140000208DF81500CB484FF6FF7101809DF81100811C04A806F033FE9DF80000B1
:202D600013284FD19DF8010000284BD19DF80200002847D19DF80300002843D14FF480723E
:202D8000002104A806F0D4FE68208DF8100004208DF8110023208DF8120000208DF8130035
:202DA00000208DF8140000208DF81500B24800210180B248002101809DF81100811C04A879
:202DC00006F0FFFD4FF48072002104A806F0B0FE68208DF8100001208DF8110002208DF8E0
:202DE00012000822DFF82C1D0DF1130006F082FF00208DF81B0000208DF81C000D2104A894
:202E000006F0DFFD9DF8000083280FD19DF8010000280BD19DF80200002807D19DF80300F7
:202E2000002803D10021002006F09AFE9DF8000043280FD19DF8010000280BD19DF80200B6
:202E4000002807D19DF80300002803D10021002006F086FE9DF85801642840F01F8186480B
:202E600000884FF6FF71884240F018814FF48072002104A806F05CFE9DF80100DFF8341E71
:202E80000880DFF8300E00880002DFF8281E0880DFF8200E00889DF800100843DFF8141EE0
:202EA0000880DFF8100E008880B24008DFF8041E088068208DF810000E208DF81100DFF85A
:202EC000F80D008840008DF81200DFF8EC0D008880B2C0098DF81300DFF8D80D008840001F
:202EE0008DF81400DFF8CC0D008880B2C0098DF81500DFF8C40D0088401CDFF8BC1D0880A8
:202F000064208DF8160001208DF8170007208DF8180000208DF8190000208DF81A00002074
:202F20008DF81B0000208DF81C0000208DF81D0000208DF81E0014208DF81F009DF811002D
:202F4000811C04A806F03DFD142004F05BFBDFF8500E80F80090DFF84C0E80F8008068208C
:202F60008DF8100020208DF81100DFF84C0D008840008DF81200DFF8400D008880B2C009B0
:202F80008DF81300DFF82C0D008840008DF81400DFF8200D008880B2C0098DF81500DFF830
:202FA000180D0088401CDFF8101D088086208DF8160000208DF8170003208DF8180000209F
:202FC0008DF8190000208DF81A0000208DF81B0001208DF81C0030008DF81D00B6B2300A9E
:202FE0008DF81E0038008DF81F00BFB2380A8DF82000BDF804008DF821008DF8228028004C
:203000008DF82300280A8DF82400280C8DF82500280E8DF826000822DFF8F81A0DF1270036
:2030200006F068FE5FFA88F8B8F1020F02D0BFB2012F03D301208DF82F0002E000208DF8FC
:203040002F009DF89902002808D102208DF83000DFF8D00700788DF8310019E09DF8990234
:2030600006280DD101208DF83000DFF8B80700788DF831000CE000BF7287002074870020CB
:2030800003208DF83000DFF89C0700788DF831009DF81100811C04A806F093FC9DF858014E
:2030A000852841F0D5859DF80100DFF8081C0880DFF8000C00880002DFF8F81B0880DFF809
:2030C000F40B00889DF800100843DFF8E81B0880DFF8E00B008880B24008DFF8D81B088001
:2030E0009DF85E01012834D0022800F0A682032800F0A582042800F0DE840F2800F0F7840B
:20310000152800F00985162800F090851A2801F01D801B2801F05C811C2801F05A821D287A
:2031200001F04E831E2801F050831F2801F0E883212800F0A186222800F03A87232801F089
:203140004C84352801F05685362800F0978401F07FBD5FF0010A46A80021002206C008384F
:203160009DF87001182802D316208DF87001002414E0DFF8340E0088401EDFF82C1E088048
:203180000222DFF8241E4FF4137007F024F90322DFF8141E282005F009FB641C9DF8700123
:2031A000A4B280B2844280F0D0810821A4B2092055AA00FB04201D3006F084FE0222DFF87A
:2031C000E81D4FF4137007F0F1F8DFF8DC0D00884FF49671884280F0DB80A4B2092055A9A0
:2031E00000FB041090F8250001285ED15FF0010A01E01AF1010ADFF8B00D00881FFA8AFAB1
:2032000050451CD31FFA8AFA4AF2F34010EBCA00DFF8981D0860082246A9DFF8900D006870
:2032200007F0C4F80822A4B2092055A900FB041010F11D0146A807F0E3F80028D9D1DFF89D
:20324000680D00881FFA8AFA5045A6D2DFF8580D00884AF2FB4111EBC000DFF8501D086023
:203260000822A4B2092055A900FB041010F11D01DFF8380D006807F0AEF80A2004F0C2F97F
:20328000DFF8240D0088401CDFF81C1D08800222DFF8141D4FF4137007F09DF80322DFF830
:2032A000081D282005F082FA77E7A4B2092055A900FB041090F8250002287FF46EAF5FF090
:2032C000010A01E01AF1010ADFF8DC0C00881FFA8AFA5045FFF461AF1FFA8AFA4AF2F34064
:2032E00010EBCA00DFF8C41C0860082246A9DFF8BC0C006807F05AF80822A4B2092055A9DA
:2033000000FB041010F11D0146A807F079F80028D8D1DFF8940C00881FFA8AFA504522D332
:203320001FFA8AFA4AF2FB4010EBCA00DFF87C1C0860082246A9DFF8740C006807F036F8E0
:203340001FFA8AFA4AF2F34010EBCA00DFF85C1C0860082246A9DFF8540C006807F03BF803
:203360001AF1010AD5E7DFF8400C0088401EDFF8381C08800222DFF8301C4FF4137007F0BB
:203380002AF80322DFF8201C282005F00FFA04E7A4B2092055A900FB041090F82500012840
:2033A00074D15FF0010A01E01AF1010ADFF8F80B00881FFA8AFA50451CD31FFA8AFA4AF21B
:2033C000F34010EBCA00DFF8E41B0860082246A9DFF8D80B006806F0E9FF0822A4B20920F5
:2033E00055A900FB041010F11D0146A807F008F80028D9D1DFF8B00B00881FFA8AFA50459E
:20340000BFF4CBAE5FF0010A21E01FFA8AFA4AF2FB4010EBCA00DFF8941B0860082246A945
:20342000DFF8880B006806F0C1FF1FFA8AFA4AF2F34010EBCA00DFF8741B0860082246A94C
:20344000DFF8680B006806F0C6FF1AF1010ADFF8580B0088401E1FFA8AFA5045D5DA1FFACF
:203460008AFA4AF2F34010EBCA00DFF8401B08600822A4B2092055A900FB041010F11D0125
:20348000DFF8280B006806F0A6FF86E6A4B2092055A900FB041090F8250002287FF47DAEB2
:2034A0005FF0010A01E01AF1010ADFF8FC0A00881FFA8AFA5045FFF470AE1FFA8AFA4AF23A
:2034C000F34010EBCA00DFF8E41A0860082246A9DFF8D80A006806F069FF0822A4B2092076
:2034E00055A900FB041010F11D0146A806F088FF0028D8D1DFF8B00A00881FFA8AFA504519
:20350000FFF437AE1FFA8AFA4AF2FB4010EBCA00DFF8981A0860082246A9DFF8900A006817
:2035200006F044FF1FFA8AFA4AF2F34010EBCA00DFF8781A0860082246A9DFF8700A0068DE
:2035400006F049FF1AF1010AD4E7DFF8600A4AF2E9410160092159A8C01C06F0B3FC09227D
:2035600059A9C91CDFF8440A006806F034FF4FF48072002104A806F0DBFA68208DF81000C4
:203580001D208DF81100DFF83007008840008DF81200DFF82407008880B2C0098DF81300CE
:2035A000DFF81007008840008DF81400DFF80407008880B2C0098DF81500DFF8FC0600885C
:2035C000401CDFF8F416088082208DF8160000208DF8170003208DF8180000208DF81900AF
:2035E00000208DF81A0000208DF81B000C208DF81C000D240822DFF81C15A4B204A82018E2
:2036000006F078FB0834092159A8C01C06F05AFC092259A9C91CA4B204A8201806F021FF50
:203620000934A4B204A8002121549DF81100811C04A806F0C6F901F00BBB01F009BBDFF8CE
:203640004C0E00210180042265A9C91CDFF8400E06F007FF9DF89B01112840F080804FF457
:203660008072002104A806F063FA04F025F9002825D100208DF82500082259A9C91CDFF856
:20368000140E06F0EEFE20225BA9C91CDFF89C0E06F0E7FE10220DF5CF71DFF8940E06F0BC
:2036A000E0FEDFF8900E11210170DFF88C0E2A210170DFF8841E012003F013FF02E0012045
:2036C0008DF8250068208DF8100014208DF81100DFF8E405008840008DF81200DFF8D80586
:2036E000008880B2C0098DF81300DFF8C805008840008DF81400DFF8BC05008880B2C0098F
:203700008DF81500DFF8B0050088401CDFF8A815088082208DF8160000208DF81700032067
:203720008DF8180000208DF8190000208DF81A0000208DF81B000D208DF81C000D24082286
:20374000DFF8D013A4B204A8201806F0D3FA08349DF81100811C04A806F033F98CE19DF863
:203760009B01102868D14FF48072002104A806F0DFF968208DF8100014208DF81100DFF8AE
:203780003805008840008DF81200DFF82C05008880B2C0098DF81300DFF8180500884000AE
:2037A0008DF81400DFF80C05008880B2C0098DF81500DFF804050088401CDFF8FC14088038
:2037C00082208DF8160000208DF8170003208DF8180000208DF8190000208DF81A00002093
:2037E0008DF81B000D208DF81C000D240822C949A4B204A8201806F07DFA0834A4B204A809
:20380000012121549DF81100811C04A806F0D9F832E100BF44870020000020410000C84233
:20382000E0870020378800202088002088870020D8860020745400209DF89B01212827D153
:2038400004F03AF8032840F01781082259A9C91CDFF8400C06F005FE20225BA9C91CDFF820
:20386000CC0C06F0FEFD10220DF5CF71DFF8C00C06F0F7FDDFF8BC0C21210170DFF8B80C91
:203880002B210170DFF8B01C012003F02AFEF3E09DF89B01202860D104F00EF8032840F0BA
:2038A000EB80022267A9DFF8D80D06F0DAFDDFF8880C202101709DF89C01012804D1DFF8BC
:2038C000780C2021017042E09DF89C01022804D1DFF8640C2121017039E09DF89C010328EF
:2038E00004D1DFF8540C2221017030E09DF89C01042804D1DFF8400C2321017027E09DF851
:203900009C01052804D1DFF8300C242101701EE09DF89C01062804D1DFF81C0C2521017056
:2039200015E09DF89C01072804D1DFF80C0C262101700CE09DF89C01082804D1DFF8F80BB8
:203940002721017003E0DFF8F00B27210170DFF8E81B012003F0C5FD8EE09DF89B01312898
:2039600027D103F0A9FF002840F08680082259A9C91CDFF8200B06F074FD20225BA9C91CB1
:20398000DFF8A80B06F06DFD10220DF5CF71DFF8A00B06F066FDDFF89C0B31210170DFF8D6
:2039A000980B1F210170DFF8901B012003F099FD62E09DF89B0130285ED103F07DFF0028F6
:2039C0005AD1022267A9DFF8B80C06F04AFDDFF8680B202101709DF89C01012804D1DFF8AD
:2039E000580B2021017042E09DF89C01022804D1DFF8440B2121017039E09DF89C01032810
:203A000004D1DFF8340B2221017030E09DF89C01042804D1DFF8200B2321017027E09DF871
:203A20009C01052804D1DFF8100B242101701EE09DF89C01062804D1DFF8FC0A2521017078
:203A400015E09DF89C01072804D1DFF8EC0A262101700CE09DF89C01082804D1DFF8D80ADA
:203A60002721017003E0DFF8D00A27210170DFF8C81A012003F035FD01F0EAB803F01CFFA0
:203A80000F2816D19DF86701002809D1DFF8A80A2D210170DFF8A01A012003F022FD08E015
:203AA000DFF8940A1C210170DFF88C1A012003F018FD01F0CDB8DFF8340E00210180DFF835
:203AC000300E4FF6FF7101809DF87701012807D09DF87701002803D09DF87701022804D151
:203AE000DFF8101E012003F0FCFC01F0B1B89DF86701012807D09DF86701002803D09DF8D1
:203B00006701022803D1DFF8F00D0021016001F09FB800BF088400200024082159A8C01C0C
:203B200006F024F94FF6FF71884227D1082259A9C91CDFF8C80D06F0FBF80C22DFF8BC1D77
:203B40005E2004F033FE3B21CBA806F091FC1022DFF8A81DCBA806F053FC00280ED03B2188
:203B6000DFF8980D06F0A3FCDFF89C0E00210180DFF8980E002101804FF6FF744FF4807205
:203B8000002104A805F0D4FF68208DF810001B208DF811004848008840008DF81200464825
:203BA000008880B2C0098DF813004248008840008DF814003F48008880B2C0098DF815005B
:203BC0003D480088401C3C49088082208DF8160000208DF8170003208DF8180000208DF811
:203BE000190000208DF81A0000208DF81B0015208DF81C000822DFF8041D0DF11D0006F024
:203C000079F80822DFF8F41C0DF1250006F072F89DF81100811C04A805F0D3FE4FF6FF7036
:203C2000A4B2844200D1FEE701F012B800245FF0000A4FF48072022104A805F079FF9DF874
:203C40009902002804D09DF89902062840F0B3809DF86701012834D106225AA953A806F0C5
:203C600000FC00208DF8520153A806F097F84FF6FF71884222D108214BA806F0F9FB53A85D
:203C800007F03EFDDFF8701E08600422DFF8681E292004F08BFD4B98DFF85C1E096888426E
:203CA00004D00821DFF8500E06F001FC00208DF8250006E08A8700208C87002001208DF825
:203CC00025009DF86E01012821D13C230DF58E625FF4C811022007F02CFD3C225BA9C91C9A
:203CE0000DF58E6006F08CFB00280DD05FF4C81008F0B2F83C235BAAD21C5FF4C8110220E5
:203D000007F031FD4FF6FF7400208DF826009DF8AB0101284CD1A4B2002C45D14521C5A809
:203D200006F0A6FB4521DFF8D40D06F0A1FBDFF8CC0D9DF8AC114170DFF8C00D9DF8AD1192
:203D40008170DFF8B80D9DF8AE11C170DFF8AC0D9DF8AF1101719DF8B0019DF8B11110EB62
:203D60000120DFF8981DC8801622C5A9DFF88C0D06F046FB00280ED04521DFF8800D06F03B
:203D800096FBDFF8840C00210180DFF8800C002101804FF6FF7A00208DF827000BE000BF50
:203DA000338800203488002001208DF8270002E002208DF8270068208DF8100016208DF8F7
:203DC0001100DFF87C0E008840008DF81200DFF8700E008880B2C0098DF81300DFF8640E59
:203DE000008840008DF81400DFF8580E008880B2C0098DF81500DFF8480E0088401CDFF820
:203E0000401E088082208DF8160000208DF8170003208DF8180000208DF8190000208DF8A0
:203E20001A0000208DF81B0016208DF81C000822DFF8C81A0DF11D0005F05CFF9DF81100DD
:203E4000811C04A805F0BDFD4FF6FF701FFA8AFA824509D1DFF8F00D4FF6FF710180DFF897
:203E6000EC0D4FF6FF7101804FF6FF70A4B2844200D1FEE700F0ECBE0422DFF87C1C292015
:203E800004F06FFC4FF48072002104A805F050FE68208DF810005B208DF81100DFF8A00DCC
:203EA000008840008DF81200DFF8940D008880B2C0098DF81300DFF88C0D008840008DF853
:203EC0001400DFF8800D008880B2C0098DF81500DFF86C0D0088401CDFF8641D0880822097
:203EE0008DF8160000208DF8170003208DF8180000208DF8190000208DF81A0000208DF889
:203F00001B0021208DF81C000822DFF8F0190DF11D0005F0EFFE1524DFF8DC0B0268DFF865
:203F2000841EA4B204A8201808F030F8A41D3C230DF12B025FF4C811022007F0FAFB572089
:203F400004004521A0A806F093FAA4B204A89DF881122154641CA4B204A89DF8821221546D
:203F6000641CA4B204A89DF883122154641CA4B204A89DF884122154641CA4B204A8BDF8C7
:203F800086122154641CA4B204A8BDF8861289B2090A2154641C9DF81100811C04A805F01E
:203FA00010FD00F055BE00BF48870020788600204FF48072002104A805F0BAFD68208DF86A
:203FC000100023208DF81100DFF8740C008840008DF81200DFF8680C008880B2C0098DF8EF
:203FE0001300DFF8600C008840008DF81400DFF8540C008880B2C0098DF81500DFF8400C93
:204000000088401CDFF8381C088082208DF8160000208DF8170003208DF8180000208DF8AB
:20402000190000208DF81A0000208DF81B0022208DF81C000822DFF8C4180DF11D0005F018
:2040400059FE1524002245A9382004F08AFB4598DFF8E01D05F0EEFC05F058FDA4B204A912
:204060006054641CA4B204A9020A6254641CA4B204A9020C6254641CA4B204A9000E6054BB
:20408000641C002245A9392004F06BFB4598DFF8A41D05F0CFFC05F039FDA4B204A96054C6
:2040A000641CA4B204A9020A6254641CA4B204A9020C6254641CA4B204A9000E6054641CAF
:2040C000002245A93A2004F04CFB4598DFF8641D05F0B0FC05F01AFDA4B204A96054641C22
:2040E000A4B204A9020A6254641CA4B204A9020C6254641CA4B204A9000E6054641C0022CD
:2041000045A93B2004F02DFB4598DFF8281D05F091FC05F0FBFCA4B204A96054641CA4B246
:2041200004A9020A6254641CA4B204A9020C6254641CA4B204A9000E6054641C9DF811005E
:20414000811C04A805F03DFC00F082BD5FF0000A16240020A4B255A9615C0800641E000269
:20416000A4B255A9615C0818641E0002A4B255A9615C0818641E0002A4B255A9615C0818A4
:20418000641E07F027FFDFF8AC1C07F031FF02900298DFF8681E07F0A9FF12D2002202A9E1
:2041A000382004F003FB092144A806F061F94498029907F0ADFF06D0092102A806F077F925
:2041C00001E05FF0010A1A240020A4B255A9615C0800641E0002A4B255A9615C0818641EF6
:2041E0000002A4B255A9615C0818641E0002A4B255A9615C0818641E07F0ECFEDFF8341C4D
:2042000007F0F6FE02900298DFF8F01D07F06EFF12D2002202A9392004F0C8FA0A2144A868
:2042200006F026F94498029907F072FF06D00A2102A806F03CF901E05FF0010A1E24002017
:20424000A4B255A9615C0800641E0002A4B255A9615C0818641E0002A4B255A9615C0818DB
:20426000641E0002A4B255A9615C0818641E07F0B1FEDFF8C01B07F0BBFE02900298DFF8FC
:204280007C1D07F033FF12D2002202A93A2004F08DFA0B2144A806F0EBF84498029907F077
:2042A00037FF06D00B2102A806F001F901E05FF0010A22240020A4B255A9615C0800641EF0
:2042C0000002A4B255A9615C0818641E0002A4B255A9615C0818641E0002A4B255A9615C61
:2042E0000818641E07F076FEDFF8481B07F080FE02900298DFF8041D07F0F8FE12D20022EB
:2043000002A93B2004F052FA0C2144A806F0B0F84498029907F0FCFE06D00C2102A806F095
:20432000C6F801E05FF0010A4FF48072002104A805F0FEFB68208DF8100014208DF81100AD
:20434000DFF8FC08008840008DF81200DFF8F008008880B2C0098DF81300DFF8E8080088EA
:2043600040008DF81400DFF8DC08008880B2C0098DF81500DFF8C8080088401CDFF8C01852
:20438000088082208DF8160000208DF8170003208DF8180000208DF8190000208DF81A005F
:2043A00000208DF81B001A208DF81C000822DFF84C150DF11D0005F09DFC00208DF825008D
:2043C0009DF81100811C04A805F0FBFA00F040BC4FF48072002104A805F0AAFB68208DF86F
:2043E000100015208DF81100DFF85408008840008DF81200DFF84808008880B2C0098DF821
:204400001300DFF84008008840008DF81400DFF83408008880B2C0098DF81500DFF82008DA
:204420000088401CDFF81818088082208DF8160000208DF8170003208DF8180000208DF8AB
:20444000190000208DF81A0000208DF81B001B208DF81C000822DFF8A4140DF11D0005F01F
:2044600049FC1524A4B204A89DF867112154641CA4B204A8012121549DF8670100280BD120
:20448000A4B204A8002121548BE000BF80870020508600204D7C00209DF8670102280FD04E
:2044A0009DF8670103280BD09DF86701042807D09DF86701052803D09DF8670106284CD1B4
:2044C0009DF89902002803D09DF8990206283FD19DF86701022807D09DF86701032803D04A
:2044E0009DF86701042829D19DF86701DFF8081E08700222DFF8001E692004F057F9002021
:204500008DF80D0048210DF10D0005F0B1FF8DF80D009DF80D00DFF8E01D0978884212D0BB
:204520004821DFF8D40D05F0C2FF0CE0557C0020757C00204C7C0020F50900209DF86701B3
:20454000DFF8B81D0870A4B204A80021215428E0A4B204A80121215423E09DF86701DFF827
:20456000981D08700222DFF8901D692004F01EF900208DF80C00482103A805F079FF8DF81B
:204580000C009DF80C00DFF8701D0978884204D04821DFF8640D05F08AFFA4B204A8002199
:2045A00021549DF81100811C04A805F00AFADFF84C0D0078052800D1FEE7DFF8400D007877
:2045C000062805D106F0DCFF212007F0BFFDFEE73EE39DF86701012854D10020DFF8201D8D
:2045E00000220A709DF8681104290BD29DF86801DFF8781E08709DF86A0100029DF8691113
:20460000081803E0DFF8641E00220A70DFF85C1E097801290AD180B207F0DCFCDFF8701E65
:2046200007F0E6FCDFF86C1E08602BE0DFF83C1E097802290AD180B207F0CCFCDFF8501EDF
:2046400007F0D6FCDFF8501E08601BE0DFF81C1E0978032916D1DFF8441E00228A7080B2BD
:204660003C2190FBF1F201FB1201DFF8302E517080B23C2190FBF1F0DFF8201E087001E001
:204680004C8700204FF48072002104A805F050FA9DF86701012821D103F00EF90C2803D0CD
:2046A00003F00AF90E2816D1DFF8F40D0078012804D0DFF8EC0D007802280CD1DFF85C0E0A
:2046C0002C210170DFF8541E012002F00AFF00208DF8260002E001208DF826009DF8670141
:2046E000022820D1DFF8380E0078AA2818D103F0E3F80E2807D003F0DFF80F2803D003F0AD
:20470000DBF811280CD1DFF8140E2D210170DFF80C1E012002F0E5FE00208DF8260002E054
:2047200001208DF8260068208DF8100015208DF81100DFF80C05008840008DF81200DFF8A7
:204740000005008880B2C0098DF81300DFF8F404008840008DF81400DFF8E804008880B28C
:20476000C0098DF81500DFF8D8040088401CDFF8D014088082208DF8160000208DF8170003
:2047800003208DF8180000208DF8190000208DF81A0000208DF81B001C208DF81C00082215
:2047A00056490DF11D0005F0A5FA9DF867018DF825009DF81100811C04A805F002F947E2FC
:2047C000DFF86C0D0021018042E20020002108009DF86811080000029DF867110818411ED6
:2047E00089B2B1F5616F02D2DFF8481D088000209DF86A11080000029DF869110818411EA8
:2048000089B2B1F5616F02D2DFF82C1D088000209DF86C11080000029DF86B110818411E9F
:2048200089B2B1F5616F02D2DFF8101D088000209DF86E11080000029DF86D110818411E97
:2048400089B2B1F5616F02D2DFF8F41C08804FF48072002104A805F06BF968208DF81000EC
:2048600013208DF81100DFF8D803008840008DF81200DFF8CC03008880B2C0098DF813009D
:20488000DFF8C003008840008DF81400DFF8B403008880B2C0098DF81500DFF8A40300886C
:2048A000401CDFF89C13088082208DF8160000208DF8170003208DF8180000208DF8190017
:2048C00000208DF81A0000208DF81B001E208DF81C00082209490DF11D0005F00BFA9DF854
:2048E0001100811C04A805F06CF8B1E1828700202C870020F6090020A809002008840020DB
:204900004FF48072002104A805F012F968208DF810003D208DF81100C948008840008DF827
:204920001200C748008880B2C0098DF81300C548008840008DF81400C248008880B2C00940
:204940008DF81500BE480088401CBD49088082208DF8160000208DF8170003208DF818008C
:2049600000208DF8190000208DF81A0000208DF81B001F208DF81C000822DFF8C81B0DF138
:204980001D0005F0B7F915241122DFF8BC1BA4B204A8201805F065FD29241122DFF81C1E19
:2049A000A4B204A8201805F05CFD3D24A4B204A8DFF80C1E09882154641CA4B204A8DFF8AC
:2049C000001E098889B2090A2154641C9DF81100811C04A804F0F5FF3AE15FF0000A652213
:2049E0000021DFF8E00D05F0A3F815220021DFF8D80D05F09DF815220021DFF8D00D05F0A3
:204A000097F8002411E000BF7287002074870020A4B255A82018C07C5FFA8AFADFF8A41DC3
:204A20000AF801001AF1010A641CA4B2142C05D2A4B255A82018C07C0028E9D15FFA8AFAEA
:204A4000DFF8800D3A210AF800101AF1010A00240DE0A4B255A8201890F827005FFA8AFA47
:204A6000DFF8601D0AF801001AF1010A641CA4B2052C06D2A4B255A8201890F82700002888
:204A8000E7D100240DE0A4B255A8201890F868005FFA8AFADFF82C1D0AF801001AF1010ABC
:204AA000641CA4B2462C06D2A4B255A8201890F868000028E7D100245FF0000A0DE0A4B2BB
:204AC00055A8201890F82C005FFA8AFADFF8F81C0AF801001AF1010A641CA4B2142C06D21E
:204AE000A4B255A8201890F82C000028E7D100245FF0000A12E000BF488600206C7E002071
:204B0000A4B255A8201890F840005FFA8AFADFF8BC1C0AF801001AF1010A641CA4B2142C87
:204B200006D2A4B255A8201890F840000028E7D14FF48072002104A804F0FAFF68208DF86E
:204B4000100014208DF811003D48008840008DF812003B48008880B2C0098DF81300394878
:204B6000008840008DF814003648008880B2C0098DF8150032480088401C31490880822037
:204B80008DF8160000208DF8170003208DF8180000208DF8190000208DF81A0000208DF8DC
:204BA0001B0023208DF81C000822DFF898190DF11D0005F09FF802F07FFE002803D002F041
:204BC0007BFE01280CD1DFF8080C4FF6FF710180DFF8000C0421017000208DF8250002E010
:204BE00001208DF825009DF81100811C04A804F0E8FE2DE0DFF8DC0B00210170DFF8D80B0A
:204C000000210180DFF8D40B4AF6AA2101800322DFF8C81B5D2003F0C9FD3A210DF10E0034
:204C200005F026FCBDF80E00DFF8B01B0988884204D03A21DFF8A40B05F039FC08E000BF17
:204C40008C8700208A870020388700203E8700209DF85801672840F0A0849DF80100DFF8EE
:204C6000801B0880DFF8780B00880002DFF8701B0880DFF86C0B00889DF800100843DFF8A6
:204C8000601B0880DFF8580B008880B24008DFF8501B08809DF8670110F5FA60ADF83001D9
:204CA0009DF866018DF832019DF865018DF833019DF864018DF835019DF863018DF8360122
:204CC0009DF8620100029DF8611108184FF47A71B0FBF1F08DF837019DF89902002804D010
:204CE0009DF89902062840F058844CA804F033FB4FF6FF71884240F050844CA803F0DAFFF1
:204D00004FF48072002104A804F012FF68208DF8100012208DF81100DFF8C80A0088400036
:204D20008DF81200DFF8BC0A008880B2C0098DF81300DFF8AC0A008840008DF81400DFF85F
:204D4000A00A008880B2C0098DF81500DFF8940A0088401CDFF88C1A088067208DF816000C
:204D600000208DF8170003208DF8180000208DF8190000208DF81A0000208DF81B00012059
:204D80008DF81C00072258A9491C0DF11D0005F068FB9DF81100811C04A804F012FE00F08D
:204DA000FCBB00BF98730008DFF83C0A0088401CDFF8341A0880F0E31FFA8BFBBBF1010F8E
:204DC00042D11AF1010A40F226201FFA8AFA824503D340F22620BAEB000A1FFA8AFADFF85D
:204DE000440E1AF80000022826D100240CE01AF1010A40F226201FFA8AFA824503D340F224
:204E00002620BAEB000A641CA4B2092CEFD3DFF8D809A0F800A0DFF8100E4FF6FF710180B5
:204E2000DFF8080E4FF6FF7101800021002004F097FEB2E30050C347DFF8AC090088401C26
:204E4000DFF8A4190880A8E3DFF89C090088401CDFF894190880A0E31FFA8AFADFF8C40D77
:204E60001AF80000552840F05D831AF1010A40F226201FFA8AFA824503D340F22620BAEBAE
:204E8000000A1FFA8AFADFF89C0D1AF80000BC2840F0F8804FF48C72002155A804F048FEB4
:204EA000002415E01AF1010A40F226201FFA8AFA824503D340F22620BAEB000AA4B255A897
:204EC0001FFA8AFADFF85C1D1AF801102154641CA4B21E2CE6D31AF1010A40F226201FFACD
:204EE0008AFA824503D340F22620BAEB000ADFF8F808A0F800A01D2155A8FDF745FA9DF858
:204F0000711189B280B281427AD1DFF8240D9DF857114170DFF8180D9DF856118170DFF81E
:204F2000100D9DF85511C170DFF8040D9DF8541101719DF858019DF8591110EB0120DFF8F4
:204F4000F01CC880DFF8E80C9DF85D110172DFF8E00C9DF85C114172DFF8D40C9DF85B118C
:204F60008172DFF8CC0C9DF85A11C1729DF85E019DF85F1110EB0120DFF8B41C8881DFF8C0
:204F8000B00C9DF863118173DFF8A40C9DF86211C173DFF89C0C9DF861110174DFF8900C27
:204FA0009DF860114174DFF8880C9DF86F118174DFF87C0C9DF86E11C174DFF8740C9DF82D
:204FC0006D110175DFF8680C9DF86C114175DFF8600C012101704521BFA805F049FA1622B7
:204FE000DFF84C1CBFA805F00BFA002800F0D5824521DFF83C0C05F05AFACEE20100C84219
:20500000DFF8E4070088401CDFF8DC17088006E0DFF8D4070088401CDFF8CC170880DFF803
:20502000C8070088DFF80C1C0988884200F0B582DFF8B407008840F22621884208D3DFF889
:20504000A807008840F22621401ADFF89C170880DFF894070088DFF8DC1B0988884200F021
:205060009C82DFF884070088DFF8B81B405C682807D0DFF874070088DFF8A81B405C5528EE
:20508000C6D18AE21FFA8AFADFF8980B1AF80000002808D01FFA8AFADFF8880B1AF80000CB
:2050A000012840F006821FFA8AFADFF8780B1AF800005FEA002B1AF1010A40F226201FFAEB
:2050C0008AFA824503D340F22620BAEB000A1FFA8AFADFF8500B1AF8000010EB0B0BBBF1EA
:2050E000040040F20B1180B2884280F0DC81A4B21FFA8BFB1BF101008442C0F24E824FF408
:205100008C72002155A804F013FD55208DF854011FFA8BFB5FEA1B208DF8550158468DF8FF
:20512000560100240320040015E01AF1010A40F226201FFA8AFA824503D340F22620BAEBF3
:20514000000AA4B255A81FFA8AFADFF8D81A1AF801102154641CA4B21FFA8BFB1BF1010072
:205160008442E2DB1AF1010A40F226201FFA8AFA824503D340F22620BAEB000ADFF8680678
:20518000A0F800A0594689B255A8FDF717F91FFA8BFB55A91BF8011089B280B2814240F0DB
:2051A000FC819DF85701A0280CD0A12821D0A22836D0A3284BD0A42800F0B480AF2800F0BA
:2051C00057816FE19DF85801012811D1DFF8680A008800280CD1DFF8640A00210180DFF81A
:2051E000600A4FF6FF710180DFF8580A00210180D3E19DF85801012811D1DFF83C0A0088E2
:2052000000280CD1DFF8380A00210180DFF8380A4FF6FF710180DFF82C0A00210180BCE133
:205220009DF85801012811D1DFF80C0A008800280CD1DFF8140A00210180DFF8100A4FF62E
:20524000FF710180DFF8FC0900210180A5E19DF85801012865D1DFF8E0090088002860D16B
:20526000DFF8E80900210180DFF8E4094FF6FF710180DFF8C4094FF6FF7101809DF85C01FE
:20528000DFF8D0190860DFF8CC0900689DF85B1110EB0120DFF8BC190860DFF8B8090068A1
:2052A0009DF85A1110EB0140DFF8A8190860DFF8A40900689DF8591110EB0160DFF89419E7
:2052C0000860DFF8900900684FF48071B0FBF1F202FB1102002A04D1DFF878090068000AF3
:2052E00004E0DFF870090068000A401CDFF86819088000240EE000BF20880020EC0900201E
:2053000013880020A4B24FF4805000FB04F006F0A3FD641CA4B2502CF4D3DFF828090021A2
:2053200001803AE19DF85501012840F09D809DF85601082840F098809DF858019DF859111F
:2053400011EB0020DFF81019098880B2814208D0DFF89C0E4FF6FF710180DFF8F408002128
:205360000180DFF8900E0088401C9DF85A119DF85B2112EB0121884276D19DF85A019DF88D
:205380005B1111EB0020DFF86C1E0880DFF8680EDFF8601E09880180DFF8A80800210180BF
:2053A000DFF8500E0088DFF8B0180988884229D10023DFF8A0080068DFF89C180988491EAF
:2053C0004FF480725143401A0300DBB29BB257AADFF8200E00884FF48071484310F57061AA
:2053E000022006F0C0F9DFF8140E4FF6FF710180DFF8FC0D4FF6FF710180DFF85408002143
:20540000018031E0DFF8EC0D0088032815D10C22DFF8EC1D57A804F0F3FF002816D0DFF8B9
:20542000B40301210170DFF8C80D4FF6FF710180DFF81C080021018008E0DFF8B80D008897
:20544000042803D3DFF88C03032101704FF4807357AADFF8A00D00884FF48071484310F548
:205460007061022006F07FF997E000BF148800209DF8580101280AD1DFF8740D00210180ED
:20548000D34800210180DFF8BC070021018084E00000C8421486002018860020C8840020C1
:2054A0002E88002079E0D0480088401CCE49088073E0CD480088401CCB49088004E0CA4844
:2054C0000088401CC8490880C7480088DFF864170988884261D0C448008840F22621884203
:2054E00006D3C148008840F22621401ABE490880BD480088DFF83C17098888424DD0BA48AF
:205500000088DFF82017405C682806D0B6480088DFF81017405C5528D1D13EE0F709002076
:20552000ED090020B0480088401CAF49088012E086870020C0090020C2090020C409002019
:20554000C609002008840020C8730008A6480088401CA5490880A4480088DFF8D81609885B
:2055600088421AD0A048008840F22621884206D39D48008840F22621401A9B4908809A485D
:205580000088DFF8B0160988884206D096480088DFF89016405C6828D8D18D480088002878
:2055A00041F05A83DFF88006008800282DD1DFF8540C0088642190FBF1F201FB12000028EA
:2055C00023D14FF48072002104A804F0B1FA68208DF8100001208DF8110002208DF81200A9
:2055E0000822DFF8241C0DF1130004F083FB00208DF81B0000208DF81C000D2104A804F098
:20560000E0F90121002004F0ABFADFF8F80B0088DFF8FC1E09880A22514390FBF1F201FBC8
:205620001200002826D1DFF8040600884FF6FF7188421FD14FF48072002104A804F078FAF9
:2056400068208DF8100004208DF8110043208DF8120000208DF8130000208DF814000020E8
:205660008DF81500062104A804F0ABF90121002004F076FADFF88C0B0088DFF8981E09886B
:205680000A22514390FBF1F201FB1200002816D0DFF8840E00785FFA89F948450FD1DFF8C0
:2056A0007C0E00785FFA88F8404508D1DFF8700E0078DFF8701E0978884200F0A780DFF846
:2056C0006C0500884FF6FF71884240F09F80DFF8480E80F80090DFF8440E80F80080DFF8D6
:2056E000400EDFF8401E0978017068208DF8100020208DF811003B48008840008DF8120060
:205700003848008880B2C0098DF813003448008840008DF814003248008880B2C0098DF88F
:20572000150030480088401C2E49088086208DF8160000208DF8170003208DF8180000201C
:205740008DF8190000208DF81A0000208DF81B0001208DF81C0030008DF81D00B6B2300AF6
:205760008DF81E0038008DF81F00BFB2380A8DF82000BDF804008DF821008DF822802800A4
:205780008DF82300280A8DF82400280C8DF82500280E8DF826000822DFF86C1A0DF127001B
:2057A00004F0A8FA5FFA88F8B8F1020F02D0BFB2012F1BD301208DF82F001AE0A073000875
:2057C0004A87002090790020847E00209C7E00204E870020288800205887002044870020A4
:2057E0008A8700208C8700208887002000208DF82F008DF83090DFF82C0D00788DF83100BF
:205800009DF81100811C04A804F0DBF8DFF8180D00884FF6FF71884240F0D480DFF80C0464
:2058200000884FF6FF71884240F0CC80DFF8D40900884FF4FA7190FBF1F201FB1200002857
:2058400040F0C0804FF48072002104A804F070F968208DF8100013208DF81100DFF8CC0CE4
:20586000008840008DF81200DFF8C00C008880B2C0098DF81300DFF8B80C008840008DF823
:205880001400DFF8AC0C008880B2C0098DF81500DFF8980C0088401CDFF8901C088082203C
:2058A0008DF8160000208DF8170003208DF8180000208DF8190000208DF81A0000208DF8AF
:2058C0001B0005208DF81C000D240822DFF83819A4B204A8201804F00DFA9DF81100811CEC
:2058E00004A804F06EF80121002004F039F94FF48072002104A804F01BF968208DF8100013
:205900001D208DF81100DFF8240C008840008DF81200DFF8180C008880B2C0098DF8130038
:20592000DFF80C0C008840008DF81400DFF8000C008880B2C0098DF81500DFF8F00B0088BD
:20594000401CDFF8E81B088082208DF8160000208DF8170003208DF8180000208DF8190012
:2059600000208DF81A0000208DF81B000C208DF81C000D240822DFF89018A4B204A82018C7
:2059800004F0B8F90834DFF8AC0B4AF2E94101600922A4B204A82118DFF8980B006804F095
:2059A00005FD0921A4B204A8201804F08BFA0934A4B204A8002121549DF81100811C04A844
:2059C00003F0FFFFDFF8700B00884FF6FF71884240F0B080954800884FF6FF71884240F009
:2059E000A980DFF8540B002101804FF48072002104A804F09DF868208DF8100079208DF8E0
:205A00001100DFF8280B008840008DF81200DFF81C0B008880B2C0098DF81300DFF8100B01
:205A2000008840008DF81400DFF8040B008880B2C0098DF81500DFF8F40A0088401CDFF872
:205A4000EC1A088082208DF8160000208DF8170003208DF8180000208DF8190000208DF89C
:205A60001A0000208DF81B0001208DF81C000822DFF894170DF11D0004F03CF9DFF8BC1AED
:205A800049A804F005FA082249A90DF1250004F0E8FC08210DF1250004F014FA0622002174
:205AA0000DF12D0004F044F806210DF12D0004F009FA0A2200210DF1330004F039F810226D
:205AC000DFF8E41E0DF13D0004F0CBFC042200210DF14D0004F02CF8022200210DF15100B9
:205AE00004F026F8202200210DF1530004F020F8082200210DF1730004F01AF80822DFF811
:205B0000AC1E0DF17B0004F0ACFC082200210DF1830004F00DF808210DF1830004F0D2F978
:205B20009DF81100811C04A803F04BFF0121002004F016F8DFF8780E00884FF6FF71884291
:205B400040F0A480394800884FF6FF71884240F09D80DFF85C0E002101804FF480720021E3
:205B600004A803F0E5FF68208DF810004C208DF81100DFF8B809008840008DF81200DFF8B5
:205B8000AC09008880B2C0098DF81300DFF8A009008840008DF81400DFF89409008880B226
:205BA000C0098DF81500DFF884090088401CDFF87C19088082208DF8160000208DF817004D
:205BC00003208DF8180000208DF8190000208DF81A0000208DF81B0036208DF81C000822A7
:205BE000DFF824160DF11D0004F084F8DFF8C40D00788DF82500DFF8C00D007831282DD1CC
:205C0000DFF8B81D49A804F043F9082249A90DF1260004F026FC08210DF1260004F052F9D5
:205C200023E000BF7454002074870020728700206C7E0020D88600209C870020C8090020CA
:205C40008E8700209E8700209087002092870020948700207C860020548700201022DFF8F9
:205C60005C1D0DF12E0004F0FCFB2022DFF8501D0DF13E0004F0F5FB9DF81100811C04A8FF
:205C800003F09FFE0121002003F06AFFDFF8340D00884FF6FF71884263D1DFF82C0D0088EB
:205CA0004FF6FF7188425CD1DFF858050088142190FBF1F201FB1200002852D14FF480724B
:205CC000002104A803F034FF68208DF8100013208DF81100DFF85408008840008DF8120059
:205CE000DFF84808008880B2C0098DF81300DFF84008008840008DF81400DFF83408008847
:205D000080B2C0098DF81500DFF820080088401CDFF81818088082208DF8160000208DF89A
:205D2000170003208DF8180000208DF8190000208DF81A0000208DF81B001D208DF81C0071
:205D40000822DFF8C4140DF11D0003F0D3FF9DF81100811C04A803F034FE0121002003F041
:205D6000FFFEDFF8240F00884FF6FF71884240F0BE81DFF8540C00884FF6FF71884240F038
:205D8000B681DFF8040F002101804FF48072002104A803F0CDFE68208DF81000D0208DF8EE
:205DA0001100DFF88807008840008DF81200DFF87C07008880B2C0098DF81300DFF870074A
:205DC000008840008DF81400DFF86407008880B2C0098DF81500DFF854070088401CDFF816
:205DE0004C17088082208DF8160000208DF8170003208DF8180000208DF8190000208DF89C
:205E00001A0000208DF81B0002208DF81C000322DFF8781E4FF4097004F0C8FADFF86C0E90
:205E20004078E121484300F25020DFF808170860DC22DFF85C1EDFF8FC06006804F0B6FA29
:205E40000D240822F049A4B204A8201803F052FF0834DFF83C0E806A03F0C6FFA4B204A92E
:205E60006054641CA4B204A9000A6054641CDFF8200E90F83E0003F0B7FFA4B204A9605482
:205E8000641CDFF80C0E90F83D0003F0ADFFA4B204A96054641CDFF8F80D90F83C0003F063
:205EA000A3FFA4B204A96054641CDFF8E40D90F83B0003F099FFA4B204A96054641CDFF8E5
:205EC000D00D90F83A0003F08FFFA4B204A96054641CDFF8BC0D008FB0F5FA6003F084FFC7
:205EE000A4B204A96054641C0822C749A4B204A8201803F0FFFE0834A4B204A8DFF8901D45
:205F000091F8B5102154641CA4B204A800212154641C0822DFF8941AA4B204A8201804F049
:205F2000A0FA08340822DFF86C1DA4B204A8201804F097FA0834DFF8580D90F83E004FF4C1
:205F40007A714843A4B204A96054641CA4B204A9000A6054641CA4B204A8DFF8341D91F8A0
:205F60003D102154641CA4B204A8DFF8241D91F83C102154641CA4B204A8DFF8141D91F868
:205F80003B102154641CA4B204A8DFF8041D91F83A102154641CA4B204A8DFF8F41C098F7E
:205FA00030312154641CDFF8E80C90F846004FF47A714843A4B204A96054641CA4B204A9FF
:205FC000000A6054641CA4B204A8DFF8C41C91F845102154641CA4B204A8DFF8B41C91F8C5
:205FE00044102154641CA4B204A8DFF8A41C91F843102154641CA4B204A8DFF8941C91F8DC
:2060000042102154641CA4B204A8DFF8841CB1F8401030312154641C00200021080018E030
:20602000C0B2DFF86C1C11EB4001B1F85410A4B204AAA154641CC0B2DFF8541C11EB4001D6
:20604000B1F8541089B2090AA4B204AAA154641C401CC0B23028E3D3DFF8340C006DDFF835
:20606000A81E03F0E7FC03F051FDA4B204A96054641CA4B204A9020A6254641CA4B204A9C4
:20608000020C6254641CA4B204A9000E6054641CA4B204A802212154641CA4B204A800213A
:2060A0002154641CA4B204A800212154641CA4B204A800212154641CA4B204A8DFF8D01BF7
:2060C00091F8B4102154641C241D2022DFF83C1EA4B204A8201804F0C4F99DF81100811C9C
:2060E00004A803F06EFC0121002003F039FD01F0E3FB44490988DFF8182E12880A235A43BE
:2061000091FBF2F302FB1311002940F0C58280B2112800F0C182DFF8B00800884FF6FF71E3
:20612000884240F0B9820322DFF8601B4FF4097004F03CF90222DFF8DC1D262002F036FB71
:20614000DFF8480B80780128C0F0A682DFF8C80D006800285AD1DFF8C40D0078E121484308
:2061600000F25020DFF8CC130860DC22DFF8201BDFF8C003006804F019F90621DFF8940DE8
:2061800004F095F9DFF8080B0079AA2822D0DFF8000BAA210171DC22DFF8F41AE5480068BF
:2061A00004F019F9DFF8E40A8078012812D3DFF8DC0A8078401EDFF8D41A88700322DFF842
:2061C000CC1A4FF4097004F006F90621DFF8440D04F06DF9DFF8440D0078401CDFF83C1D55
:2061E0000870DFF8340D42F20F71016054E200BF9687002056870020528700209887002093
:20620000002200087687002008840020DFF80C0D0078A12803D3DFF8040D01210170DFF832
:20622000FC0C0078E121484300F25020C1490860DC22DFF85C1ABF48006804F0B7F8DFF849
:20624000CC0E00210170DFF8480A0079552841D0DFF8C80C0078401CDFF8C01C0870DFF821
:20626000BC0C0078A12803D3DFF8B00C01210170DFF8A80C0078E121484300F25020AD4931
:206280000860DC22DFF8081AAA48006804F08EF8DFF8780E0078401CDFF8701E0870DFF8E6
:2062A0006C0E0078A128CED3DFF8E009002181700322DFF8D8194FF4097004F08CF802226B
:2062C000DFF8501C262002F071FA0621DFF8440C04F0EDF8DFF8B8090079AA2800F0DC8181
:2062E000DFF8AC09806ADFF8301C08604FF48072002104A803F01CFC68208DF81000DA2079
:206300008DF811008948008840008DF812008748008880B2C0098DF8130085480088400038
:206320008DF814008248008880B2C0098DF815007E480088401C7D49088082208DF81600A8
:2063400000208DF8170003208DF8180000208DF8190000208DF81A0000208DF81B00032061
:206360008DF81C000822DFF8A81D0DF11D0003F0C1FCDFF81C09806A03F036FD01008DF859
:206380002510000A8DF82600DFF8040990F83E0003F02AFD8DF82700DFF8F40890F83D000B
:2063A00003F022FD8DF82800DFF8E40890F83C0003F01AFD8DF82900DFF8D40890F83B0069
:2063C00003F012FD8DF82A00DFF8C40890F83A0003F00AFD8DF82B00DFF8B408008FB0F536
:2063E000FA6003F001FD8DF82C000822DFF8201D0DF12D0003F07EFC0822DFF8B41E49A807
:2064000004F02FF8082249A90DF1350004F029F80822DFF880180DF13D0004F022F83524C2
:20642000641CDFF86C0890F83E004FF47A714843A4B204A96054641CA4B204A9000A60541A
:20644000641CA4B204A8DFF8481891F83D102154641CA4B204A8DFF8381891F83C10215445
:20646000641CA4B204A8DFF8281891F83B102154641CA4B204A8DFF8181891F83A10215469
:20648000641CA4B204A8DFF80818098F30312154641CDFF8FC0790F846004FF47A71484334
:2064A000A4B204A96054641CA4B204A9000A6054641CA4B204A8DFF8D81791F84510215449
:2064C000641CA4B204A8DFF8C81791F844102154641CA4B204A8DFF8B81791F843102154B9
:2064E000641CA4B204A8DFF8A81791F842102154641CA4B204A8DFF89817B1F840103031D2
:206500002154641C4420040000200021080030E0C2090020C4090020338800203488002036
:206520003588002037880020848700208C8700208A8700207886002080870020267C002009
:20654000C0B2DFF84C1711EB4001B1F85410A4B204AAA154641CC0B2DFF8341711EB4001FB
:20656000B1F8541089B2090AA4B204AAA154641C401CC0B23028E3D3DFF81407006DDFF835
:20658000881903F057FA03F0C1FAA4B204A96054641CA4B204A9020A6254641CA4B204A9E9
:2065A000020C6254641CA4B204A9000E6054641CA4B204A802212154641CA4B204A8002115
:2065C0002154641CA4B204A8DFF8C41691F8B5102154641CA4B204A800212154641C002098
:2065E0004890DFF8AC06406BDFF81C1903F022FA03F08CFA4890042248A9A4B204A82018D2
:2066000003F02FFF241D241DDFF88406C06CDFF8F81803F00FFA03F079FAA4B204A960544A
:20662000641CA4B204A9020A6254641CA4B204A9020C6254641CA4B204A9000E6054641C09
:20664000A4B204A8DFF8481691F8B5102154641CA4B204A800212154641CA4B204A8002185
:206660002154641CA4B204A8DFF8241691F8B4102154641C2022DFF89418A4B204A82018D1
:2066800003F0EFFE9DF81100811C04A803F099F90121002003F064FADFF85C0C00884AF60C
:2066A000AA21884206D1DFF8540C00884FF6FF7188426ED1C44800884FF6FF71884268D1A5
:2066C000DFF83C0C0088642190FBF1F201FB120000285ED14FF48072002104A803F028FAA4
:2066E00068208DF8100028208DF81100DFF8140C008840008DF81200DFF8080C008880B2A4
:20670000C0098DF81300DFF8000C008840008DF81400DFF8F40B008880B2C0098DF81500E1
:20672000DFF8E00B0088401CDFF8D81B088082208DF8160000208DF8170003208DF81800A8
:2067400000208DF8190000208DF81A0000208DF81B0035208DF81C000822DFF8B4190DF13A
:206760001D0003F0C7FA1122DFF8A01B0DF1250003F077FEDFF8980B00788DF839009DF8B3
:206780001100811C04A803F01CF90121002003F0E7F9DFF8800B00884FF6FF71884213D135
:2067A000DFF8700B002101804FF48072002104A803F0BEF955208DF81000BC208DF81100BD
:2067C000022104A803F0FDF8DFF84C0B00884FF6FF71884240F0C880DFF83C0B0021018095
:2067E0004521B9A803F044FE1622DFF8301BB9A803F006FE002804D04521DFF8200B03F094
:2068000056FE4FF48072002104A803F091F955208DF81000BA208DF81100DFF8000B0079D0
:206820008DF81200DFF8F40AC0788DF81300DFF8EC0A80788DF81400DFF8E00A40788DF8C0
:206840001500DFF8D80AC0888DF81600DFF8CC0AC08880B2000A8DF81700DFF8C00AC07ADF
:206860008DF81800DFF8B40A807A8DF81900DFF8AC0A407A8DF81A00DFF8A00A007A8DF8E8
:206880001B00DFF8980A80898DF81C00DFF88C0A808980B2000A8DF81D00DFF8800A407C49
:2068A0008DF81E00DFF8740A007C8DF81F00DFF86C0AC07B8DF82000DFF8600A807B8DF8D2
:2068C000210001208DF8220000208DF82300C2208DF8240001208DF8250003208DF82600E3
:2068E00000208DF8270000208DF8280004208DF82900DFF8280A407D8DF82A00DFF81C0ABB
:20690000007D8DF82B00DFF8140AC07C8DF82C00DFF8080A807C8DF82D001E2104A8FBF7F4
:2069200062FD8DF82E001F2104A803F04AF84FF47A7000F067FE1F2104A803F042F84FF446
:206940007A7000F05FFE1F2104A803F03AF84FF47A7000F057FE1F2104A803F032F8DFF89D
:20696000C0094FF6FF710180DFF8B40900884FF6FF71884255D1DFF8880900881E2190FB9D
:20698000F1F201FB120000284BD14FF48072002104A803F0CDF855208DF81000FF208DF85A
:2069A0001100002417E000BF167C0020367C00205A8700204C7C00202988002028840020E2
:2069C000557C00208687002072870020A4B204A820188470641CA4B21C2CF7D37A208DF84B
:2069E0002E001F2104A802F0ECFF4FF47A7000F009FE1F2104A802F0E4FF4FF47A7000F09E
:206A000001FE1F2104A802F0DCFF4FF47A7000F0F9FD1F2104A802F0D4FFDFF804090021F5
:206A20000180DFF8000900884FF6FF71884240F0B780DFF8F00800210180DFF8E008002136
:206A400001704521B3A803F013FD1622DFF8CC18B3A803F0D5FC002804D04521DFF8BC08F2
:206A600003F025FD4FF48072002104A803F060F81222DFF8B41804A803F0F3FC31208DF879
:206A800022002C208DF8230022208DF8240054208DF8250043208DF8260050208DF82700AD
:206AA00022208DF828002C208DF8290022208DF82A0000244521DFF8640803F0D9FCDFF890
:206AC0005C1884B06846162205F048FB0FBCFBF7A3FC0400E4B22200DFF850180DF12B0070
:206AE00003F0BFFCE4B204A820182C21C176E4B204A8201831210177E4B204A820180D21FE
:206B00004177E4B204A820180A218177E4B214F11F0104A802F055FF4FF47A7000F072FDE7
:206B2000E4B214F11F0104A802F04BFF4FF47A7000F068FDE4B214F11F0104A802F041FF97
:206B4000FFA84030342105F041FBE4B214F119020DF11601FFA8403003F083FCE4B214F1A9
:206B60001901FFA8403002F02CFF4FF47A7000F049FDE4B214F11901FFA8403002F021FF86
:206B80004FF47A7000F03EFDE4B214F11901FFA8403002F016FFDFF898074FF6FF7101801E
:206BA000DFF88C0700884FF6FF71884251D1DFF850070088142190FBF1F201FB12000028B3
:206BC00047D14FF48072002104A802F0B1FF1022DFF8601704A803F044FC0D208DF82000C8
:206BE0000A208DF82100122104A802F0EAFE40F2DC5000F007FD122104A802F0E2FE40F2D7
:206C0000DC5000F0FFFC122104A802F0DAFE9BA8142105F0DBFA0C220DF116019BA803F0F9
:206C200020FC0C219BA802F0CCFE40F2DC5000F0E9FC0C219BA802F0C4FE40F2DC5000F067
:206C4000E1FC0C219BA802F0BCFEDFF8E40600210180FBF736FE4AE30021002002F080FFD3
:206C6000DFF8D4060088642816D3DFF8D00600210180DFF8CC064FF6FF710180DFF87C06DF
:206C80004FF6FF71018018E08287002074860020F46B0020F96B0020DFF8640600880A218C
:206CA00090FBF1F201FB1200002806D1DFF888060088401CDFF880160880DFF8880600882E
:206CC0004FF6FF71884231D1DFF834060088322190FBF1F201FB1200002827D14FF4807276
:206CE000002104A802F024FF55208DF8100000208DF8110004208DF81200A0208DF81300DF
:206D00009DF811009DF8121011EB002189B204A8FBF754FB8DF814009DF811009DF81210DB
:206D200011EB0020411C04A802F04BFEDFF8180600884FF6FF71884250D1DFF8C4050088AE
:206D40000A2190FBF1F201FB1200002846D14FF48072002104A802F0EBFE55208DF8100066
:206D6000002401222F21DFF8E40502F0E1FE01220021DFF8DC0502F0DBFE08E0E4B204A8FA
:206D80002018E4B2DFF8CC15615C0171641CE4B2DFF8C005205C2F28F0D100208DF8110042
:206DA000201D8DF81200A1208DF813009DF811009DF8121011EB002189B204A8FBF7FEFA5B
:206DC000E4B204A9611808719DF811009DF8121011EB0020411C04A802F0F3FDDFF87805C6
:206DE00000884FF6FF71884264D1DFF8140500880A2190FBF1F201FB120000285AD14FF4A2
:206E00008072002104A802F093FE55208DF810000024002501220021DFF8400502F088FE05
:206E2000DFF83C0505F0DCF90400E4B22200DFF8301505A803F015FBE4B204A8201800214D
:206E4000417101220021DFF81C0502F071FEDFF8180505F0C5F90500EDB22A00DFF808157A
:206E6000E4B204A82018401D03F0FBFA00208DF811002819401D8DF81200A2208DF813000E
:206E8000E4B2EDB2281904A944189DF811009DF8121011EB002189B204A8FBF78FFA6071C6
:206EA0009DF811009DF8121011EB0020411C04A802F087FDDFF8B40400884FF6FF71884244
:206EC00068D1DFF83C0400880A2190FBF1F201FB120000285ED14FF48072002104A802F0E8
:206EE00027FE55208DF810000025002401222F21DFF8580402F01CFE01220021DFF85004F9
:206F000002F016FE0DE000BF0000C842AE6C0020C609002076860020A8090020F409002082
:206F20006D1CEDB2DFF82C04285C2F28F8D1EDB2DFF820042818401C05F052F90400E4B26E
:206F40002200EDB2DFF80C042818411C05A803F088FA00208DF81100201D8DF81200A3207D
:206F60008DF813009DF811009DF8121011EB002189B204A8FBF722FAE4B204A961180871D5
:206F80009DF811009DF8121011EB0020411C04A802F017FDDFF8D80300884FF6FF718842B0
:206FA0006ED1D7480088022190FBF1F202FB1102002A65D14FF48072002104A802F0B8FD41
:206FC00055208DF8100000208DF8110009208DF81200A4208DF8130001208DF81400DFF844
:206FE0009403008880B2000A8DF81500DFF8840300888DF816000020DF490988491C0800D5
:2070000080B2010A8DF817108DF818009DF811009DF8121011EB002189B204A8FBF7CEF9D0
:207020008DF81900D5480088D3490988491C88420FD09DF811009DF8121011EB0020411C7C
:2070400004A802F0BEFCCC480088401CCB49088016E0CB48007801280DD3C9480021017017
:207060009DF811009DF8121011EB0020411C04A802F0A7FC04E0C2480078401CC0490870B6
:20708000C04800884FF6FF71884240F030819C480088142190FBF1F201FB1200002840F08B
:2070A00026814FF48072002104A802F041FD55208DF8100000208DF8110004208DF812007C
:2070C000AF208DF813009DF811009DF8121011EB002189B204A8FBF771F98DF814009DF85E
:2070E00011009DF8121011EB0020411C04A802F068FCA54800884FF6FF71884240F0EC80BD
:20710000A2480021018000241DE000BF2F880020088400204FF480720021CFA802F008FDBC
:207120004FF48073CFAAA4B24FF4807000FB04F010F58051022004F0FCFA4FF48071CFA89B
:2071400002F0D6FF641CA4B291480068801EB4EB102FDFD3A4B24FF4807000FB04F08C49D6
:207160000968891E884227D24FF480720021CFA802F0DEFC86480068801EA4B24FF480713D
:2071800001FB04F1431A9BB2CFAAA4B24FF4807000FB04F010F58051022004F0CAFA7C48EF
:2071A0000068801EA4B24FF4807101FB04F1411A89B2CFA802F09CFF4FF480720021CFA8E7
:2071C00002F0B6FC0223CFAA7148006800F6FE71022004F0AEFA6D4800889DF83D139DF872
:2071E0003C2312EB0121884264D100A869490A680260042300AA0021022004F0B4FA644882
:207200000068801E000E8DF8000061480068801E000C8DF801005E480068801E000A8DF859
:2072200002005B480068801E8DF80300042300AA0421022004F097FA55480068801EC043D8
:20724000000E8DF8000052480068801EC043000C8DF801004E480068801EC043000A8DF838
:2072600002004B480068801EC0438DF80300042300AA0821022004F076FA1F48002101805F
:2072800003221D495D2001F091FA0020ADF804003A2101A803F0ECF8BDF80400164909881D
:2072A000884203D03A21144803F001F9FEE700BF096C002016480221017020480021018058
:2072C0003048002101801E484FF6FF7101800B484FF6FF7101800AE0184800210180184823
:2072E0004FF6FF71018005484FF6FF7101800DF2AC4DBDE8F08F00004487002058870020CF
:20730000768700208C8700208A870020A0730008288800203A870020388700206C7E002037
:207320003C8700203E870020B4730008387E002040870020D87300089E8700204E8700200C
:207340009A870020C80900208E870020F3790020F47900209079002090870020987E002017
:20736000847E0020B07E00209C7E002092870020948700205487002056870020A0870020B0
:20738000368800209687002098870020508700207C860020EC730008253036640000000024
:2073A00056312E3030372D30322D3138303331320000000061646D696E2C41542B434950C5
:2073C00053434F4E543D0000534820584420414320504F4C4500000061646D696E2C4154D4
:2073E0002B43495245534554000000005A5A5A5A10B4B84A002306210024230002E002F2BE
:207400000C025B1C9BB2062B05D21478A4B280B28442F4D11900080080B210BC704710B459
:20742000AD4A002304210024230001E010325B1C9BB2042B05D21478A4B280B28442F5D139
:207440001900080080B210BC704738B5A14C0020ADF8000000250020050008E000AB0022B8
:20746000A168606804F0DCFE04F20C046D1CADB2062DF3D3002000F0A1F831BD38B5964C20
:207480000020ADF8000000250020050008E000AB227B92B2A168606805F032F810346D1CAC
:2074A000ADB2042DF3D331BD1CB50C0000218DF8041080B2FFF7B3FF01A9009100230A228D
:2074C000210080B2844C14EB0010406805F035F99DF80400002802D14FF6FF7000E0002067
:2074E00016BD1CB50C0000218DF8041080B2FFF796FF01A9009110230A22210080B2764CB6
:2075000014EB0010406805F018F99DF80400002802D14FF6FF7000E0002016BD30B585B079
:207520000C00150000218DF8081080B2FFF777FF02A9019103A900910A230022ADB229007D
:2075400080B2654D15EB0010406805F017F820609DF80800002802D14FF6FF7000E00020BF
:2075600005B030BD30B583B000228DF8042089B24FF47A725143594A1268B1FBF2F480B2A7
:20758000FFF736FF010089B2062901D1002014E001A9009100230022210080B20C244D4DD2
:2075A00004FB0050406804F06EFE9DF80400002802D14FF6FF7000E000203EBD10B582B03A
:2075C00000218DF8001080B2FFF712FF010089B2062901D1002011E000AA002180B20C2342
:2075E0003C4C03FB0040406804F007FF9DF80000002802D14FF6FF7000E0002016BD4FF6C7
:20760000FF70704780B500218DF8001000AA002180B205F017F99DF80000002802D14FF682
:20762000FF7000E0002002BD30B58BB0002409A805F04EFAFFF709FFFFF720FF00200400B3
:2076400040E009A80890032007900020069000200590A4B228201E4900FB0410008C049068
:20766000A4B228201A4900FB0410C0690390A4B22820174900FB041080690290A4B2282018
:20768000134900FB041040690190A4B22820104900FB0410007C00900023A4B228200C491D
:2076A00000FB0410C268A4B22820094900FB04108168A4B22820064D00FB0450406805F0CC
:2076C000C1FE641CA4B2072CBBD30BB030BD000050030020F007002038080020D4320108B3
:2076E00080B500A805F09FFB01BD50F8041B61B150F8042BD30744BFA9F101039A18002320
:2077000042F8043B091FFAD1EFE7704738B5DFF8EC55002404E0A868804705F21C05641CF4
:20772000A4B22E2CF7D30020DFF8D4150880DFF8E816088006F0A0FF31BD38B50400DFF8BF
:20774000BC5500F02BF8A4B2FF2C0CD1DFF8CC06007878280BD2DFF8C4060078401CDFF8BD
:20776000BC16087003E0DFF8B40600210170002002E005F21C05401C80B22E280CD2DFF806
:20778000801509882A889142F3D1200080B2E96888474FF6FF7000E0002032BD70B500241C
:2077A000DFF85855DFF858050088DFF86C160988884223D0002602E005F21C05761CB6B2C8
:2077C0002E2E1BD2DFF8380500882988884202D128698047641CDFF840060088298888427E
:2077E00002D168698047641CE4B2022CE4D3DFF82806DFF80C1509880180FFE770BD10B53C
:207800000FF2A474FFF7CAFFDFF810060078782839D3DFF8EC0400880E2834D0DFF8E0043B
:2078200000880F282FD0DFF8D804008810282AD0DFF8CC040088002825D0DFF8C4040088AA
:20784000012820D0DFF8B80400880C281BD0DFF8D00500780E2804D1DFF8A4040E21018077
:207860000DE0DFF8BC0500780F2804D1DFF890040F21018003E0DFF8880400210180DFF824
:207880009C0500210170002002E004F21C04401C80B22E280AD2DFF868140988228891427C
:2078A000F3D1A06980474FF6FF7000E0002010BDDFF84C1408807047DFF8440400887047DF
:2078C00010B584B0040008000A280DD20A2200A907F003F8302020702E2060703020A0706D
:2078E0009DF80000E07005E1B0F10A015A290ED20A2200A906F0F1FF302020702E206070F5
:207900009DF80000A0709DF80100E070F2E0B0F164014FF4617291420FD20A2200A906F06F
:20792000DCFF9DF8000020702E2060709DF80100A0709DF80200E070DCE0A0F2E83142F201
:207940002832914212D20A2200A906F0C6FF9DF8000020709DF8010060702E20A0709DF808
:207960000200E0709DF803002071C3E042F21071411ADFF80826914215D20A2200A906F04F
:20798000ACFF9DF8000020709DF8010060709DF80200A0702E20E0709DF8030020719DF8AE
:2079A00004006071A6E0DFF8D815411ADFF8D425914218D20A2200A906F08FFF9DF80000D2
:2079C00020709DF8010060709DF80200A0709DF80300E0702E2020719DF8040060719DF844
:2079E0000500A07186E0DFF8A015411ADFF89C2591421BD20A2200A906F06FFF9DF80000FE
:207A000020709DF8010060709DF80200A0709DF80300E0709DF8040020712E2060719DF803
:207A20000500A0719DF80600E07163E0DFF86015411ADFF8602591421BD20A2200A906F073
:207A40004CFF9DF8000020709DF8010060709DF80200A0709DF80300E0709DF80400207197
:207A60009DF8050060712E20A0719DF80600E07140E0DFF82415411ADFF82025914219D2EB
:207A80000A2200A906F029FF9DF8000020709DF8010060709DF80200A0709DF80300E070D9
:207AA0009DF8040020719DF8050060719DF80600A0711FE0DFF8E81488421BD30A2200A926
:207AC00006F00BFF9DF8000020709DF8010060709DF80200A0709DF80300E0709DF80400F3
:207AE00020719DF8050060719DF80600A0719DF80700E0711FBD80B5022200A91F2000F0E4
:207B000030FE01220DF102011E2000F02AFEDFF894040078012818D19DF80000012803D033
:207B20009DF80000022805D1BDF802004FF6FF7188420AD10221002006F04BFF0020FFF706
:207B4000B7FEDFF8B80A0121018001BD80B500200090042200A92B2000F003FE009843F2B9
:207B6000F501084242D0DFF8B80200780E283DD0DFF8AC0200780F2838D0DFF8A402007836
:207B800006281DD0DFF8980200780A2818D0DFF890020078072813D0DFF8840200780828CF
:207BA0000ED0DFF87C020078092809D0DFF8700200780B2804D0DFF8680200780C280DD17D
:207BC000DFF83C0A4FF6FF7101800120FFF770FEDFF8280A4FF4FA71018007E00120FFF797
:207BE00067FEDFF8180A4FF4FA7101800098C00403D5DFF8100A01210170DFF8080A0078DF
:207C0000012809D0009850F400500090042200A92B2000F0CBFD08E0009830F40050009050
:207C2000042200A92B2000F0C1FD01BDDFF8D80900210170DFF8D40900210170DFF8D0097E
:207C4000002101707047DFF8C009012101707047DFF8B809022101707047DFF8B00901215C
:207C600001707047DFF8A409002101707047DFF8A009022101707047DFF89409002101703E
:207C80007047002008E0C0B23E21DFF8882901FB002100228A87401CC0B20A28F3D37047FF
:207CA000002008E0C0B21221DFF86C2901FB002100224A74401CC0B20C28F3D3704770B50A
:207CC00004000D00160028222021DFF8500901F02FFFF6B232002900DFF8400902F0C1FBD2
:207CE00001220021F6B2DFF83409301801F020FF2100DFF8280906F021FF70BDA87F000891
:207D00002E87002000B591B00020009001A801F076F804A9002000F06BFF9DF811000128EA
:207D200002D1002007F0E6F8DFF8F40804210170DFF8EC08AA210171DFF8E408552101725E
:207D40000822DFF8E018DFF8E00802F08AFB1022DFF8D818DFF8D80802F083FB2022DFF8BB
:207D6000D418DFF8D40802F07CFBDFF8B408DFF8CC18097880F8B910DFF8A408DFF8C018B9
:207D800009684163DFF8B80800680D9907F03AFADFF88C18886305A9DFF8A80801F0CEFAAA
:207DA00001A9DFF8A40801F0C9FADFF874080B2180F8B81000AA01A905A801F07CF9DFF8E5
:207DC00060080099C1640322DFF88018222000F0C8FC0022DFF87818062000F0C2FC002274
:207DE000DFF87018002000F0BCFC0020002108000CE0C0B2DFF8281811EB4001C0B2DFF818
:207E0000582832F81020A1F85820401CC0B23028EFD311B000BD0000308700200D88002085
:207E2000DE0900202DE9F04184B004000D005FF000080026002700A800F0E1FFBDF80000DE
:207E4000642190FBF1F201FB12004F499DF8022042F210735A4301FB00209DF80310642234
:207E600002FB01009DF80510081880469DF80500401C00FB08F8DFF8E40710EB08000600B8
:207E8000DFF8DC0710EB080007000A20B6FBF0F100FB1160303020700A20B6FBF0F00A2120
:207EA000B0FBF1F201FB1200303060706420B6FBF0F00A21B0FBF1F201FB12003030A070AA
:207EC0004FF47A70B6FBF0F00A21B0FBF1F201FB12003030E07042F21070B6FBF0F00A21FD
:207EE000B0FBF1F201FB1200303020712448B6FBF0F00A21B0FBF1F201FB12003030607100
:207F00000A20B7FBF0F100FB1170303028700A20B7FBF0F00A21B0FBF1F201FB120030304D
:207F200068706420B7FBF0F00A21B0FBF1F201FB12003030A8704FF47A70B7FBF0F00A212A
:207F4000B0FBF1F201FB12003030E87042F21070B7FBF0F00A21B0FBF1F201FB1200303060
:207F600028710748B7FBF0F00A21B0FBF1F201FB120030306871BDE8FF810000905F010072
:207F8000A0860100A0BB0D0040420F004054890080969800804A5D0500E1F50500E9A4352D
:207FA00000CA9A3B1D88002000000000608000204BDB00088FDB000879E6000885E70008E2
:207FC000C5DD000801000000748000206504020897040208F12B0208812C0208D505020809
:207FE0000200000088800020FD5803083F590308CD5F03086560030897590308030000004F
:208000009C80002011CB020853CB0208B7D402082FD5020849CE020804000000B0800020FE
:20802000FDC2030841C3030837C603086BC603086BC3030805000000C480002065E303082E
:2080400097E30308E1E503082DE60308B7E3030806000000D8800020BDD60308F1D6030819
:20806000A3D9030825DA0308C7D70308070000000081002075870308B7870308C58C030872
:20808000078D0308798A03080800000014810020657B0308A77B0308CD8003080F8103086B
:2080A000817E030809000000288100205D6E03089F6E03082774030883740308A170030832
:2080C0000A000000EC80002069E003089BE00308FBE2030861E3030831E103080B000000D1
:2080E0003C810020E574030827750308B17A0308037B0308297703080C0000005081002031
:2081000029AD03086DAD030821B103087FB10308C1AD03080D000000648100200DBF0308DF
:208120004FBF03089DC20308F9C203088DBF03080E00000078810020EDCA03081FCB0308C1
:20814000E7CC030865CE030829CB03080F0000008C8100206DD201089FD2010871030208A8
:20816000B703020869D4010810000000A0810020FDA103083FA2030867A60308E5A6030861
:20818000EFA2030811000000B481002069600308AB6003082D6503088F660308D760030814
:2081A00012000000C881002019BB03085DBB030847BE03087DBE03088DBC03081300000085
:2081C000DC81002055E6030887E60308A5E80308F9E803080FE703081400000068820020C1
:2081E00061F2030893F2030813F4030851F4030813F3030815000000F081002069CE030836
:20820000ADCE0308C9D103081DD2030835CF030816000000987F0020E1F4020823F50208DC
:20822000F1FC020809FE0208B5F7020817000000C07F0020E1910208239202082D9D0208FB
:20824000959E02084D97020818000000D47F002049C002088BC002088DC90208EDCA0208DF
:2082600033C3020819000000E87F0020A99E0208EB9E020859AB0208D9AC020809A3020827
:208280001A000000FC7F00201DFE02085FFE02086D050308C9060308070203081B00000017
:2082A0001080002009B203084BB2030837B60308C1B6030823B403081C0000002480002004
:2082C000D99C03081B9D0308F3A00308EDA103088F9E03081D000000388000206DDD0308A2
:2082E0009FDD0308EFDF03084DE00308E1DE03081E000000707F0020E1C6030823C7030848
:208300000BCA03089DCA0308F9C703081F0000005482002005EE030837EE0308D1EF030832
:208320001DF00308B7EE030820000000847F0020F95003083B510308B9570308E7570308E3
:20834000A951030821000000AC7F002029DA03085BDA0308E9DC030829DD030895DA030803
:208360002200000004820020612E0308A32E0308D73503080D3703084B32030823000000AE
:20838000188200205D9703089F970308699B0308C19C03081F990308240000002C820020B7
:2083A00091EB0308C3EB0308A9ED030801EE03084BEC0308250000004C800020B540020890
:2083C000F7400208735202085D5402083544020826000000E47E0020F12C0208332D020816
:2083E000AF3E0208A14002087130020827000000F87E002071540208A9540208FF650208EF
:20840000F1670208C1570208280000000C7F00201D06040855060408590604085B06040897
:208420005706040829000000207F00205107030893070308850E0308D70F0308F50703084D
:208440002A00000040820020FDE803082FE903083FEB03088DEB0308E1E903082B00000045
:20846000347F002061F0030893F0030807F2030855F20308AFF003082C000000487F00202C
:2084800049B502088BB50208B5BE02082DC0020865B702082D0000005C7F00206D670308E9
:2084A000AF670308B56D0308456E03086568030800B585B06B4801905FF084400090694856
:2084C00003905FF08440029000226749672000F048F965480068654906F006FF2CD862486E
:2084E0000068634903F002FE26D25F48006806F00DFF5FF033325F4B06F030FF07F000F8FA
:2085000000900098029000985B4903F0EFFD06D200985FF0804107F03BF8019009E00098CA
:2085200006F0F4FE554A564B06F018FF06F0E8FF0190019803903AE04B4800684C4906F0CC
:20854000D3FE34D8484800684E4903F0CFFD2ED2454800684C4907F01BF806F0D7FE00226F
:208560004A4B06F0FBFE06F0CBFF00900098484906F0BAFE01D84748009000980290009896
:208580003D4903F0B3FD06D200985FF0804106F0FFFF019009E0009806F0B8FE374A384B7C
:2085A00006F0DCFE06F0ACFF019001980390352101A801F07CFF002201A9342000F0F6F824
:2085C000362100A801F073FF002200A9352000F0EDF8372103A801F06AFF002203A93620C3
:2085E00000F0E4F8382102A801F061FF002202A9372000F0DBF805B000BD0000BA0900201F
:2086000086870020EC0900201588002016880020178800200852002068040020247D002017
:20862000A06700204D7C0020A9670020367C0020B9670020557C00205E6800204C7C002029
:208640000C7C0020DC670020E4670020D0670020F0670020F46700202C7B0020D038030089
:2086600040E20100CDCC0C422C860020000020410100AA423333E33F0100A0419A99999901
:208680009999F13F0100B442000080C20000044001007C4200007C42010002000300040074
:2086A00013000000050006000A0000001400220023002A0007000800090000000B000C00E0
:2086C00016001700180019001B001C001D001E0020002100250026002700280029000000C6
:2086E0000D000E000F0000001000110010B4002304E00C780470401C491C5B1C9342F8D394
:2087000010BC70470021C0B2002812D0022814D011D3042815D012D3062810D00DD3082833
:2087200011D00ED30A2812D00FD30C2813D010D313E0042112E0022110E001210EE0022137
:208740000CE004210AE0322108E00C2106E0082104E0022102E0102100E00021080080B252
:20876000704770B506000C0010000025B6B2224911EBC6018978C0B2814214D1B6B21E4956
:2087800031F83610B6B2B1420DD1C0B2FFF7BAFF0500EDB22A00B6B2174810EBC600416811
:2087A0002000FFF7A3FF2800C0B270BD70B505000E0010000024ADB20F4911EBC501897854
:2087C000C0B2814214D1ADB20B4931F83510ADB2A9420DD1C0B2FFF795FF0400E4B222007E
:2087E0003100ADB2044810EBC5004068FFF77EFF2000C0B270BD0000000000202DE9F0439A
:208800009BB00D0016001F0000245FF000085FF000092A00D2B20DA980B2FFF7A2FF804605
:208820003A00D2B200A9300080B2FFF79AFF81461FFA88F81FFA89F9C84503D003242000BE
:20884000C0B2FCE01FFA88F8424600A90DA801F0D7FD002800F0F180EDB2002D0FD0022D23
:2088600028D019D3042D5DD040D3062D4CD02FD3082D6FD062D3092D00F08880DDE0009826
:208880000D9903F033FC03D201200400C0B202E002200400C0B2D0E0BDF80000BDF83410CC
:2088A000884203D201200400C0B202E002200400C0B2C2E09DF800009DF83410884203D259
:2088C00001200400C0B202E002200400C0B2B4E09DF900009DF93410884203DA01200400B7
:2088E000C0B202E002200400C0B2A6E0BDF80000BDF83410884203D201200400C0B202E040
:2089000002200400C0B298E0BDF90000BDF93410884203DA01200400C0B202E00220040051
:20892000C0B28AE000980D99884203D201200400C0B202E002200400C0B27EE000980D99D1
:20894000884203DA01200400C0B202E002200400C0B272E000200021080000E0401CC0B216
:20896000322812D2C0B200A9415CC0B20DAA825C914201D2012408E0C0B20DA9415CC0B210
:2089800000AA825C9142E9D2022456E00DA800A90A8803889A4201D201244DE002880B88CC
:2089A0009A4201D2022447E08A7883789A4201D2012441E082788B789A4201D202243BE0DC
:2089C000CA78C3789A4201D2012435E0C278CB789A4201D202242FE04A7943799A4201D2A2
:2089E000012429E042794B799A4201D2022423E08A7983799A4201D201241DE082798B7923
:208A00009A4201D2022417E0CA79C3799A4201D2012411E0C279CB799A4201D202240BE007
:208A20008A6883689A4201D2012405E080688968884201D20224FFE7FFE72000C0B21BB0DB
:208A4000BDE8F083C0B2012802D37FF0040007E0C0B23421844A01FB002000214170002091
:208A60007047C0B2012802D37FF004000EE0C0B234227D4B02FB00320968D161C0B2342145
:208A8000794A01FB0020002181700020704700B502000B00D2B2012A02D37FF004001CE059
:208AA0001868596806F020FC01D858681860D2B234206D4900FB021001218170D2B23420CC
:208AC000694900FB02105968C161D2B23420664900FB021019680162002000BDC0B2012804
:208AE00002D37FF0040015E0C0B234225E4B02FB003202239370C0B234225B4B02FB0032D4
:208B00004B68D361C0B23422574B02FB00300968C162002070473EB504000D00E4B2012CA5
:208B200002D37FF0040029E000A800F068F94FF6FF71884220D1E4B234204B4900FB0410EE
:208B400003218170E4B23420474900FB041003218170E4B23420444900FB041010300ECDC1
:208B60000EC00C3D0C38E4B234203F4900FB0410E968C161002001E07FF005003EBD80B501
:208B800001000020C9B23422374B02FB01325278022A07D0C9B23422334B02FB013252781B
:208BA000032A23D1C9B234202F4A00FB01208078002805D0022808D011D303280AD013E05D
:208BC0000800C0B206F0A6F910E00800C0B206F03FFA0BE00800C0B206F09CFA06E008000E
:208BE000C0B206F0CEF901E07FF0050040B202BD10B50B003422C0B234211B4C01FB0041AF
:208C0000180001F02EFC002010BDC0B23421164A01FB00200521417000207047C0B234217C
:208C2000114A01FB00200621417000207047C0B234210D4A01FB002000214170002070472B
:208C400010B5C0B23421084A01FB002100224A7034220021C0B23423034C03FB004000F080
:208C600067FF002010BD0000887C002080B5DFF8E4090078002801D106F0CCFC06F0EFFC73
:208C8000DFF8D4094FF6FF710180DFF8CC09008802BDC9B20A2291FBF2F2D2B212010270D7
:208CA000C9B20A220378CB1891FBF2F102FB11310170704710B586B00400DFF89C090088D6
:208CC0004FF6FF71884240F09780DFF88809007800281FD12088ADF80000A0788DF80200EA
:208CE000E0788DF8030020798DF8040060798DF80500A0798DF80600E0798DF8070006F090
:208D0000AFFCDDE9000106F0CDFC06F0A8FC4FF6FF7072E02088ADF80000A0788DF8020096
:208D2000E0788DF803009DF803209DF80210BDF8000006F026FD8DF8040060798DF805003A
:208D4000A0798DF80600E0798DF807000922002102A800F0EDFE9DF8020010F01F010DF104
:208D60000F00FFF796FFBDF80000B0F5FA6F08D3BDF8000010F13001C9B204A8FFF789FF2F
:208D80000DE0BDF80000B0F16C01C9B204A8FFF780FF9DF80F0050F080008DF80F009DF8FA
:208DA0000400072803D100208DF80E0003E09DF804008DF80E009DF803100DF10D00FFF741
:208DC00068FF9DF8051003A8FFF763FF9DF806100DF10B00FFF75DFF9DF807100DF10A00C5
:208DE000FFF757FF07220DF10A01DFF8780901F0F2FA4FF6FF7000E0002006B010BD10B5C4
:208E000086B00400DFF8500800884FF6FF71884240F0A980DFF83C080078002803D100A852
:208E200006F0E8FC87E0092202A95FF0405001F0BDFA9DF80F00000601D5132000E01420CD
:208E400064214843ADF80000BDF800009DF81010C9B20909C9B20A2202FB0100ADF800001C
:208E6000BDF800009DF8101011F00F010818ADF800009DF80F00C0F300100A2148438DF810
:208E800002009DF802009DF80F1011F00F0108188DF802009DF80E000721084204D09DF84F
:208EA0000E0010F0070000E007208DF804009DF80D00C0F301100A2148438DF803009DF8D4
:208EC00003009DF80D1011F00F0108188DF803009DF80C00C0F301100A2148438DF805007F
:208EE0009DF805009DF80C1011F00F0108188DF805009DF80B00C0F302100A2148438DF8CC
:208F000006009DF806009DF80B1011F00F0108188DF806009DF80A00C0F302100A2148432A
:208F20008DF807009DF807009DF80A1011F00F0108188DF80700BDF8000020809DF80200B1
:208F4000A0709DF80300E0709DF8040020719DF8050060719DF80600A0719DF80700E071EB
:208F60004FF6FF7000E0002006B010BD0A8803889A4201D2022042E002880B889A4201D2DE
:208F800001203CE08A7883789A4201D2022036E082788B789A4201D2012030E0CA78C37856
:208FA0009A4201D202202AE0C278CB789A4201D2012024E04A7943799A4201D202201EE037
:208FC00042794B799A4201D2012018E08A7983799A4201D2022012E082798B799A4201D2DA
:208FE00001200CE0CA79C3799A4201D2022006E0C079C979884201D2012000E0002070473E
:209000000A7803789A4201D2022012E002780B789A4201D201200CE04A7843789A4201D2AB
:20902000022006E040784978884201D2012000E00020704770B504000E0015000020288026
:2090400031002000FFF7DCFF01280CD130782178401A3C21727801FB00206178401A28800F
:209060004FF6FF700BE031002000FFF7C9FF002804D1002028804FF6FF7000E0002070BD9C
:209080004A7902708A794270CA79827089684160704710B584B0040000A8FFF7B0FE0028F7
:2090A00001D1002005E000A92000FFF7E9FF4FF6FF7004B010BD2DE9F04104000D0016008F
:2090C0001C275FF01E080020306029002000FFF74DFF012873D12088401C2988884204DBD2
:2090E000A078401CA978884201DA002073E028882188491C884207D1A078401CA9780C3191
:20910000884201DA002066E028884FF4C87190FBF1F201FB120000280FD02888642190FBD5
:20912000F1F201FB1200002809D02888042190FBF1F202FB1102002A01D11D2700E01C2787
:20914000A078012811D0A07803280ED0A07805280BD0A078072808D0A078082805D0A07858
:209160000A2802D0A0780C2802D15FF01F0806E0A078022801D1B84601E05FF01E08288858
:209180002188401A0C21AA7801FB0020A178401A5FFA88F8E97808FB0010E178401A1821B5
:2091A0006A7901FB00206179401A3C21AA7901FB0020A179401A30604FF6FF700BE0290014
:2091C0002000FFF7D3FE002804D1002030604FF6FF7000E00020BDE8F0812DE9F0410400E6
:2091E0000D0016001C275FF01E080020306029002000FFF7BBFE012879D12088401C2988C4
:20920000884204DBA078401CA978884201DA002079E028882188491C884207D1A078401C1E
:20922000A9780C31884201DA00206CE028884FF4C87190FBF1F201FB120000280FD0288860
:20924000642190FBF1F201FB1200002809D02888042190FBF1F202FB1102002A01D11D2779
:2092600000E01C27A078012811D0A07803280ED0A07805280BD0A078072808D0A078082801
:2092800005D0A0780A2802D0A0780C2802D15FF01F0806E0A078022801D1B84601E05FF020
:2092A0001E0828882188401A0C21AA7801FB0020A178401A5FFA88F8E97808FB0010E17851
:2092C000401A18216A7901FB00206179401A3C21AA7901FB0020A179401A3C21EA7901FBFC
:2092E0000020E179401A30604FF6FF700BE029002000FFF73BFE002804D1002030604FF601
:20930000FF7000E00020BDE8F08110B584B0040000A8FFF774FDBDF8000020809DF80200D0
:20932000A0709DF80300E0709DF8050020719DF8060060719DF80700A0711FBD0A88028001
:209340008A788270CA78C2704A7902718A794271C97981717047F0B4002301888478C27848
:2093600045798679C079A1F2B277BFB2822F5CD2631EDBB20C2B58D2531EDBB21F2B54D20E
:20938000EDB2182D51D2F6B23C2E4ED2C0B23C284BD2E4B2042C08D0E4B2062C05D0E4B2D0
:2093A000092C02D0E4B20B2C07D1D2B21F2A01D3002330E04FF6FF732DE0E4B2022C28D1AC
:2093C00089B24FF4C87091FBF0F300FB131000280FD089B2642091FBF0F300FB13100028CF
:2093E0000FD089B2042091FBF0F303FB1013002B07D1D2B21E2A01D300230CE04FF6FF7336
:2094000009E0D2B21D2A01D3002304E04FF6FF7301E04FF6FF734FF6FF709BB2834202D1D5
:209420004FF6FF7002E0002000E00020F0BC704770B504000D0000260A222900208805F0C5
:2094400007FA0A22DFF82013A07805F001FA0A22DFF81813E07805F0FBF92D202871DFF8A1
:20946000080300786871DFF800034078A8712D20E871DFF8F80200782872DFF8F0024078DB
:2094800068722020A8722020E8720A22DFF8E012207905F0DDF90A22DFF8D812607905F0EA
:2094A000D7F90A22DFF8D012A07905F0D1F9DFF8C00200782873DFF8B802407868733A20F5
:2094C000A873DFF8B0020078E873DFF8A802407828743A206874DFF8A0020078A874DFF826
:2094E00098024078E874002028750020060007E0B6B2132E03D1A87CE8743020A874761CF9
:20950000B6B2142E23D2B6B2705D0028F7D1B6B2062E04D16879A87130206871EFE7B6B2B5
:20952000092E04D1287A687230202872E7E7B6B20D2E04D1287B687330202873DFE7B6B2DC
:20954000102ED5D1E87B28743020E873D7E770BD70B504000D0000260A222900208805F044
:2095600077F90A228549A07805F072F90A228449E07805F06DF92D2028718048007868715E
:209580007E484078A8712D20E8717D48007828727B48407868722020A8722020E8720A2242
:2095A0007849607905F054F90A227749A07905F04FF90A227549E07905F04AF971480078E1
:2095C00028737048407868733A20A8736E480078E8736D48407828743A2068746B4800783D
:2095E000A8746A484078E874002028750020060007E0B6B2132E03D1A87CE8743020A87456
:20960000761CB6B2142E23D2B6B2705D0028F7D1B6B2062E04D16879A87130206871EFE78A
:20962000B6B2092E04D1287A687230202872E7E7B6B20D2E04D1287B687330202873DFE7DB
:20964000B6B2102ED5D1E87B28743020E873D7E770BD0000D9870020FA8600203EB5040012
:20966000002500A8FFF7CBFB0A222100BDF8000005F0EEF80A2246499DF8020005F0E8F85D
:209680000A2244499DF8030005F0E2F84048007820713F48407860713E480078A0713D4875
:2096A0004078E071202020720A223B499DF8050005F0CEF80A2239499DF8060005F0C8F8CC
:2096C0000A2237499DF8070005F0C2F832480078607231484078A0723A20E0722F480078F1
:2096E00020732E48407860733A20A0732C480078E0732B4840782074002060740020050052
:2097000007E0ADB2102D03D1E07B20743020E0736D1CADB2112D23D2ADB2285D0028F7D171
:20972000ADB2052D04D12079607130202071EFE7ADB2072D04D1A079E0713020A071E7E7A1
:20974000ADB20A2D04D1607AA07230206072DFE7ADB20D2DD5D1207B607330202073D7E77C
:2097600037BD0000020000300287002004870020FC860020FE860020008700200C870020CF
:209780000E87002006870020088700200A870020168700201887002010870020128700201B
:2097A0001487002038B504000D002000FFF727FBA07969780818A071607929780818607122
:2097C000A0793C2805D3A0793C38A0716079401C60716079182866D3607918386071E078EC
:2097E000401CE070A078012811D0A07803280ED0A07805280BD0A078072808D0A0780828F3
:2098000005D0A0780A2802D0A0780C2809D1E07820283FD3E0781F38E070A078401CA070FC
:2098200038E0A07802282CD120884FF4C87190FBF1F201FB120000280FD02088642190FB72
:20984000F1F201FB1200002811D02088042190FBF1F202FB1102002A09D1E0781E2819D335
:20986000E0781D38E070A078401CA07012E0E0781D280FD3E0781C38E070A078401CA07076
:2098800008E0E0781F2805D3E0781E38E070A078401CA070A0780D2805D3A0780C38A07056
:2098A0002088401C208031BD38B5C0B2032812D201230122C0B20321204C01FB0041897821
:2098C000C0B203241D4D04FB0050407806F010F84FF6FF7000E0002032BD10B5C0B203287B
:2098E00011D20122C0B20321144B01FB00318978C0B20323114C03FB0040407806F079F8ED
:209900004FF6FF7000E0002010BD10B5C0B2032811D20022C0B20321084B01FB0031897848
:20992000C0B20323054C03FB0040407806F061F84FF6FF7000E0002010BD000064090020EB
:2099400080B5354A3548008835494118012006F0A3F93248008840F22621884204D22F4832
:209960000088401C2D4908802C48008840F22621884202D129480021018001BD70477047B4
:2099800080B526480021018023480021018001200090002308225FF4E131012006F030F9D2
:2099A000002801D100200BE01E4B1F4A1F49012006F084F9002801D1002001E04FF6FF7025
:2099C00002BD10B50C0022000100012006F04DF9002801D1002000E0200010BD0E48002119
:2099E00001800E4800210180704711480088704780B200280BD00E4800884FF47A71884294
:209A000008D20B480088401C0949088002E008480021018070470000DA860020D8860020D2
:209A2000745400207F9900087D99000841990008AC090020FF2212EAD05C1DBF12EAD15304
:209A4000944593422BE09C44D30780EA01021A4043EA002043EA0121A1FB0030410038BF2C
:209A600040007CF17F010BDBFE294ADA5B0842EAC15153EA006373F1004C51EB1020704774
:209A8000D1F1080CDCF120012FDB5B0810FA01F10B4373F1004120FA0CF05041704794456F
:209AA0001CBF02EAD153934280EA010202F000421DD0400019D0490017D05BB9634514D05F
:209AC0000902B1FA81F39940BCEB030CC00140F00040C1E70002B0FA80FC10FA0CF0B3EB28
:209AE0000C0CC90141F00041B6E71000704740000AD0490008D010F1807F94BF11F1807F1F
:209B000002E042F0FF407047D043704740000DD2010E7F390AD4D1F11F0104D4C00140F002
:209B20000040C84070477FF0000070470020704710B5040010000A000100200006F0D0F867
:209B4000200010BD80B5C0B2012807D2C0B214210B4A01FB00200069804700E00A2002BD5E
:209B600080B502000800D2B2012A07D280B2D2B21421034B01FB0231C968884701BD0000F8
:209B800030B1020838B50400002020801C2006F0E4FE05001C2006F0E0FE6560A060606873
:209BA000A1688161606800214161A06800218161A0686168416131BD0088704700881428C0
:209BC00002D14FF6FF7000E0002070470088002802D14FF6FF7000E000207047F8B50400A8
:209BE0000D00002600272800FFF7E8FF002807D02900002000F03BF8002801D1002035E06C
:209C0000DFF83005FFF7D8FF0600DFF8280540688069002701E080697F1CBFB2B6B2B74272
:209C200006D2217802789142F5D14FF6FF701DE01C2006F092FE0600002E01D1002015E012
:209C4000207830700822A11CB01C00F00AFC68688069B06168688069466168687061686888
:209C600086612888401C28804FF6FF70F2BD70B505000C002000FFF7A9FF002801D00020D9
:209C800037E02000FFF798FF002D10D12088401E2080A168A0684069A060A0680022826185
:209CA000080006F082FF00214FF6FF7021E061688E69002101E0B669491C814218DA2A78B2
:209CC00033789A42F7D12088401E2080A81CB11C082202F043FA7069B1698161B0697169DD
:209CE0004161300006F061FF00264FF6FF7000E0002070BD70B4002314E0DBB2022493FBB9
:209D0000F4F455006D1EDBB2ED1A6D5C5600761EDBB2F61A761816F8016C15EB0615303D06
:209D200025549B1CDBB2B3EB420FE6D370BC704730B4002315E0541EDBB2E41A645CE4B28C
:209D400024093034DBB200F81340541EDBB2E41A645C14F00F043034DBB210EB43056C70B6
:209D60005B1CDBB29342E6D330BC7047002200E0521CD2B28A420ED200230A2B01D30020C2
:209D80000BE04B1ED2B29B1A1B5C13F00F030A2BEEDB002001E04FF6FF707047002100E03F
:209DA000491CC9B2062907D2C9B20A5C303AD2B20A2AF5D3002001E04FF6FF707047C0B212
:209DC000642190FBF1F201FB1200C0B20A2190FBF1F10901C0B20A2290FBF2F302FB130050
:209DE00001430800C0B270470021DFF84C23B0FBF2F251EA0271DFF84023B0FBF2F302FB83
:209E00001302DFF83833B2FBF3F251EA0261DFF82C23B0FBF2F302FB1302DFF82433B2FB18
:209E2000F3F251EA0251DFF81823B0FBF2F302FB130242F21073B2FBF3F251EA024142F200
:209E40001072B0FBF2F302FB13024FF47A73B2FBF3F251EA02314FF47A72B0FBF2F302FBF2
:209E600013026423B2FBF3F251EA02216422B0FBF2F302FB13020A23B2FBF3F251EA021121
:209E80000A22B0FBF2F302FB130211430800704710B4002211E0D2B211F812301B01D2B29B
:209EA0001354D2B2135CD2B211EB4204647814F00F042343D2B21354521CD2B2082AEAD35D
:209EC00010BC704730B400220EE0C9B24B1ED2B29B1A1B5CC9B24C1ED2B2A41AD2B2155C5B
:209EE0002554D2B21354521CC9B2022391FBF3F3D2B29A42E9DB30BC70472DE9F0438DB031
:209F000004000D0017001E0000A8342102F05EF9F6B2032EC0F097803222002100A8FFF702
:209F200007FE3F68380007F0A3F8844901FB00F884483900FFF77EFD8146404602F040F8FD
:209F40000100484605F05EF907F092F8002800D5404203009846380007F08AF80200434609
:209F60000FF2382100A802F011F82900EDB2072D00D30621002000E0401CC0B2F6B2B21EA8
:209F800090423BDAC0B200AA825C2E2AF4D1EDB2002D09D1C0B200A920224254C0B200A90F
:209FA00040182021417029E0C0B2C9B20A1800ABD21820235370C0B2C9B20A1800ABD21800
:209FC00020239370C0B2C9B20A1800ABD2182023D370C0B2C9B20A1800ABD21820231371A6
:209FE000C0B2C9B20A1800ABD21820235371C0B2C9B2081800A9401820218171F6B200A825
:20A00000301810F8030C2E2805D1F6B200A83018202100F8031CF6B200A83018202100F8F4
:20A02000021CF6B200A83018202100F8011C002005E0C0B2C0B200A9415C0155401CC0B2C1
:20A04000F6B2B042F5D30DB0BDE8F08330B4002308E0DBB25C5C14F00F043734DBB200F88E
:20A0600013405B1CDBB2D2B2934227D2DBB25C5CE4B224090A2C09D2DBB210EB4304DBB2C2
:20A080005D5CEDB22D093035657008E0DBB210EB4304DBB25D5CEDB22D0937356570DBB258
:20A0A0005C5C14F00F040A2CD3DADBB25C5C14F00F043034DBB200F81340D2E730BC7047FA
:20A0C00010B400220BE092B2130A1202DBB2047863400FF2D00434F813305A40401C0B0049
:20A0E000591E9BB2002BEED1100080B210BC704710B415E0144A128892B2120A124B1B88DC
:20A100001B02114C2380104B1B88D2B2047862400FF2900434F812205A400B4B1A80401CA9
:20A120000A00511E92B2002AE4D10748008810BC704700009C8400208096980040420F00AA
:20A14000A0860100002474495087002010B5ADF5FE6D4FF40050002415E0A4B24FF4806009
:20A1600000FB04F010F500504FF48062FBA906F0ADFF4FF48061FBA8FFF7A2FFA4B200A9D3
:20A1800021F81400641CA4B2FD2CE6D34FF4FD7100A8FFF795FF0DF5FE6D10BD25642E25E1
:20A1A0003036640000002110422063308440A550C660E770088129914AA16BB18CC1ADD164
:20A1C000CEE1EFF13112100273325222B5529442F772D662399318837BB35AA3BDD39CC383
:20A1E000FFF3DEE36224433420040114E664C774A44485546AA54BB528850995EEE5CFF53F
:20A20000ACC58DD55336722611163006D776F6669556B4465BB77AA719973887DFF7FEE702
:20A220009DD7BCC7C448E5588668A7784008611802282338CCC9EDD98EE9AFF9488969993E
:20A240000AA92BB9F55AD44AB77A966A711A500A333A122AFDDBDCCBBFFB9EEB799B588B82
:20A260003BBB1AABA66C877CE44CC55C222C033C600C411CAEED8FFDECCDCDDD2AAD0BBD3E
:20A28000688D499D977EB66ED55EF44E133E322E511E700E9FFFBEEFDDDFFCCF1BBF3AAF02
:20A2A000599F788F8891A981CAB1EBA10CD12DC14EF16FE18010A100C230E320045025401C
:20A2C00046706760B9839893FBA3DAB33DC31CD37FE35EF3B1029012F322D2323542145282
:20A2E00077625672EAB5CBA5A89589856EF54FE52CD50DC5E234C324A0148104667447643E
:20A3000024540544DBA7FAB79987B8975FE77EF71DC73CD7D326F2369106B0165766767601
:20A32000154634564CD96DC90EF92FE9C899E9898AB9ABA94458654806782768C018E1083D
:20A340008238A3287DCB5CDB3FEB1EFBF98BD89BBBAB9ABB754A545A376A167AF10AD01A81
:20A36000B32A923A2EFD0FED6CDD4DCDAABD8BADE89DC98D267C076C645C454CA23C832C3D
:20A38000E01CC10C1FEF3EFF5DCF7CDF9BAFBABFD98FF89F176E367E554E745E932EB23E01
:20A3A000D10EF01E80B506F09AFE02BD70B504000D00160000210020FDF7D4F83200290086
:20A3C000200006F0A6FE0028F8D00020FDF7F6F84FF6FF7070BD70B504000D001600002183
:20A3E0000020FDF7BFF832002900200006F07CFE0028F8D00020FDF7E1F84FF6FF7070BDE9
:20A400000300002013F0030F09D0521E22BF13F8010B11F801CBB0EB0C00F3D07047121F9C
:20A4200022BF53F8040B51F804CB6045F7D0121D0AD200BA9CFA8CFCB0EB0C0038BF6FF07D
:20A44000000088BF01207047521E22BF13F8010B11F801CBB0EB0C00F6D0521C08BF1046A8
:20A46000704710B50400200001F078FE200010BD10B50B000024DBB2492B01D2002801D126
:20A48000002411E0DBB2DFF8A81E51F833200100DBB20FF6A46010EBC3004068FFF786FF69
:20A4A000002801D04FF6FF74200080B210BD10B50B000024DBB2492B01D2002801D10024E6
:20A4C00011E0DBB20FF6706151F833200100DBB20FF6646010EBC3004068FFF77CFF002836
:20A4E00001D04FF6FF74200080B210BD30B585B000AC02250320207001212000FFF7D7FF06
:20A500002A00D2B221002120FEF750F903251020208002212000FFF7CAFF2A00D2B2210024
:20A520002220FEF743F902250120207003212000FFF7BDFF2A00D2B221002320FEF736F9A4
:20A5400002250020207004212000FFF7B0FF2A00D2B221002420FEF729F902250120207038
:20A5600005212000FFF7A3FF2A00D2B221002520FEF71CF902250020207006212000FFF7CB
:20A5800096FF2A00D2B221002620FEF70FF902250020207007212000FFF789FF2A00D2B2C9
:20A5A00021002720FEF702F90425DFF8880D206008212000FFF77BFF2A00D2B2210029205D
:20A5C000FEF7F4F800255FF07E50206009212000FFF76DFF2A00D2B221003820FEF7E6F832
:20A5E00000255FF07E5020600A212000FFF75FFF2A00D2B221003920FEF7D8F800255FF099
:20A600007E5020600B212000FFF751FF2A00D2B221003A20FEF7CAF800255FF07E502060B8
:20A620000C212000FFF743FF2A00D2B221003B20FEF7BCF800255FF07E5020600D212000B2
:20A64000FFF735FF2A00D2B221003C20FEF7AEF800255FF07E5020600E212000FFF727FFDD
:20A660002A00D2B221003D20FEF7A0F800255FF07E5020600F212000FFF719FF2A00D2B253
:20A6800021003E20FEF792F800255FF07E50206010212000FFF70BFF2A00D2B221003F207B
:20A6A000FEF784F80B25062020700020607011212000FFF7FCFE2A00D2B221004020FEF7ED
:20A6C00075F80225022020701F212000FFF7EFFE2A00D2B221004E20FEF768F80B251620F9
:20A6E00020700020607012212000FFF7E0FE2A00D2B221004120FEF759F802250420207062
:20A7000020212000FFF7D3FE2A00D2B221004F20FEF74CF80B250320207000206070132193
:20A720002000FFF7C4FE2A00D2B221004220FEF73DF802250320207021212000FFF7B7FEFF
:20A740002A00D2B221005020FEF730F80B25042020700020607014212000FFF7A8FE2A00AE
:20A76000D2B221004320FEF721F802250420207022212000FFF79BFE2A00D2B221005120B6
:20A78000FEF714F80B25052020700020607015212000FFF78CFE2A00D2B221004420FEF7E5
:20A7A00005F802250120207023212000FFF77FFE2A00D2B221005220FDF7F8FF0B2506206B
:20A7C00020700020607016212000FFF770FE2A00D2B221004520FDF7E9FF02250220207055
:20A7E00024212000FFF763FE2A00D2B221005320FDF7DCFF0B25072020700020607017217D
:20A800002000FFF754FE2A00D2B221004620FDF7CDFF02250320207025212000FFF747FE60
:20A820002A00D2B221005420FDF7C0FF0B25082020700020607018212000FFF738FE2A009B
:20A84000D2B221004720FDF7B1FF02250420207026212000FFF72BFE2A00D2B221005520A3
:20A86000FDF7A4FF0B25092020700020607019212000FFF71CFE2A00D2B221004820FDF7D3
:20A8800095FF02250120207027212000FFF70FFE2A00D2B221005620FDF788FF0B250A20C7
:20A8A0002070002060701A212000FFF700FE2A00D2B221004920FDF779FF0225022020704C
:20A8C00028212000FFF7F3FD2A00D2B221005720FDF76CFF0B250B202070002060701B216D
:20A8E0002000FFF7E4FD2A00D2B221004A20FDF75DFF02250320207029212000FFF7D7FDCA
:20A900002A00D2B221005820FDF750FF0B250C202070002060701C212000FFF7C8FD2A008F
:20A92000D2B221004B20FDF741FF0225042020702A212000FFF7BBFD2A00D2B22100592097
:20A94000FDF734FF0B250D202070002060701D212000FFF7ACFD2A00D2B221004C20FDF7C7
:20A9600025FF0225012020702B212000FFF79FFD2A00D2B221005A20FDF718FF0B250E202B
:20A980002070002060701E212000FFF790FD2A00D2B221004D20FDF709FF02250120207045
:20A9A0002C212000FFF783FD2A00D2B221005B20FDF7FCFE0025DFF8E80C20602D2120009E
:20A9C000FFF775FD2A00D2B221002C20FDF7EEFE0025DFF8D00C20602E212000FFF767FDF3
:20A9E0002A00D2B221002D20FDF7E0FE0025DFF8B80C20602F212000FFF759FD2A00D2B2BF
:20AA000021002E20FDF7D2FE0025DFF8A00C206030212000FFF74BFD2A00D2B221002F200E
:20AA2000FDF7C4FE0025DFF8880C206031212000FFF73DFD2A00D2B221003020FDF7B6FEE7
:20AA40000025DFF8700C206032212000FFF72FFD2A00D2B221003120FDF7A8FE0025DFF8B3
:20AA6000580C206033212000FFF721FD2A00D2B221003220FDF79AFE0025DFF8400C2060F5
:20AA800034212000FFF713FD2A00D2B221003320FDF78CFE0025DFF8280C20603521200075
:20AAA000FFF705FD2A00D2B221003420FDF77EFE00255FF08440206036212000FFF7F7FCF3
:20AAC0002A00D2B221003520FDF770FE0025DFF8F00B206037212000FFF7E9FC2A00D2B278
:20AAE00021003620FDF762FE00255FF08440206038212000FFF7DBFC2A00D2B22100372067
:20AB0000FDF754FE04250020206039212000FFF7CEFC2A00D2B221005C20FDF747FE032540
:20AB20007D2020803A212000FFF7C1FC2A00D2B221005D20FDF73AFE04250A2020603C2102
:20AB40002000FFF7B4FC2A00D2B221005F20FDF72DFE03250A2020803D212000FFF7A7FCB9
:20AB60002A00D2B221006020FDF720FE0225012020703E212000FFF79AFC2A00D2B22100C2
:20AB80006120FDF713FE0225212020703F212000FFF78DFC2A00D2B221006220FDF706FEEF
:20ABA00002250220207040212000FFF780FC2A00D2B221006320FDF7F9FD022504202070B2
:20ABC00041212000FFF773FC2A00D2B221006420FDF7ECFD02250020207042212000FFF70E
:20ABE00066FC2A00D2B221006520FDF7DFFD02250120207043212000FFF759FC2A00D2B27A
:20AC000021006620FDF7D2FD0025DFF8B80A206044212000FFF74BFC2A00D2B22100672074
:20AC2000FDF7C4FD02250120207048212000FFF73EFC2A00D2B221006920FDF7B7FD05B019
:20AC400030BD30B585B000AC022501212000FFF70FFC2A00D2B221002120FDF7A7FD032507
:20AC600002212000FFF704FC2A00D2B221002220FDF79CFD022503212000FFF7F9FB2A007E
:20AC8000D2B221002320FDF791FD022504212000FFF7EEFB2A00D2B221002420FDF786FD75
:20ACA000022505212000FFF7E3FB2A00D2B221002520FDF77BFD022506212000FFF7D8FB9C
:20ACC0002A00D2B221002620FDF770FD022507212000FFF7CDFB2A00D2B221002720FDF7C7
:20ACE00065FD042508212000FFF7C2FB2A00D2B221002920FDF75AFD002509212000FFF705
:20AD0000B7FB2A00D2B221003820FDF74FFD00250A212000FFF7ACFB2A00D2B221003920E5
:20AD2000FDF744FD00250B212000FFF7A1FB2A00D2B221003A20FDF739FD00250C21200016
:20AD4000FFF796FB2A00D2B221003B20FDF72EFD00250D212000FFF78BFB2A00D2B2210065
:20AD60003C20FDF723FD00250E212000FFF780FB2A00D2B221003D20FDF718FD00250F21F4
:20AD80002000FFF775FB2A00D2B221003E20FDF70DFD002510212000FFF76AFB2A00D2B283
:20ADA00021003F20FDF702FD0B2511212000FFF75FFB2A00D2B221004020FDF7F7FC022511
:20ADC0001F212000FFF754FB2A00D2B221004E20FDF7ECFC0B2512212000FFF749FB2A00CE
:20ADE000D2B221004120FDF7E1FC022520212000FFF73EFB2A00D2B221004F20FDF7D6FCC1
:20AE00000B2513212000FFF733FB2A00D2B221004220FDF7CBFC022521212000FFF728FBFC
:20AE20002A00D2B221005020FDF7C0FC0B2514212000FFF71DFB2A00D2B221004320FDF76A
:20AE4000B5FC022522212000FFF712FB2A00D2B221005120FDF7AAFC0B2515212000FFF75E
:20AE600007FB2A00D2B221004420FDF79FFC022523212000FFF7FCFA2A00D2B22100522056
:20AE8000FDF794FC0B2516212000FFF7F1FA2A00D2B221004520FDF789FC0225242120008D
:20AEA000FFF7E6FA2A00D2B221005320FDF77EFC0B2517212000FFF7DBFA2A00D2B22100EA
:20AEC0004620FDF773FC022525212000FFF7D0FA2A00D2B221005420FDF768FC0B25182158
:20AEE0002000FFF7C5FA2A00D2B221004720FDF75DFC022526212000FFF7BAFA2A00D2B214
:20AF000021005520FDF752FC0B2519212000FFF7AFFA2A00D2B221004820FDF747FC02259B
:20AF200027212000FFF7A4FA2A00D2B221005620FDF73CFC0B251A212000FFF799FA2A0066
:20AF4000D2B221004920FDF731FC022528212000FFF78EFA2A00D2B221005720FDF726FC58
:20AF60000B251B212000FFF783FA2A00D2B221004A20FDF71BFC022529212000FFF778FA95
:20AF80002A00D2B221005820FDF710FC0B251C212000FFF76DFA2A00D2B221004B20FDF752
:20AFA00005FC02252A212000FFF762FA2A00D2B221005920FDF7FAFB0B251D212000FFF7F7
:20AFC00057FA2A00D2B221004C20FDF7EFFB02252B212000FFF74CFA2A00D2B221005A20EF
:20AFE000FDF7E4FB0B251E212000FFF741FA2A00D2B221004D20FDF7D9FB02252C21200026
:20B00000FFF736FA2A00D2B221005B20FDF7CEFB00252D212000FFF72BFA2A00D2B2210086
:20B020002C20FDF7C3FB00252E212000FFF720FA2A00D2B221002D20FDF7B8FB00252F2136
:20B040002000FFF715FA2A00D2B221002E20FDF7ADFB002530212000FFF70AFA2A00D2B2D4
:20B0600021002F20FDF7A2FB002531212000FFF7FFF92A00D2B221003020FDF797FB002580
:20B0800032212000FFF7F4F92A00D2B221003120FDF78CFB002533212000FFF7E9F92A0024
:20B0A000D2B221003220FDF781FB002534212000FFF7DEF92A00D2B221003320FDF776FB3B
:20B0C000002535212000FFF7D3F92A00D2B221003420FDF76BFB002536212000FFF7C8F943
:20B0E0002A00D2B221003520FDF760FB002537212000FFF7BDF92A00D2B221003620FDF77B
:20B1000055FB002538212000FFF7B2F92A00D2B221003720FDF74AFB042539212000FFF7A8
:20B12000A7F92A00D2B221005C20FDF73FFB03253A212000FFF79CF92A00D2B221005D207C
:20B14000FDF734FB0C253B212000FFF791F92A00D2B221005E20FDF729FB0C22DFF86815B8
:20B160005E20FDF7FEFA04253C212000FFF780F92A00D2B221005F20FDF718FB03253D2175
:20B180002000FFF775F92A00D2B221006020FDF70DFB02253E212000FFF76AF92A00D2B233
:20B1A00021006120FDF702FB02253F212000FFF75FF92A00D2B221006220FDF7F7FA0225AA
:20B1C00040212000FFF754F92A00D2B221006320FDF7ECFA022541212000FFF749F92A0074
:20B1E000D2B221006420FDF7E1FA022542212000FFF73EF92078022805D3002020704221D3
:20B200002000FFF754F92A00D2B221006520FDF7CDFA022543212000FFF72AF92078042834
:20B2200005D30020207043212000FFF740F92A00D2B221006620FDF7B9FA0025442120002D
:20B24000FFF716F92A00D2B221006720FDF7AEFA032547212000FFF70BF92A00D2B221007E
:20B260006820FDF7A3FA022548212000FFF700F92A00D2B221006920FDF798FA0222DFF83D
:20B280004C146920FDF76DFA0222DFF844146520FDF767FA0222DFF83C146620FDF761FA1D
:20B2A0000222DFF830146620FDF75BFA0022DFF828146720FDF755FA0322DFF820146820C9
:20B2C000FDF74FFA0222DFF818142520FDF749FA0721DFF81004FFF7CBF84621DFF8080478
:20B2E000FFF7C6F80024DFF800040068DFF8FC13FEF7A0FB05F0BCFE0400601EDFF8F013B2
:20B30000884213D3DFF8E003002101604621DFF8D803FFF7CCF80022DFF8CC130520FDF77D
:20B3200045FA4621DFF8C003FFF7A2F805B030BD38B300082A2C0A00040000000001000043
:20B340000100000004010000020000000601000001000000080100000100000009010000C9
:20B36000010000000A010000010000000B010000010000000C010000040000001001000091
:20B3800004000000140100000400000018010000040000001C010000040000002001000031
:20B3A00004000000240100000400000028010000040000002C0100000400000030010000D1
:20B3C000020000003401000002000000360100000200000038010000020000003A01000085
:20B3E000020000003C010000020000003E0100000200000040010000020000004201000045
:20B40000020000004401000002000000460100000200000048010000020000004A01000004
:20B42000020000004C010000020000004E01000001000000500100000100000051010000C7
:20B44000010000005201000001000000530100000100000054010000010000005501000096
:20B46000010000005601000001000000570100000100000058010000010000005901000066
:20B48000010000005A010000010000005B010000010000005C010000010000005D01000036
:20B4A000040000006001000004000000680100000400000064010000040000006C010000E0
:20B4C000040000008001000004000000880100000400000084010000040000008C01000040
:20B4E000040000007001000004000000780100000400000074010000040000007C01000060
:20B5000004000000900100000200000094010000100000009601000004000000A8010000AB
:20B5200002000000AC01000001000000AE01000001000000AF01000001000000B001000049
:20B5400001000000B101000001000000B201000001000000B301000004000000B401000016
:20B5600016000000B801000004000000D001000002000000D401000001000000D601000078
:20B5800000B585B001A80021002200230EC00C38FEF708FF3220FCF735F80020ADF800006D
:20B5A000022200A94FF40370FEF715FF3220FCF729F80020ADF80000022200A94FF4137041
:20B5C000FEF709FF3220FCF71DF84A4800210170484800214170474800218170032245493A
:20B5E0004FF40570FEF7F7FE3220FCF70BF84148002101703F48002141703E480021817055
:20B6000003223C494FF40D70FEF7E5FE3220FBF7F9FF3848002101703648002141703548CD
:20B6200000218170032233494FF40970FEF7D3FE3220FBF7E7FF30480021018002222E49F6
:20B640004FF41370FEF7C7FE03222B492820FDF7ADF8FEF74BFFFFF7F4FA092201A94AF2BC
:20B66000E940FEF7B8FE05B000BD80B500200090FEF798FE002100A8FEF7FAFE00981F495E
:20B68000884207D01D480090002100A8FEF70FFFFEF72CFFFFF7D5FAFFF7D3FA01BD0000E2
:20B6A00000007243000068430000844300007E4300004643000050430000044300000E43EE
:20B6C000CDCC0C423333554208840020208800201E8800201F8800202C86002042870020CA
:20B6E0001D880020268800205486002000002041002D3101E8850020488700201203180252
:20B700000A22002105F0ADBD10B50024C0B203280CD2C0B20C21214A01FB002000688047C4
:20B720004FF6FF71884201D14FF6FF74200080B210BD70B50400080011001A000025E4B2CA
:20B74000032C0DD292B2E4B20C23144E03FB04635B6898474FF6FF71884201D14FF6FF755F
:20B76000280080B270BD70B50400080011001A000025E4B2032C0DD292B2E4B20C23074EBF
:20B7800003FB04639B6898474FF6FF71884201D14FF6FF75280080B270BD000068BF0008A2
:20B7A00000B587B0012141F2040005F0F7FEE020ADF8000003208DF8020018208DF803004B
:20B7C00000A9DFF88C0705F055FF1020ADF8000003208DF8020010208DF8030000A9DFF856
:20B7E000700705F047FF1021DFF8640705F0B3FF0020ADF804004FF48270ADF806000020B4
:20B80000ADF808000220ADF80A000120ADF80C004FF40070ADF80E000020ADF8100000207D
:20B82000ADF812000720ADF8140001A9DFF8240705F0FCFF0121DFF81C0706F017F84FF66F
:20B84000FF7007B000BD00B587B00121082005F0A5FE01214FF4804005F0B0FE4FF42040CC
:20B86000ADF8000003208DF802001C208DF8030000A9DFF8E40605F0FDFE4FF48040ADF8B3
:20B88000000003208DF8020004208DF8030000A9DFF8C40605F0EEFE4FF48050ADF800006F
:20B8A00003208DF8020014208DF8030000A9DFF8A80605F0DFFE4FF48051DFF89C0605F0A0
:20B8C0004AFF0020ADF804004FF48270ADF806000020ADF808000020ADF80A000120ADF814
:20B8E0000C004FF40070ADF80E003820ADF810000020ADF812000720ADF8140001A9DFF891
:20B900005C0605F093FF0121DFF8500605F0AEFF4FF6FF7007B000BD00B587B001210120F6
:20B9200005F03CFE0121DFF8380605F01AFF01210C2005F033FE01214FF4004005F03EFE49
:20B940003820ADF8000003208DF8020018208DF8030000A9DFF8000605F08CFE4FF40040F8
:20B96000ADF8000003208DF8020010208DF8030000A9DFF8DC0505F07DFE4FF40041DFF894
:20B98000D00505F0E8FE0020ADF804004FF48270ADF806000020ADF808000220ADF80A00B0
:20B9A0000120ADF80C004FF40070ADF80E000020ADF810000020ADF812000720ADF81400C3
:20B9C00001A9DFF8A00505F031FF0121DFF8940505F04CFF4FF6FF7007B000BD80B51021BC
:20B9E000DFF86C0505F0BAFE062000F05CFA1021DFF85C0505F0AFFE01BD80B54FF4004164
:20BA0000DFF84C0505F0AAFE062000F088FA4FF40041DFF83C0505F09EFE01BD80B5102178
:20BA2000DFF82C0505F09AFE042000F03CFA1021DFF81C0505F08FFE00F05AF801BD80B547
:20BA40004FF40041DFF8080505F088FE042000F066FA4FF40041DFF8F80405F07CFE00F0D9
:20BA600057F801BD80B51021DFF8E40405F076FE502000F018FA1021DFF8D40405F06BFE7B
:20BA80001021DFF8CC0405F069FE012000F00BFA002000F008FA1021DFF8B40405F05BFE3C
:20BAA00000F026F801BD80B54FF40041DFF8A00405F054FE502000F032FA4FF40041DFF858
:20BAC000900405F048FE4FF40041DFF8840405F045FE012000F023FA002000F020FA4FF4E1
:20BAE0000041DFF86C0405F036FE00F011F801BD10B50120002401E000F01AF8C0B2C007B8
:20BB000005D52000441C42F210718842F4D310BD10B50120002401E000F01EF8C0B2C0078E
:20BB200005D52000441C42F210718842F4D310BD10B51021DFF8180405F010FE052000F097
:20BB4000B2F900F0ABF904001021DFF8040405F002FE2000C0B210BD10B54FF40041DFF81E
:20BB6000F00305F0FBFD052000F0D9F900F0D2F904004FF40041DFF8D80305F0ECFD20000B
:20BB8000C0B210BDF8B504000D00160000271021DFF8BC0305F0E2FD0B2000F084F9200C0C
:20BBA000C0B200F080F9200AC0B200F07CF92000C0B200F078F9002000F075F904E000F064
:20BBC0006DF9BFB278557F1CBFB2B6B2B742F6D31021DFF87C0305F0BEFD4FF6FF70F2BDF1
:20BBE00070B504000D0000264FF48051DFF8680305F0B4FD14F07F0000F073F904E000F03A
:20BC00006BF9B6B27055761CB6B2032EF7D34FF48051DFF8440305F09EFD4FF6FF7070BDFB
:20BC2000F8B504000D00160000274FF40041C84805F094FD0B2000F072F9200CC0B200F0DB
:20BC40006EF9200AC0B200F06AF92000C0B200F066F9002000F063F904E000F05BF9BFB2A8
:20BC600078557F1CBFB2B6B2B742F6D34FF40041B74805F070FD4FF6FF70F2BDF8B50400C8
:20BC80000D0016000027200000F0C6F8FFF7EAFEFFF7A4FE1021AE4805F060FDAD2000F0E0
:20BCA00002F9200CC0B200F0FEF8200AC0B200F0FAF82000C0B200F0F6F8287800F0F3F89C
:20BCC000687800F0F0F81021A14805F044FD0220070015E0401E0028FCD110219C4805F0E1
:20BCE0003DFDAD2000F0DFF8785D00F0DCF87F1C785D00F0D8F87F1C1021954805F02BFDE7
:20BD0000B6B2B74201D27820E5E7642000E0401E0028FCD1FFF782FE10218D4805F01EFD48
:20BD2000FFF7E6FE4FF6FF70F2BD38B504000D004FF48051884805F011FD54F08000C0B2AB
:20BD400000F0CFF8287800F0CCF8687800F0C9F8A87800F0C6F84FF480517F4805F0FBFCB2
:20BD60004FF6FF7032BDF8B504000D0016000027FFF799FEFFF741FE4FF40041744805F02E
:20BD8000EDFCAD2000F0CBF8200CC0B200F0C7F8200AC0B200F0C3F82000C0B200F0BFF86D
:20BDA000287800F0BCF8687800F0B9F84FF40041674805F0D0FC0220070017E0401E002824
:20BDC000FCD14FF40041624805F0C8FCAD2000F0A6F8785D00F0A3F87F1C785D00F09FF8FD
:20BDE0007F1C4FF400415A4805F0B5FCB6B2B74201D27820E3E7642000E0401E0028FCD18F
:20BE0000FFF71DFE4FF40041514805F0A7FCFFF77FFE4FF6FF70F2BD10B50400FFF722FEA7
:20BE2000FFF7DCFD10214A4805F098FC202000F03AF8200CC0B200F036F8200AC0B200F03D
:20BE400032F82000C0B200F02EF81021404805F082FCFFF74DFE10BD10B50400FFF723FEF6
:20BE6000FFF7CBFD4FF40041394805F077FC202000F055F8200CC0B200F051F8200AC0B2A7
:20BE800000F04DF82000C0B200F049F84FF400412F4805F060FCFFF73BFE10BD80B500200D
:20BEA00000F001F802BD10B504000221294805F0EFFC0028F9D0E4B2210089B2254805F058
:20BEC000E3FC0121234805F0E3FC0028F9D0214805F0DCFCC0B210BD80B5002000F001F87E
:20BEE00002BD10B5040002211C4805F0D1FC0028F9D0E4B2210089B2184805F0C5FC012156
:20BF0000164805F0C5FC0028F9D0144805F0BEFCC0B210BD80B5002000F001F802BD10B510
:20BF2000040002210F4805F0B3FC0028F9D0E4B2210089B20B4805F0A7FC0121094805F0A9
:20BF4000A7FC0028F9D0074805F0A0FCC0B210BD0008014000300140000C014000380040AF
:20BF600000023000003C0040A1B7000885BB00087DBC000847B80008E1BB00082BBD00088F
:20BF800019B9000821BC000867BD00080CB41CB5044604A80190009401AB0A4600A9074816
:20BFA0007844183005F07EFC009900220A7000285CBF0098001B16BC5DF80CFB5B02000058
:20BFC000002840F10880F446404200F004F850F00040604700280AD0B0FA80F18840D1F10A
:20BFE0009D01C905020672F1004241EB1020704710B5FF2313EAD0541DBF13EAD1529C4233
:20C000009A4239E0A41ADA0780EA0103134042EA012142EA0020421A3CBF641E01EB420228
:20C02000090AB2FBF1FE01FB1E221202B2FBF1F001FB10226EF30F201202B2FBF1FE4EEACD
:20C0400000207F3406DDFE2C24DA53EA500050EBC45010BDD4F1020401FB1E2240F0807131
:20C06000192C1DDC21FA04F0C4F12004A140114371F10042584110BD9C421ABF03EAD15294
:20C080009A420FE080EA010E0EF00043400004D0490016D143F0FF4010BD490008BFD34372
:20C0A000180010BD9C4205D1D21AF7D001F00041484010BD4A0212BF0846484000F000408A
:20C0C00010BD4AB90902B1FA81F2914044B1A418C00140F000409EE7C90141F0004152425F
:20C0E0000002B0FA80F4A040141B94E74FF0807C1CEB400F94BF1CEB410F05E040EA010C3F
:20C100005FEA4C0C01D28842704718BF8142704740EA010C5FEA4C0C07D0884205D14FEA51
:20C12000400C1CF1807F98BF8042704780B50A480069804702BD80B507484069804702BDAE
:20C1400080B5C0B20449096A884702BD80B5C0B20149496A884702BDB40800204AB38B074D
:20C1600007D0521E11F8013B00F8013B21D08B07F7D183071ED1103A07D330B4B1E8381052
:20C18000103AA0E83810F9D230BC530724BFB1E80810A0E8081044BF51F8043B40F8043B3E
:20C1A000D20724BF31F8022B20F8022B44BF0B7803707047083A07D3B1E80810083A40F831
:20C1C000043B40F804CBF7D25307E4E7002206F0F9B9FEE7FEE7FEE7FEE7FEE7FEE770474C
:20C1E00000F10103810704D010F8011B89B18107FAD10268B2F10131914311F0803F04BFA7
:20C2000050F8042FF6E710F8011B11B110F8011BFBE7C01A70470268531C036011707047D5
:20C220002DE9F04105000E0090461C000027DFF814020078012803D342F6E160208020E00E
:20C24000002D03D145F6C35020801AE006F0D6F90700DFF8F4012860C5F814800020A8615B
:20C260006E6015F1080000F094FEDFF8E0010088401CDFF8D8110880380006F0C3F9002072
:20C280002080BDE8F0812DE9F04389B006000F0091469846109C00256A480078012804D3A1
:20C2A00046F2AE10208000207AE0002E04D145F6C3502080002073E01FFA89F948460028B9
:20C2C00002D0B0F5004F20D130685F49884221D1B8F1000F02D00020C8F8000006F08EF9C4
:20C2E0000500706900281AD07069401E7061B8F1000F02D0B069C8F800007669280006F0E6
:20C3000081F90020208030004AE045F625602080002045E045F6C4502080002040E05FEA6C
:20C32000094008D57669280006F06CF946F2B0102080300034E046480078012807D3280068
:20C3400006F060F946F663502080002028E03B000622310000A800F0D2FD280006F052F973
:20C3600000F0ACFC06F04AF905003A48006890F83500002805D002282BD014D303281ED01E
:20C3800033E0B8F1000F04D032480068006CC8F80000002020807669280006F033F93000D7
:20C3A00009B0BDE8F083B8F1000F04D029480068006CC8F8000046F2A9102080EBE7B8F10F
:20C3C000000F02D00020C8F8000047F2D9202080E1E7B8F1000F04D01E480068006CC8F87C
:20C3E000000045F6C2502080D5E746F62B602080280006F007F90020D2E770B504000D0000
:20C400001600002C04D145F6C3503080002011E020680D49884204D045F6C450308000205B
:20C4200008E006F052F902003300290089B2200000F012F870BD054900220A800021018057
:20C44000704700003888002053454D41AA8700203C880020BC8600202DE9F04782B0040005
:20C460000D0016001F005FF0000806F0C7F8804614F108000189002918D1606910F1010F25
:20C4800007D1404606F0BEF846F6C5503880002033E06069401C6061D4F81490A661404673
:20C4A00006F0B0F800203880484626E0A90502D5B0F8089001E05FF00109D0F800A00BE020
:20C4C000DAF80810DAF804A0009600230022200000F0D5FDB9F101091FFA89F9B9F1000F37
:20C4E000EED1D4F81490404606F08CF8280401D400F0E4FB002038804846BDE8F6870000B5
:20C500002DE9F04106000F0090461C000025DFF87C020078012803D342F6E16020802BE0B8
:20C52000002E03D145F6C350208025E01FFA88F8B8F1000F03D146F2945020801CE006F033
:20C540005DF80500DFF8480230607760414689B216F1140006F028F916F1080000F019FDF0
:20C56000DFF830020088401CDFF828120880280006F048F800202080BDE8F0812DE9F04FAC
:20C5800089B004000D0016001F00DDF84880DDF84C905FF0000A7D480078012805D346F2FF
:20C5A000AE10A9F800000020C4E0002C05D145F6C350A9F800000020BCE0002F05D146F26E
:20C5C000D520A9F800000020B4E0B6B23000002802D0B0F5004F1DD120686D4988421FD1A5
:20C5E000B8F1000F02D00020C8F8000006F006F882464B464246390014F1140006F0DEF8DE
:20C600008346B9F80000002810D1504605F0FAFF58468FE045F62560A9F80000002089E01C
:20C6200045F6C450A9F80000002083E0300408D5504605F0E7FF46F2B010A9F8000000204C
:20C6400078E055480078012808D3504605F0DAFF46F66350A9F8000000206BE02B000522B8
:20C66000210000A800F04BFC504605F0CBFF00F025FB05F0C3FF82464848006890F8350021
:20C68000002805D0022838D017D3032826D045E042480068D0F85CB040480068B0F860007D
:20C6A0003880B8F1000F04D03C480068006CC8F800000020A9F8000038E05FF0000B0020CB
:20C6C0003880B8F1000F04D034480068006CC8F8000046F2A910A9F8000027E05FF0000B13
:20C6E00000203880B8F1000F02D00020C8F8000047F2D920A9F8000018E05FF0000B0020B3
:20C700003880B8F1000F04D024480068006CC8F8000045F6C250A9F8000007E05FF0000BA6
:20C720000020388046F62B60A9F80000504605F069FF584609B0BDE8F08F2DE9FC410500F3
:20C740000E0017009846089C002D03D145F6C350208013E028680E49884203D045F6C4507D
:20C7600020800BE005F0B1FF0194009043469BB23A0092B23100280000F012F8BDE8F381A4
:20C78000044900220A800021018070473888002051554555A88700203C880020BC86002092
:20C7A0002DE9F04F83B004000D0016001F00DDF83080DDF834905FF0000A05F01FFF824659
:20C7C00014F108000189002914D1F80601D4002300E01023CDF80490CDF800809BB232008E
:20C7E00092B2290014F1140006F020F8504605F009FF25E0B90502D5B0F808B001E05FF0E8
:20C80000010B00680DE0816840680190CDF8008033009BB22A00200000F031FC0198BBF124
:20C82000010B1FFA8BFBBBF1000FECD1504605F0E9FE380401D400F041FA0020A9F8000066
:20C84000BDE8F78FF8B505000E0014000027DFF858020078012803D347F2752020803FE07D
:20C86000DFF848020078012803D346F66350208036E0B6B23000002805D0022803D00428BD
:20C880001ED008281DD1002D03D147F27E20208026E005F0B3FE070085480068012180F892
:20C8A00036102300320092B229008148006806F071F82088002808D0380005F0A3FE0FE07B
:20C8C000E7E745F6256020800AE07948006800F0C0FC380005F096FE00F0F0F90020208011
:20C8E000F1BDF8B5069C079D00276F4E3678012E03D347F275202880B0E06C4E3678012E63
:20C9000003D346F663502880A8E014F00E06B6B23700002F05D0022F03D0042F17D0082F12
:20C9200016D1002B0CD192B2002A09D189B2002906D180B2002803D147F27E2028808DE06B
:20C940004FF6E17C14EA0C0F06D1002705E0F7E745F62560288081E00127FFB2012F03D1B5
:20C9600045F62560288079E0C4F30014A4B214F00104E4B2012C1CD04FF47A74A34203D331
:20C9800047F27B20288069E092B23C2A03D347F27A20288062E089B23C2903D347F279204D
:20C9A00028805BE080B2642815D347F27820288054E042F2107489B2A14203D347F27920C3
:20C9C00028804BE04FF47A7480B2A04203D347F27820288042E0374C246880B24FF4616782
:20C9E00089B25FF03C0C0CFB01F107FB001092B210184FF4FA71B1FBF4F1C91801FB04F1DD
:20CA00004FF47A72B1FBF2F104FB0014002C22D005F0F4FD070026480068012180F8361084
:20CA20002B00320092B221002148006805F0B2FF2888002803D0380005F0E4FD0EE01C48B2
:20CA4000006800F006FC380005F0DCFD00F036F90020288002E047F27E202880F1BD10B5BB
:20CA600082B006F0B7F900AA0021134800F000FF0400124800780C21114A01FB002000F05F
:20CA800037FC10480068401E0E4908600D480068002808D10B480C490968016000AA002183
:20CAA0000A4800F0E5FE13BD388800203C880020BC860020D4320108587400203A8800207E
:20CAC000F0640020B8860020B48600201875002010B5040006F0F9F8DFF8A00800210170BC
:20CAE000DFF89C0800210170DFF8980800210170DFF8940800210160DFF89008002101603A
:20CB0000DFF88C0800210160DFF8880800210170DFF8840800680A21B0FBF1F0DFF87C1842
:20CB20000860DFF87C08006800280ED0DFF874080068002809D0DFF86818096803E0491EF6
:20CB400000220260001D0029F9D106F083F900F001FB200000F09AFE2088002837D1200043
:20CB600000F0A5F92088002831D1200005F0C4FE208800282BD1200006F0B0F92088002823
:20CB800025D1200006F0B2F9208800281FD1200005F0C2FD2088002819D1200006F0AEF9D3
:20CBA0002088002813D12000FFF7EAFD208800280DD12000FFF73FFC2088002807D12000FD
:20CBC00006F0A6F92088002801D106F019FB10BDDFF8AC07007801280BD1DFF8A00700784A
:20CBE000FA2806D2DFF894070078401CDFF88C170870704710B50024DFF884070078012860
:20CC00005BD105F0FBFC0400DFF870070078002803D1200005F0F6FC4FE0DFF8600700784A
:20CC2000401EDFF858170870DFF850070078012803D3200005F0E6FC3FE0DFF8480700787F
:20CC4000012803D3200005F0DDFC36E006F00CF9DFF854170870DFF8500700780C21DFF872
:20CC60004C2701FB00200068DFF844170860DFF840070068DFF83C170968884203D1200044
:20CC800005F0C0FC19E0DFF828070068D0F88C00401CDFF81C170968C1F88C00DFF8180716
:20CCA0000068401CDFF810170860DFF810075FF080510160200005F0A5FC10BD10B500246F
:20CCC000DFF8B806007801283ED2DFF8B8060078012839D205F092FC040006F0C5F8DFF8BC
:20CCE000C8160870DFF8C00600780C21DFF8BC2601FB00200068DFF8B8160860DFF8B006C5
:20CD00000068DFF8B0160968884203D1200005F079FC19E0DFF898060068D0F88C00401CEF
:20CD2000DFF88C160968C1F88C00DFF88C060068401CDFF884160860DFF880065FF0805141
:20CD40000160200005F05EFC10BD38B504000025DFF828060078012803D346F66250208016
:20CD600022E0DFF81C060078012803D045F68960208019E0DFF80C060078FA2803D345F2F7
:20CD80000920208010E005F039FC0500DFF8F4050078401CDFF8EC15087000F088FA28001D
:20CDA00005F030FC0020208031BD38B504000025DFF8C8050078012803D346F665502080E2
:20CDC00030E0DFF8BC050078012803D045F68960208027E0DFF8AC050078002803D146F634
:20CDE000645020801EE005F009FC0500DFF894050078401EDFF88C150870DFF888050078D0
:20CE0000012806D3280005F0FDFB46F66350208008E000F056FA280005F0F4FBFFF74EFFF5
:20CE20000020208031BD10B50400DFF854050078002826D106F018F8DFF86C150870DFF807
:20CE40008005DFF8641509780170DFF85C0500780C21DFF8582501FB00200068DFF850151A
:20CE60000860DFF85005DFF8481509680160DFF810050121017006F04FFA43F699202080C8
:20CE800002E045F68A60208010BD80B5002105F0B5FB0100DFF82C050068401CDFF8242536
:20CEA0001060080005F0AEFB05F00EFFEFE700B589B0DFF8101500220A60089003200790BC
:20CEC000002006900020059000200490DFF8F80400680390DFF8F40400680290DFF8F004D1
:20CEE00000680190132000900023DFF8E8240FF24051DFF8E40400F0A5FA09B000BD70B5F5
:20CF000004000D001900DFF8AC04006880F83420DFF8A0040068002280F83520DFF89404EB
:20CF2000006800F05BFA002D0ED015F10806E56001222100DFF87C04006800F010F82100C4
:20CF4000300000F02DF809E0DFF8680400680021C187DFF8600400680021016370BD10B476
:20CF6000C287016300230EE000244C6000240C6000240C6100244C6100240C830024CC612D
:20CF8000886020315B1C9BB292B29342ECD310BC704700210160002141600021018170479B
:20CFA00010B48A6892F837200389002B08D10122028100224A6000220A600160416024E046
:20CFC00003895B1C0381046800E06468002C05D0A36893F83730D2B29A42F6D2002C06D189
:20CFE00000224A6042680A60516041600DE02268002A05D1216000220A604C60016004E08A
:20D0000022680A604C605160216010BC704770B50400266BE58F06E0F0680830310000F0F6
:20D020000AF820366D1EADB2012DF5D20020E0870020206370BD0289012A04D10022026053
:20D040000022426013E00A68002A04D14B6800221A6003600BE04A68002A04D10A680023C5
:20D060005360426003E00A684B6853601A600289521E02810020486000200860704738B5B4
:20D0800005000C00049894F8361000290BD002290AD008D3042906D006D3062925D002D358
:20D0A000072922D042E041E094F83410032906D100909BB22100280000F039F803E0E265C7
:20D0C000A4F860302064002D02D02000FFF79FFF200000F0A0F9002084F83600002084F8D6
:20D0E0003500002084F8340020E094F83410032906D100909BB22100280000F018F803E04F
:20D10000E265A4F860302064200005F0D1FC002D02D02000FFF77BFF042084F836000020B1
:20D1200084F83500002084F83400FFE731BD70B4039C0D6BC98F01E02035491E89B2012905
:20D1400006D3EE68B042F7D128616A612B83EC6170BC704700200BE0C0B20C21934A01FB31
:20D16000002100220A8100220A6000224A60401CC0B21428F0D3704710B5040094F8370079
:20D1800005F082FE94F837008D490978884203D1200000F022F802E0200000F001F810BD80
:20D1A00090F837100C22814B02FB01310A89002A08D101220A810022C26000220261086002
:20D1C000486009E00A89521C0A810A68C260002202610A6810610860704790F837100C221A
:20D1E000724B02FB01310A89002A08D101220A810022C260002202610860486008E00A89AB
:20D20000521C0A810022C2604A680261D0604860704710B40189002902D0022901D00BD20B
:20D2200015E0016842680A610023CB6000231361D160026041600AE001684268CB6800240E
:20D240001C610024CC600A61D1600360416010BC704710B5040094F837000C21534A01FB8C
:20D2600000202169E268002913D1002A0AD100210181002101600021416094F8370005F009
:20D2800016FE0FE00189491E018100211161026008E003895B1E0381CA60002A01D14160EB
:20D2A00000E01161002020610020E06010BD80B534480078012803D105F007FA324908604F
:20D2C00001BD80B52F480078002810D105F0FDF92D490968401A2D490968814201D22B4946
:20D2E00008602B490968814201D22949086001BD38B5040000252748007801283CD105F08B
:20D300007DF905002068002803D1280005F07AF932E03149884203D1280005F073F92BE0C0
:20D32000816D002902D0816D491E8165806D002803D0280005F066F91EE02089022803D2BF
:20D34000280005F05FF917E00E480078012803D3280005F057F90FE02000FFF75AFF206841
:20D36000416D002903D10D490968816501E0416D8165280005F046F931BD000038880020B6
:20D38000398800203C8800209086002094860020988600203D880020D43201089C860020E4
:20D3A000BC320108B83201083B880020F0640020C0860020BC860020A086002004ED00E04D
:20D3C0003A8800208C860020B0320108AC320108A83201088BCE00089873002010B582B001
:20D3E0000400002910D000AB0222200005F0D2FABDF80000002803D1032084F8360006E004
:20D40000022084F8360002E0022084F836002000FFF71FFF13BD10B50400200005F048FB5D
:20D4200094F83600400702D42000FFF7A5FE10BD75432F4F532D4949492049646C652054E4
:20D4400061736B002DE9FE4F82B005000F9EDDF84090119FDDF84C80159CDDF858A05FF083
:20D46000000BDFF83C040078012804D347F24A10AAF80000ABE0002D04D147F2AD10AAF8B8
:20D480000000A4E00398002804D147F24F10AAF800009CE0002E04D146F62C60AAF800004D
:20D4A00095E0DFF820050068874204D246F62D60AAF800008BE0B94504D346F62E60AAF8DD
:20D4C000000084E09DF83800142804D346F27320AAF800007BE09DF83800132808D1DFF888
:20D4E000E804854204D046F27320AAF800006EE0280000F0D9F90020AAF80000E0070AD578
:20D50000A00708D53000002103E000220260001D491CB942F9D316EB8909A4B20194009771
:20D520004B4632000499039805F0DCFB0399A9620499E962029929629DF8381085F83710CE
:20D540002860C5F80890C5F85480B8F1000F04D1DFF834050068A86501E0C5F85880149829
:20D5600068606E62AF63AC87002005E080B215EB80010022CA67401C80B20028F6D0BDF892
:20D58000481015F1640005F00FF9280005F0A7FB05F034F8834695F8370005F075FC2800D1
:20D5A000FFF71BFEDFF8E4040088401CDFF8DC140880DFF8DC040078012803D0584605F0AC
:20D5C00021F804E0584605F01DF8FFF777FB05B0BDE8F08FF8B505000C000026DFF8C002E8
:20D5E0000078012803D347F24E10208044E0DFF8D803854203D147F24C1020803CE0002D8E
:20D6000008D104F0FBFF0600DFF898020568300004F0F8FF04F0F2FF060095F8360000286E
:20D620000BD002282ED029D3042826D02AD3062828D023D3072825D03AE02800FFF709FE4D
:20D6400015F1640005F08EF80700280005F048FBDFF838040088401EDFF8301408802800BA
:20D6600000F022F9FF2085F83600300004F0CAFFFFF724FB00202080F1BDE1E7280005F078
:20D6800017FADDE7280005F013FA95F83400002808D0401E07D0401E04D0401E032802D9FF
:20D6A000001F04D103E02800FFF7B1FCFFE7C7E7300004F0A7FF46F62A602080DCE72DE92B
:20D6C000F0410700884616001C000025DFF8D0010078012804D346F2AE1020800020C5E072
:20D6E000002E01D00020306004F088FF0500DFF8A4030068406C00283CD0DFF8980300685B
:20D70000406C401EDFF88C1309684864DFF884030068476C002E04D0DFF878030068006CCB
:20D72000306004F0D2FFDFF86C130968096C401ADFF860130968C1F8A800DFF85803006848
:20D74000D0F8AC00DFF84C130968D1F8A810884209D2DFF840030068DFF838130968D1F8AA
:20D76000A810C0F8AC10280004F04CFF0020208038007BE05FEA084007D5280004F042FFF9
:20D7800046F2B0102080002070E0DFF80C030078012807D3280004F035FF46F66350208041
:20D7A000002063E03B00072200210020FFF7A7FB280004F027FFFFF781FA04F01FFF0500FF
:20D7C000DFF8D002006890F83500002804D001282ED0032837D03EE0002E26D0DFF8B40257
:20D7E0000068006C306004F070FFDFF8A8120968096C401ADFF89C120968C1F8A800DFF863
:20D8000094020068D0F8AC00DFF888120968D1F8A810884209D2DFF87C020068DFF8741274
:20D820000968D1F8A810C0F8AC100020208015E0002E04D0DFF85C020068006C306046F2FA
:20D84000A91020800AE0002E01D00020306047F2D920208002E046F62B602080DFF83402AE
:20D860000068476C280004F0CDFE3800BDE8F08170B504000D00160004F027FF02003300BD
:20D88000290089B2200000F0A1F870BD7F4900220A80824900220A6000210180704700002A
:20D8A00038880020BC86002010B50400002020600020A060002060600020E06000202061BC
:20D8C000002060610020A0610020E0610FF2D0102062002060620020A0620020E0620020FC
:20D8E00020630020E087002020640020E0650020A4F86000002114F1640004F055FF002007
:20D9000060670020A0670020C4F880000020A4F888000020C4F88400002005E0C0B214EBA3
:20D9200080010022CA67401CC0B20028F6D0002060640020C4F8A8000020C4F8AC00002047
:20D94000A063002084F88A000020C4F8B4000020C4F8B0000020A0875FF00040A064002088
:20D96000E06400202065002060650020A065002084F88B000020C4F88C000020C4F89000B9
:20D9800004F0A3FEC4F8940000200021C4E926010020C4F8B800002084F83400002084F88D
:20D9A0003500002084F83600142084F8370010BD80B53848006805F094F900A90020FFF74E
:20D9C00009FE01BDD0320108987300202DE9F04182B007000C0090461E00002504F00EFEA7
:20D9E0000500002F01D12B480768C7F840800020308097F8360000280BD002281DD008D336
:20DA0000042806D019D3062817D002D3072814D030E0786C10F1010F07D1280004F0F2FD33
:20DA200046F6C550308000202CE0786C401C78647E6C280004F0E6FD23E097F834000728BF
:20DA400010D1CDF800800023002239000020FFF716FB7E6C280004F0D5FD200409D4FFF72C
:20DA60002DF906E0786C401C78647E6C280004F0C9FD06E0280004F0C5FD46F62A60308078
:20DA800000263000BDE8F6819C860020AC87002039880020BC8600203C880020A086002012
:20DAA0003F5461736B00000080B500208DF80000012200A91820FAF754FE02220DF101014F
:20DAC0001F20FAF74EFE01220DF102011E20FAF748FEBDF802004FF6FF71884222D19DF873
:20DAE000010000281ED19DF8000000280DD1DFF8780B0078552803D1DFF86C0BAA210170C6
:20DB0000DFF8680B552101700CE0DFF8600B0078552803D1DFF8540BAA210170DFF8480B41
:20DB200055210170DFF86C0C0078AA280CD1DFF8400B0078052807D3DFF8580C55210170C5
:20DB40000221002005F08EFD01BDDFF8280B00210180DFF8200B00214180DFF8180B002199
:20DB6000C180DFF8100B00218180DFF8080B00214181DFF8000B04210181DFF8F80A002100
:20DB80000161DFF8F00ADFF8101CC160704780B580B20028092832D90C383AD0401E40D0F0
:20DBA000401E31D0401E29D0801F5AD0001F66D0401E012840F2FF80401F6ED0401E78D016
:20DBC000401E00F08380401E00F08D80401E00F09780401E00F0A180401E00F0AB80401EEE
:20DBE00000F0B580401E00F0BF80401E00F0C980401E00F0D380401E4FD0DDE0DCE0DFF86E
:20DC00009C0B55210170D7E0DFF8900BAA210170D2E00320F9F74CFEDFF8840B01210180F9
:20DC2000CAE0DFF84C0A00210170DFF8700B0078AA2811D1DFF86C0B4FF6FF710180062251
:20DC40000021DFF8640BFBF773FF1220F9F730FEDFF84C0B01210180DFF8400B55210170CF
:20DC6000AAE0DFF8480B4FF6FF710180DFF8400B00210170DFF83C0B002101709CE0DFF803
:20DC80002C0B4FF6FF710180DFF8240B01210170DFF8200B002101708EE0DFF81C0BAA21B3
:20DCA00001700620F9F704FEDFF8F40A0121018082E0DFF8EC0A01210180DFF8F40A022199
:20DCC0000170DFF8F00A0021017075E0DFF8D00A01210180DFF8D80A03210170DFF8D40AC4
:20DCE0000021017068E0DFF8B80A01210180DFF8C00A04210170DFF8BC0A002101705BE06D
:20DD0000DFF89C0A01210180DFF8A40A05210170DFF8A00A002101704EE0DFF8840A0121FF
:20DD20000180DFF88C0A06210170DFF8880A0021017041E0DFF8680A01210180DFF8700A04
:20DD400007210170DFF86C0A0021017034E0DFF8500A01210180DFF8580A08210170DFF8B9
:20DD6000540A0021017027E0DFF8340A01210180DFF83C0A09210170DFF8380A0021017091
:20DD80001AE0DFF81C0A01210180DFF8240A0A210170DFF8200A002101700DE0DFF8000AE7
:20DDA00001210180DFF8080A0B210170DFF8040A0021017000E0FFE7DFF8000A4FF6FF7167
:20DDC000018001BD10B588B0DFF8F4090078401EDFF8E8190988002900F04384DFF8DC0958
:20DDE0000021018000A9DFF88C08C08805F099FC4FF41B722021DFF8CC09FBF799FEF9F765
:20DE000040FF002011E0C0B2009911EB0011C0B23E22DFF8B03902FB00328A60C0B201017B
:20DE2000009A4FF6FF738B52401CC0B20428EAD30098002141730098102141770098202136
:20DE400080F82D100098302180F83D100098302180F84D10DFF854090088002840F06381A9
:20DE6000DFF864094FF6FF710180DFF8600900210170DFF83C0900210170DFF8F40700785E
:20DE8000052808D3DFF8480900210170DFF840190220F9F709FBDFF83C09007801286BD181
:20DEA000DFF8340900780C21DFF8302901FB002090F85020DFF8200900780C21DFF81C3994
:20DEC00001FB0030C16CDFF8100900780C23DFF80C4903FB004090F84800DFF8E83813EB23
:20DEE0004000F9F7ECFEDFF8F00800780C21DFF8EC2801FB002090F86820DFF8DC0800784A
:20DF00000C21DFF8D83801FB0030416EDFF8C80800780C23DFF8C44803FB004090F86000BB
:20DF2000DFF8A03813EB40003E30F9F7C8FEDFF8A80800780C21DFF8A42801FB002090F85D
:20DF40008020DFF8940800780C21DFF8903801FB0030C16FDFF8800800780C23DFF87C486D
:20DF600003FB004090F87800DFF8583813EB40007C30F9F7A4FEB9E0DFF85808007802280E
:20DF80004CD1DFF8540800780C21DFF8502801FB002090F89820DFF8400800780C21DFF846
:20DFA0003C3801FB0030D0F89410DFF82C0800780C23DFF8284803FB004090F89000DFF82F
:20DFC000043813EB4000F9F77AFEDFF80C0800780C21DFF8082801FB002090F8B020DFF87D
:20DFE000F80700780C21DFF8F43701FB0030D0F8AC10DFF8E40700780C23DFF8E04703FB66
:20E00000004090F8A800DFF8BC3713EB40003E30F9F755FE00981521417767E0DFF8B80774
:20E0200000780C21DFF8B42701FB0020027ADFF8A80700780C21DFF8A43701FB003041683F
:20E04000DFF8940700780C23DFF8904703FB00400078DFF8703713EB4000F9F730FEDFF892
:20E06000780700780C21DFF8742701FB002090F82020DFF8640700780C21DFF8603701FBD5
:20E080000030C169DFF8500700780C23DFF84C4703FB0040007EDFF82C3713EB40003E3045
:20E0A000F9F70DFEDFF8300700780C21DFF82C2701FB002090F83820DFF81C0700780C21ED
:20E0C000DFF8183701FB0030416BDFF80C0700780C23DFF8084703FB004090F83000DFF8BE
:20E0E000E43613EB40007C30F9F7E9FDDFF880050078062190FBF1F201FB1200002840F077
:20E100004F82DFF8D0060078401CDFF8C8160870DFF8C00600780328C0F04282DFF8B4063B
:20E12000002101703CE2DFF8480500210170DFF8980600210180DFF87C060078401CDFF85E
:20E1400074160870DFF868060078002811D1DFF86406007824281DD3DFF850060021018032
:20E16000DFF8500600210170DFF868060021017010E0DFF8400600780B280BD3DFF82C066A
:20E1800000210180DFF82C0600210170DFF8440600210170DFF8400600780C21DFF8402690
:20E1A00001FB0020027ADFF8300600780C21DFF8303601FB00304168DFF81C0600780C2363
:20E1C000DFF81C4603FB00400078DFF8F83513EB4000F9F774FDDFF8D8050078012827D160
:20E1E000DFF8F40500780C21DFF8F82501FB002090F86820DFF8E00500780C21DFF8E43539
:20E2000001FB0030416EDFF8D00500780C23DFF8D44503FB004090F86000DFF8A83513EB08
:20E2200040003E30F9F74BFD009815214177B7E1DFF87C050078022828D1DFF89C050078F7
:20E240000C21DFF8A02501FB002090F8E821DFF8880500780C21DFF88C3501FB0030D0F8B3
:20E26000E411DFF8740500780C23DFF8784503FB004090F8E001DFF84C3513EB40003E3073
:20E28000F9F71DFD00981521417789E1DFF820050078032828D1DFF8400500780C21DFF854
:20E2A000442501FB002090F80022DFF82C0500780C21DFF8303501FB0030D0F8FC11DFF86E
:20E2C000180500780C23DFF81C4503FB004090F8F801DFF8F03413EB40003E30F9F7EFFC01
:20E2E0000098152141775BE1DFF8C4040078042828D1DFF8E40400780C21DFF8E82401FBDD
:20E30000002090F81822DFF8D00400780C21DFF8D43401FB0030D0F81412DFF8BC040078C3
:20E320000C23DFF8C04403FB004090F81002DFF8943413EB40003E30F9F7C1FC0098152135
:20E3400041772DE1DFF868040078052828D1DFF8880400780C21DFF88C2401FB002090F8E3
:20E360003022DFF8740400780C21DFF8783401FB0030D0F82C12DFF8600400780C23DFF8E9
:20E38000644403FB004090F82802DFF8383413EB40003E30F9F793FC009815214177FFE012
:20E3A000DFF80C040078062828D1DFF82C0400780C21DFF8302401FB002090F84822DFF81B
:20E3C000180400780C21DFF81C3401FB0030D0F84412DFF8040400780C23DFF8084403FB64
:20E3E000004090F84002DFF8DC3313EB40003E30F9F765FC009815214177D1E0DFF8B0036F
:20E400000078072828D1DFF8D00300780C21DFF8D42301FB002090F86022DFF8BC0300780B
:20E420000C21DFF8C03301FB0030D0F85C12DFF8A80300780C23DFF8AC4303FB004090F8CE
:20E440005802DFF8803313EB40003E30F9F737FC009815214177A3E0DFF85403007808282A
:20E4600027D1DFF8740300780C21DFF8782301FB002090F87822DFF8600300780C21DFF84B
:20E48000643301FB0030D0F87412DFF84C0300780C23DFF8504303FB004090F87002C94BE8
:20E4A00013EB40003E30F9F70AFC00981521417776E0BF480078092821D1C74800780C2188
:20E4C000C84A01FB002090F89022C34800780C21C44B01FB0030D0F88C12BF4800780C23D5
:20E4E000C04C03FB004090F88802B64B13EB40003E30F9F7E4FB00981521417750E0AC489A
:20E50000007800284CD100200190042201A92B20FAF727F90198C00412D4AC48007806218B
:20E5200090FBF1F201FB1200002803D1AE484FF6FF710180A5480078401CA44908700EE023
:20E540009A4800210180A348002101709848002101709848002101709C48002101709E487A
:20E5600000780C219F4A01FB002090F868239A4800780C219B4B01FB0030D0F86413964828
:20E5800000780C23974C03FB004090F860038D4B13EB40003E30F9F792FB00981521417741
:20E5A00033480078401C32490870F9F7CFFAFFF77BFA02228D496920FAF7D3F88C4800885A
:20E5C0004FF6FF7188420BD088480078022807D086480078032803D084480078042805D10E
:20E5E0000120F9F765F96E480121018002A8FBF735F8794800780C21794A01FB002090F8BD
:20E600003820754800780C21754B01FB0030416B714800780C23724C03FB004090F8300094
:20E62000684B13EB4000BA30F9F749FB0F220DF10A01694800780C23694C03FB004090F8BE
:20E640004800604B13EB4000BA30F9F738FBF9F7FAFA0221002000F0BCF90221022000F07B
:20E66000B8F908B010BD0000DC090020DD0900200E8800206080002010B582B000244F48F1
:20E680004FF6FF7101805B48002101704FF41B7220214C48FBF74CFAF9F7F3FA5648552141
:20E6A00001705648552101700020FAF7CBF9E02200215348FBF73CFA00200090002200A92E
:20E6C0000020FAF773F8002200A90120FAF76EF8002200A90220FAF769F8002200A903204E
:20E6E000FAF764F8002200A90420FAF75FF84548AA2101704448AA2101702F4855210170A7
:20E70000424855210170424855210170414855210170414855210170402200213F48FBF73B
:20E7200007FA402200213E48FBF702FA392200213C48FBF7FDF93C48552101703B48552195
:20E740000170224800210170394800210170394800210170082200213748FBF7E9F9374809
:20E76000002101603648002101603648552101703548002101703548002101700B48002120
:20E78000018013BD28485521017028485521017070470000D809002098860008CE090020A5
:20E7A000BA0900203A870020D084002028870020F0870020F1870020E4090020328700203D
:20E7C000238800200852002026870020F287002084840020EF8700201E88002004B9010844
:20E7E000F4B90108FCBA010880870020208800204E8700200E880020DC090020DD090020FF
:20E80000A0670020E2090020E3090020E5090020E6090020E8090020EA0900200C7C0020D1
:20E82000CC7B00204C7C0020DE090020DF0900201388002014880020C884002014860020DD
:20E8400018860020ED090020FB870020FC87002030B589B00300080000AC911E232901D3FB
:20E86000002038E00A2A03D1002B01D5012500E00025EDB2002D01D05B4203E002E03031CC
:20E880002170641C002B02D100A98C420BD1B3FBF2F102FB1131B3FBF2F30A29EFDB37314E
:20E8A0002170641CEEE7002805D100A8201A2818401C02F052F80100002D07D02D220A70EC
:20E8C000491C03E0641E22780A70491C00AAA242F8D300220A7009B030BD10B58AB0030058
:20E8E000080000AC911E232901D3002026E002E030312170641C002B02D100A98C420BD1CA
:20E90000B3FBF2F102FB1131B3FBF2F30A29EFD337312170641CEEE7002804D100A8201A72
:20E92000401C02F01AF8010003E0641E22780A70491C00AAA242F8D300220A700AB010BD1C
:20E9400038B5C0B2042812D201230122C0B203215A4C01FB00418978C0B20324574D04FB4B
:20E960000050407800F0C4FF4FF6FF7000E0002032BD10B5C0B2042811D20122C0B203213A
:20E980004E4B01FB00318978C0B203234B4C03FB0040407801F02DF84FF6FF7000E00020C1
:20E9A00010BD10B5C0B2042811D20022C0B20321424B01FB00318978C0B203233F4C03FBB0
:20E9C0000040407801F015F84FF6FF7000E0002010BD80B5C0B2002840D1C9B2012914D156
:20E9E00037490978002968D1C0B2FFF7DAFF354802684FF47A71092004F0CCFE092005F059
:20EA00000FF92F480121017057E02D490978012953D1C0B2FFF7C5FF092005F001F92A48B2
:20EA2000007800280BD1002301220721012000F05FFF00220721012000F0DBFF0AE001233A
:20EA400001220721012000F053FF01220721012000F0CFFF1A48002101702EE0C0B2022840
:20EA60002BD1C9B2012918D118480078002803D017480078012820D10220FFF77AFF032094
:20EA8000FFF777FF13484FF6FF7101800F48012101700F48002101700FE00C4800780128C2
:20EAA0000BD10C48002101800220FFF77AFF0320FFF777FF05480021017001BD5809002046
:20EAC000DF8700202C860020D9870020E0870020D88700201A87002070B4012240F24913C2
:20EAE0005FF0FF3100E0621C1BB212B2934221DB5FF0FF3409B2A1421CD11BB212B2D4184D
:20EB0000022594FBF5F424B222253E4E05FB046535F8225C80B28542E5D324B22223394D47
:20EB200003FB045333F8223C80B2984201D2631EDAE7611E080000B270BC704770B5040091
:20EB40000D00002613E0305D00280DD0305D4FF480713219527801FB002080B2FFF7BCFF28
:20EB600000F200102880AD1CB61C00202880305D002809D0102E07DA305DA128E3D2305D43
:20EB80002880AD1C761CF0E770BDF0B4049C059D89B2102934D180B2802804D342F2200604
:20EBA00080B2B0421DD1198080B2C1B20C26164F06FB017109891B8891FBF3F1118080B293
:20EBC000C1B20C22104B02FB0131897A298080B2C0B20C210C4A01FB002040682060F0BC47
:20EBE0007047102119800221118010212980074980B22222034B02FB003008182060EEE750
:20EC0000EDE70000147101087481030802DEFFFF80B500200090002200A90520F9F7A1FD51
:20EC200060220021DFF8BC05FAF782FF002006E0C0B2DFF8B415009A41F82020401CC0B22E
:20EC40003028F5D301BD2DE9F04186B00400002500200190002002900026002700200090D0
:20EC60005FF0000803A8FAF7CAF8002202A90520F9F777FD9DF81100C0B29DF812101E227A
:20EC800091FBF2F111EB4000401CC0B2302800D30020C0B2DFF85015029A41F820200025C8
:20ECA00012E00A20B7FBF0F0EDB2DFF8381511EB450121F8020CEDB2DFF8280510EB450097
:20ECC00030F8020C86196D1CEDB2302D6FD2EDB2002D35D1DFF81005D0F8BC00DFF8081563
:20ECE0000968FDF703FAEED2DFF8FC040068DFF8F814D1F8BC1000F085FADFF8F014FAF700
:20ED000099FEFAF703FF07000A20B7FBF0F100FB1170052808D30A20B7FBF0F0401CDFF832
:20ED2000C414A1F85E0006E00A20B7FBF0F0DFF8B414A1F85E00DFF8AC04B0F85E60C2E736
:20ED4000EDB2DFF8A40410EB850050F8040CEDB2DFF8941451F82510FDF7C8F9B3D2EDB248
:20ED6000DFF8840450F82500EDB2DFF87C1411EB850151F8041C00F045FADFF87014FAF75B
:20ED800059FEFAF7C3FE07000A20B7FBF0F100FB1170052885D30A20B7FBF0F0401CEDB2EE
:20EDA000DFF8401411EB450121F8020C83E7002000903000FDF70EF9DFF83414FDF718F956
:20EDC00001900199DFF82C0400F0E2FBE4B23421DFF8242401FB042188620099DFF8140497
:20EDE00000F0D6FBE4B23421DFF80C2401FB04214862E4B23420DFF8001400FB0410816AC6
:20EE0000DFF8F803FAF716FEFAF780FE80460A20B8FBF0F100FB118005280FD318F106007E
:20EE2000FDF7D8F8DFF8D413FDF7E2F8E4B23421DFF8C42301FB042188620EE018F10200D5
:20EE4000FDF7C8F8DFF8B413FDF7D2F8E4B23421DFF8A42301FB04218862E4B23420DFF84D
:20EE6000981300FB0410416ADFF89003FAF7E2FDFAF74CFE80460A20B8FBF0F100FB1180A8
:20EE800005280FD318F10600FDF7A4F8DFF86C13FDF7AEF8E4B23421DFF85C2301FB042172
:20EEA00048620CE018F10200FDF794F8D349FDF79FF8E4B23421D04A01FB04214862E4B224
:20EEC0003420CD4900FB0410806A0190002201A90020F9F76BFCE4B23420C74900FB0410F2
:20EEE000406A0090002200A90620F9F75FFC06B0BDE8F08180B5C0B23421BF4A01FB0020AF
:20EF0000001DF9F77CFF002802D17FF0050000E0002002BD1CB50400E4B23420B64900FB82
:20EF200004104078022815D12000C0B2FFF7E2FF10F1060F02D17FF0050021E0E4B2342044
:20EF4000AD4900FB0410032141702000C0B2FFF75FFE14E0E4B23420A74900FB041040785D
:20EF600003280CD100A8FAF794F8002802D17FF0050005E000A92000C0B2FFF764FE00205D
:20EF800016BD1CB50400E4B234209B4900FB04104078022815D12000C0B2FFF7ABFF10F1F1
:20EFA000060F02D17FF0050051E0E4B23420924900FB0410032141702000C0B2FFF728FE6D
:20EFC00044E0E4B234208C4900FB0410407803283CD100A8FAF75DF8002802D17FF00500F2
:20EFE00035E000A92000C0B2FFF72DFEE4B23420814900FB0410416A8148006800F0C8FA4F
:20F000000100E4B234207C4A00FB0420006AFDF76DF81BD2E4B23420774900FB0410103077
:20F02000F9F7EDFE002802D17FF005000FE0E4B23420714900FB041005214170E4B2342023
:20F040006D4900FB0410022180F83010002016BD1CB50400E4B23420674900FB04104078E7
:20F06000022815D12000C0B2FFF744FF10F1060F02D17FF005004CE0E4B234205E4900FBA0
:20F080000410032141702000C0B2FFF7C1FD3FE0E4B23420584900FB04104078032837D19D
:20F0A00000A8F9F7F6FF002802D17FF0050030E000A92000C0B2FFF7C6FDE4B234204E49CF
:20F0C00000FB0410806AE4B234214B4A01FB0421C96A00F009F91BD8E4B23420464900FB0A
:20F0E00004101030F9F78BFE002802D17FF005000FE0E4B23420404900FB0410052141708C
:20F10000E4B234203C4900FB0410032180F83010002016BD30B585B00400E4B2342036491B
:20F1200000FB04104078022815D12000C0B2FFF7E1FE10F1060F02D17FF005004FE0E4B26F
:20F1400034202D4900FB0410032141702000C0B2FFF75EFD42E0E4B23420274900FB041093
:20F16000407803283AD100A8F9F793FF002802D17FF0050033E000A92000C0B2FFF763FD64
:20F1800002A8F9F73CFE002802D17FF0050026E0E4B23420184900FB041010F1100102A810
:20F1A000F9F7E4FE022819D1E4B23420124900FB0410103002A92CC92CC00C390C38E4B22A
:20F1C00034200D4900FB041005214170E4B23420094900FB0410042180F83010002005B0A2
:20F1E00030BD00002C7B0020D872002000007A440000C842ACC5A737887C002000401C4614
:20F20000DC85002090EA010F44BF81F0004100F0C6B9431A4FF000423EBF5340C01AC91896
:20F22000D3095FEAD05C13EB400F34BFB3EB410F40E07CEBD1530CD342EA012122D8D1EBC1
:20F24000402009D3400A28BF5FEA500140EBCC507047401A15D04002B0FA80F2521C9040CE
:20F26000400A4FEA3C23B3EB026384BF00EB730007E040F400001A16DB07C2F10102D04015
:20F2800018437047182BFCDC31FA03F202FA03F3591A38BF42F00102D2EB40203CBF400038
:20F2A000ACF1010C5FEACC5CC20572F100414CEB5020704713EB400F0FD24B0009D0ACEB81
:20F2C000D153022B03DB4902172BDDDD70479143401A4300D5D10020704713EB410FD0D322
:20F2E0006FF00000704700004FF0807C1CEB400F94BF1CEB410F05E040EA010C5FEA4C0C00
:20F3000001D28142704718BF884270475FF0FF0C1CEAD05114BF614506E0C110400721F03F
:20F32000E04101F16051704779B900F0004100020AD0B0FA80FC00FA0CF001F16051A1EBC8
:20F340000C5101EBD0214005704741020CBF40F4E0016FF00001002070470000B0B581EA4D
:20F36000030C0CF0004C40F2FF7515EA11541DBF15EA1357AC42AF4239E0E41923EA45534D
:20F3800043F48013C90241F0004141EA505EC7021100A7FB020200284FF00000EEFB01209C
:20F3A0004FF00001E3FB072118BF42F00102401800214941E3FB0E01A4F580640F0302D2A8
:20F3C00052004041494154F101046CDD470872F1004250F1000051EB0451A1F580115CBF35
:20F3E00041EA0C01B0BD4CEA05510020B0BD05EA1357AC4214BFAF4241E050EA410E1CBFBF
:20F4000052EA430E02E061460020B0BD24423C441BD15FEA070EF6D0090302BF014600201F
:20F42000AEF1140EB1FA81F7AEEB070401FA07FE0C37C7F1200100FA07F7C8404EEA000EE2
:20F4400023EA455343F48013A2E733F00043B3FA83F704BFB2FA82FE77440B3FE41BB7F18C
:20F46000200E2FBF02FA0EF3BB40C7F1200E22FA0EFE38BF43EA0E03BA40641C82E750EA18
:20F48000410E14BF52EA430E6FF000014FF4001717EB430F8ABF194617EB410FB5E74CEAE3
:20F4A00005510020B0BDD4F10104B4F120070FDAC4F12007520828BF42F0010210FA07F592
:20F4C00001FA07F7E1BF2A43E0403843E1400FE0352C98DCC7F1200452EA400220FA07F239
:20F4E00018BF42F0010231FA07F0A1400A43002172F1004250F1000051EB0C01B0BD0000F3
:20F500004FEAF17CBCF1E04C2CBFBCF5001F11E05FEA4C0C34BFBCF17F5F2EE05FEA9C0CA2
:20F520004FEA0C1C4FEA3C0CC10071F100414CEB50707047C90241EA5051C00218BF41F076
:20F54000010141F000414FEA6C50C0F10900212810D240EACC7CCCF1200C11FA0CF070F19A
:20F560000040CCF1200C21FA0CF00CF0004C40EB0C0070474FEACC707047490011F5001F7B
:20F5800004D84FEACC10FF30C0057047C817704790EA010F44BF81F00041FFF73ABE421AB0
:20F5A0003CBF801A89184FF0004CC0F3C752FF2A24D0C1F3C75313B3D21AD2F1190327DD3E
:20F5C0004CEA01214CFA03F321EA0303D140C20D4CEA0020401834BF20EA0C004CEA500069
:20F5E000D20553EA006373EB0C0C52EB1020420012F1807F38BF7047C00DC005704749022B
:20F6000012BF9A4200EB5120F8E7D2F11703D9D57047000080B501215FF0C05001F0CEFF4C
:20F62000012004F021FB012001F003FF412001F0D5FF0028FAD04FF4807001F00FFF01201A
:20F6400001F012FF04F04FFB04F048FB04F046FB47F6FF7004F034FB04F040FB01BD70478B
:20F66000704780B2042190FBF1F202FB1102002A16D180B2642190FBF1F201FB1201002990
:20F680000CD180B24FF4C87190FBF1F201FB1200002801D1012004E0002002E0012000E061
:20F6A000002070472DE9F34F81B00024BDF804509DF806609DF807709DF809809DF80A9069
:20F6C0009DF80BA0A5F2B27080B2822801D3012055E040F2B27B03E07C4804191BF1010BF0
:20F6E0001FFA8BFBADB2AB4508D2584680B2FFF7B8FF0028F0D076480419EFE7761E5FF049
:20F70000000B17E01FFA8BFB0FF2D8101BF80000704901FB0044280080B2FFF7A2FF00283A
:20F7200006D01FFA8BFBBBF1010F01D1694804191BF1010B3000C0B21FFA8BFB80B28345A5
:20F74000E0D3FFB2781E634901FB00445FFA88F84FF4616000FB08445FFA89F93C2000FB6D
:20F7600009445FFA8AFA1AEB040404F083FA200004F09AFA04F085FA04F0B0FA0020BDE863
:20F78000FE8F30B480B2642390FBF3F380B2642490FBF4F504FB1500DBB2142B00D3643059
:20F7A000C0B2C0B2042390FBF3F31B189BB2072493FBF4F504FB1533D2B2C9B20FF2181438
:20F7C0000C1914F8014CA218D318C0B2042290FBF2F404FB1204002C03D1C9B2032900D26F
:20F7E0005B1E9BB2072093FBF0F100FB1130C0B230BC7047F8B5040000260025002704F045
:20F8000048FA06003348B6FBF0F0050040F2B270070002E0A5F26D157F1CB5F5B67F0BD9DB
:20F82000380080B2FFF71DFF0028F3D0B5F5B77F02D3B5F5B775EFE72780002701E01D3DF7
:20F840007F1C1C2D16D32088FFF70BFF002805D0BFB2012F02D11D2DF1D20BE0BFB20FF258
:20F860008400385C854205D3BFB20FF27800385C2D1AE5E7781CA070681CE0701548B6FBBA
:20F88000F0F100FB11654FF46160B5FBF0F060714FF46160B5FBF0F100FB11503C21B0FBB8
:20F8A000F1F0A0714FF46160B5FBF0F100FB11503C21B0FBF1F201FB1200E071E278A178A8
:20F8C0002088FFF75EFF2071F1BD00008033E1010085E20180510100000303060104060206
:20F8E000050003051F1C1F1E1F1E1F1F1E1F1E1F70B582B004000D001600E4B2012C0AD073
:20F900002DD3032C11D00BD3052C18D012D3072C1FD019D323E00121042001F03FFE1EE078
:20F920000121082001F03AFE19E00121102001F035FE14E00121202001F030FE0FE001215F
:20F94000402001F02BFE0AE00121802001F026FE05E001214FF4807001F020FEFFE701201C
:20F96000A840ADF80000F6B2012E03D110208DF8030009E0F6B2002E03D104208DF8030058
:20F9800002E014208DF8030002208DF80200E4B2012C0AD02CD3032C11D00BD3052C18D07D
:20F9A00012D3072C1FD019D322E000A9844801F061FE1DE000A9834801F05CFE18E000A930
:20F9C000814801F057FE13E000A9804801F052FE0EE000A97E4801F04DFE09E000A97D4883
:20F9E00001F048FE04E000A97B4801F043FEFFE773BD80B5C0B201280BD0C0F08F800328A3
:20FA00002DD019D3052850D03CD3072873D05FD384E0D2B2002A07D1012010FA01F189B2BB
:20FA2000674801F09BFE06E0012010FA01F189B2634801F090FE71E0D2B2002A07D101202D
:20FA400010FA01F189B25F4801F088FE06E0012010FA01F189B25B4801F07DFE5EE0D2B242
:20FA6000002A07D1012010FA01F189B2564801F075FE06E0012010FA01F189B2524801F061
:20FA80006AFE4BE0D2B2002A07D1012010FA01F189B24E4801F062FE06E0012010FA01F10B
:20FAA00089B24A4801F057FE38E0D2B2002A07D1012010FA01F189B2454801F04FFE06E08C
:20FAC000012010FA01F189B2414801F044FE25E0D2B2002A07D1012010FA01F189B23D48AA
:20FAE00001F03CFE06E0012010FA01F189B2394801F031FE12E0D2B2002A07D1012010FA59
:20FB000001F189B2344801F029FE06E0012010FA01F189B2304801F01EFEFFE701BD10B5F8
:20FB20001400C0B201280AD048D3032819D00FD3052828D01ED3072837D02DD33EE00120A0
:20FB400010FA01F189B21E4801F0FAFD207035E0012010FA01F189B21A4801F0F1FD207052
:20FB60002CE0012010FA01F189B2174801F0E8FD207023E0012010FA01F189B2134801F0B5
:20FB8000DFFD20701AE0012010FA01F189B2104801F0D6FD207011E0012010FA01F189B2B2
:20FBA0000C4801F0CDFD207008E0012010FA01F189B2094801F0C4FD2070FFE710BD000020
:20FBC00000080140000C0140001001400014014000180140001C0140002001400749002260
:20FBE00001E01831521C0B78FF2B01D1002004E00B78C0B28342F4D108007047C8060020BE
:20FC00002DE9F0410E0017009846069CC0B2FFF7E5FF0500002D01D1002013E02300DBB2E5
:20FC20004246D2B23900C9B230006C682468A047002129724FF6FF7180B2884201D101212C
:20FC4000297280B2BDE8F08110B50C00C0B2FFF7C5FF0100002901D1002005E02000C0B231
:20FC600049684968884780B210BDF8B504000D00160000270AE0BFB2795D2000C0B2FFF7A0
:20FC8000E3FF4FF6FF71884200D17F1CBFB2B742F1D34FF6FF70F2BD38B50C001500C0B286
:20FCA000FFF79CFF0200002A01D1002005E02900200052689268904780B232BD70B50C008A
:20FCC00015001E00C0B2FFF789FF002801D1002004E004614661C5604FF6FF7070BD0000F1
:20FCE00062F30F2262F31F42401810F0030308D0C91A1FD3DB0748BF00F8012D28BF20F8AF
:20FD0000022D130030B414461546103928BF20E93C00FAD8490728BF20E90C0048BF40F836
:20FD2000042D890028BF20F8022D48BF00F8012D30BC7047C91818BF00F8012DCB0728BF74
:20FD400000F8012D70470000DFF8A406016899B94FF4803181604FF4805141604FF0FF3191
:20FD6000C160016104214161DFF888160422C1F8B821DFF8841601600120704701F1080365
:20FD800013F0070308BF002307D001F1080303F00703C3F1080303F007035918D21A8161A0
:20FDA000C26042F001034B60511828224A60DFF840160969C16170472DE9F04101F1080426
:20FDC00014F0070408BF002407D001F1080404F00704C4F1080404F00704611802F108041D
:20FDE00014F0070408BF002407D002F1080404F00704C4F1080404F00704A5185A186C1ABF
:20FE0000E41A43F003034B60AA4201D303F082BF6E68F307FAD5102CF8D383699D4207D1C3
:20FE2000C368E318C360826143F00100506042E143699D4208D18368E3188360426143F08C
:20FE4000010050609B5036E106F00303012B40F0A080F308DB004FEAD30EBEF1200F26D2B1
:20FE6000AF68D5F80CC06545D0D0BD42CED0674506D10668012707FA0EF7BE43066086E0FF
:20FE80004FEA4E0600EB860606F1280E774503D0D0F810E07745B9D32836B44502D006690A
:20FEA000B445B3D3C7F80CC0CCF808706FE0AF69EE68AE420AD0D5F808C0D0F810E0F445EF
:20FEC000A4D3CCF80C60C6F808C024E005F2140CDCF8006046B905F1100CDCF80060D6B1DA
:20FEE00002E0F446DCF8006006F2140EDEF80080B8F1000FF5D106F1100EDEF80080B8F1B0
:20FF0000000FEED1D0F810E0F445FFF47FAF4FF0000ECCF800E0002F39D0D5F81CC000EB44
:20FF20008C0C0CF2301CDCF800E075450BD1CCF800609EB946680127D5F81CC007FA0CF797
:20FF4000BE43466023E0D0F810C06745FFF45EAFD7F810C0AC450CBF3E617E61BEB1D0F8A3
:20FF600010C06645FFF452AFB7612F6937B1D0F810C06745FFF44AAF3761BE616F6937B1D3
:20FF8000D0F810C06745FFF441AF7761BE615D191C196B685B085B006B6044F00103536051
:20FFA000A450E308202B1BD25D0000EB850505F228052E46102CFFF429AF012707FA03F39A
:20FFC00004681C4204BF2343036004D0AE6800698642FFF41BAFAA60F2609660D5606AE022
:20FFE000230A08BF002523D0B3F5803F28BF1F251ED2A3F580752D0C05F00805AB40A3F528
:020000040801F1
:200000008056360C06F00406B340A3F580473F0C07F00207C5F10E05AD1BED1BBB4005EBA7
:20002000D333DD1D24FA05F505F0010505EB430500EB850303F23013D56100265661166140
:20004000012707FA05F64768374207D146EA070444601A609361D26092602CE01B681F2D30
:200060000EBF00256D08C5F1190504FA05F500E033465E68F608F600A6420ED0EE0F03EB89
:20008000860606F110076D003E68002EF0D100698742FFF4BBAE3A60DCE79C6800698342A7
:2000A000FFF4B4AE8442FFF4B1AEE2609A609460D3600020906101F10800BDE8F0812DE939
:2000C000FE4F0446A56904F2BC102E4601688E4203D3426851188E4202D380680028F5D1A8
:2000E0004168006801EB0008A8F12F0000F1080111F0070108BF002107D000F1080101F086
:200100000701C1F1080101F0070101EB000A05F11000824538BFAA460AF1080B0AF118094F
:2001200000270198A0F1280200992046FFF726FE1BF0070022D11B20CAF8040004F2BC1063
:20014000B0E80E10ABE80E10ABF1100B0098C4F8BC010198C4F8C0010298C4F8C801C4F87F
:20016000C4B100E0814609F104000721C9F804107F1C011D4145F5D3022F01DA03F0CABDDB
:20018000AA4500F09380AAEB060041194A68520852004A6040F0010169604051C1082029D2
:2001A00019D24A0004EB820202F2280213461028E4D3012606FA01F02168014206D108432B
:2001C00020609560DD60AB60EA606FE0936820698342F6D2D2E7010A08BF002223D0B1F572
:2001E000803F28BF1F221ED2A1F58072120C02F008029140A1F580531B0C03F00403994052
:20020000A1F58046360C06F00206C2F10E02D21A921BB14002EBD131CA1D20FA02F202F01F
:20022000010202EB410204EB820101F23011EA6100236B612B61012606FA02F366681E42D5
:2002400007D143EA060060600D60A961ED60AD602CE009681F2A0EBF00225208C2F1190225
:2002600000FA02F200E019464B68DB08DB0083420ED0D30F01EB830303F1100652003368F2
:20028000002BF0D120698642FFF478AF3560DCE7886822699142FFF471AF9042FFF46EAF6C
:2002A000C5608D60A860E9600020A86100F052BBF8B504460D464E4E306808B9FFF744FD3F
:2002C00003F02EFD010000F091800A6811F1010F00F08C80D4F8B0011018C4F8B001D4F8A0
:2002E000B401D4F8B031984238BF1846C4F8B401A06968BB206908B1814200D22161C4F8BB
:20030000BC11C4F8C0210020C4F8C801306860624FF0FF3020622046202300F22806F66065
:20032000B66008305B1EF8D13248844204D1283A2046FFF723FD48E054F8040CC00814EBEF
:20034000C00008385118091AA1F128020146EFE704F2BC10034600E09B68BBB15E681F6891
:20036000F619B142F8D11E7B36070FD43E46A769B7420BD35F68D4F818C0BE19B44505D27C
:20038000D0195860E0681218A169D1E72369994238BF21610346501800E09B688BB11E6852
:2003A0008642FAD1187B00070BD4304619605E6892195A602B460246204601B0BDE8F04072
:2003C000FAE400232046FFF77AFEE06885420DD2401BE060A1696A18A26140F0010050604F
:2003E00045F00300486001F10800F2BD0020F2BDB47E00207C6000206859883C2DE9F0418B
:2004000000224B420C0A08BF002423D0B4F5803F28BF1F241ED2A4F580752D0C05F00805EE
:20042000AC40A4F58056360C06F00406B440A4F580473F0C07F00207C5F10E05AD1BED1BE7
:20044000BC4005EBD434E51D21FA05F505F0010505EB440400EB8405D5F8305155B31F2C49
:200460000EBF00266608C6F1190601FA06F6002700E07600D5F804C04FEADC0C4FEACC0C0E
:20048000ACEB010C9C4502D22A4663467BB1D5F814C04FEAD67E05EB8E052D69BCF1000FBB
:2004A00002D0AC4518BF6746002DE2D13D4675BB002A3DD1012505FA04F4640065422C4393
:2004C00045682C4000F0518165422C40651E2C0B04F0100425FA04F6750905F00805EE40A5
:2004E000B70807F00407FE404FEA560C0CF0020C26FA0CF6C6F3400E2C193C196444744435
:2005000026FA0EF52C1900EB8404D4F830517DB100E025466C68E408E400641A9C423CBF3F
:2005200023462A462C69002CF3D16D69002DF1D1002A00F01A818468641AA34280F015818E
:2005400016460469A64206D38C18CD185768FF08FF00AF4201D003F0DDBBA642FBD29769C1
:20056000D66896420AD0D2F808C0D0F810E0F445F1D3CCF80C60C6F808C023E002F2140C77
:20058000DCF8006046B902F1100CDCF80060CEB102E0F446DCF8006006F2140EDEF80080A6
:2005A000B8F1000FF5D106F1100EDEF80080B8F1000FEED1D0F810E0F445CCD34FF0000EFE
:2005C000CCF800E0002F35D0D2F81CC000EB8C0C0CF2301CDCF800E072450BD1CCF8006065
:2005E00096B946680127D2F81CC007FA0CF7BE4346601FE0D0F810C06745ACD3D7F810C024
:2006000094450CBF3E617E61A6B1D0F810C06645A1D3B76117692FB1D0F810C067459AD381
:200620003761BE6157692FB1D0F810C0674592D37761BE61102B08D245F003005060A81806
:20064000416841F0010141608CE041F00301516043F0010161601B51D908202918D24B000A
:2006600000EB830303F228031E46012505FA01F105680D4204BF2943016004D09E680069DF
:200680008642FFF468AF9C60F460A660E36069E0190A08BF002623D0B1F5803F28BF1F2612
:2006A0001ED2A1F580752D0C05F00805A940A1F58056360C06F00406B140A1F580473F0C54
:2006C00007F00207C5F10E05AD1BED1BB94005EBD131CD1D23FA05F505F0010505EB410663
:2006E00000EB860101F23011E6610025656125610125B54047682F4207D13B462B434360F7
:200700000C60A161E460A4602CE009681F2E0EBF00257508C5F1190503FA05F500E03146C8
:200720004E68F608F6009E420ED0EE0F01EB860606F110076D003E68002EF0D1006987429A
:20074000FFF409AF3C60DCE78B680569A942FFF402AFAB42FFF4FFAEDC608C60A360E160A6
:200760000020A06102F1080000E00020BDE8F0812DE9F041426813465B421A40531E1A0B70
:2007800002F01002D3405C0904F00804E3409D0805F00405EB405E0806F00206F340C3F39F
:2007A0004007A218AA18B218BA18FB409A1800EB8202D2F8304123466268D208D200521AF8
:2007C00007E06568ED08ED006D1A95423CBF2A4623462569002D14BF2C466469002CF0D197
:2007E0001E460469A64206D3CC188D185F68FF08FF00AF4201D003F08DBAA642FBD29F6958
:20080000DE689E420AD0D3F808C0D0F810E0F445F1D3CCF80C60C6F808C023E003F2140CC2
:20082000DCF8006046B903F1100CDCF80060CEB102E0F446DCF8006006F2140EDEF8008002
:20084000B8F1000FF5D106F1100EDEF80080B8F1000FEED1D0F810E0F445CCD34FF0000E5B
:20086000CCF800E0002F35D0D3F81CC000EB8C0C0CF2301CDCF800E073450BD1CCF80060C0
:2008800096B946680127D3F81CC007FA0CF7BE4346601FE0D0F810C06745ACD3D7F810C080
:2008A0009C450CBF3E617E61A6B1D0F810C06645A1D3B7611F692FB1D0F810C067459AD3CF
:2008C0003761BE615F692FB1D0F810C0674592D37761BE61102A08D245F003005860E81815
:2008E000416841F00101416030E041F00301596042F001016160125187682FB341694FEA71
:20090000D70CBCF1200FBFF476AF4FEA4C0500EB850505F228052E46102FFFF46CAF012734
:2009200007FA0CF7D0F800C01CEA070F04BF47EA0C07076004D0AE680769BE42FFF45BAF4A
:20094000A960F1608E60CD608260446103F10800BDE8F08103B0BDE8F08FF8B5044601209A
:2009600003F00AFAF52C80F0D3800B2C31BF102404F10B00C408E400E308DFF8F006016870
:2009800021FA03F515F0030233D0EA4302F00102D3185A0000EB820202F22805AA68DC0052
:2009A0005668F608F600A64201D003F0B3B99668AA42FAD0B242F8D05768FF08FF00A7424F
:2009C000F3D1B54205D1012505FA03F39943016004E000698642E8D3AE60F56044F00300C4
:2009E0005060A018416841F00101416002F10805D6E08268A24280F09E80002D00F07F80E4
:200A0000012202FA03F6760005FA03F3754235432B405D422B405D1E2B0B03F0100325FAD9
:200A200003F6750905F00805EE40B70807F00407FE404FEA560C0CF0020C26FA0CF6C6F390
:200A4000400EEB18FB186344734426FA0EF5ED186B0000EB830303F22806B368EF00D3F8D8
:200A600004C04FEADC0C4FEACC0CBC459DD1D3F808C0B34299D0634597D0664502BF02FAA9
:200A800005F5A943016006D001698C458DD3C6F808C0CCF80C60391B44F003055D60E4189F
:200AA00041F001056560095186681EB34569F708202FBFF47AAF4FEA470C00EB8C0C0CF23C
:200AC000280CE646102EFFF470AFBA400668164204BF3243026005D0DCF808E00269964535
:200AE000FFF463AFCCF80850CEF80C50C5F808E0C5F80CC08160446103F1080550E0416825
:200B000000293AD02146FFF733FE050013D047E014F1400F28BF4FF0FF340CD204F10B007A
:200B2000C408E400DFF84405416821B12146FFF765FC050034D1DFF834058268A2421CD3D5
:200B4000131B4169102B0AD362184261836043F0010050609B5044F0030048600AE00023EA
:200B60008360436142F0030048605018426842F00102426001F1080512E0C1688C420BD263
:200B8000091BC1608269A318836141F00101596044F00300506029E72146FFF789FB054677
:200BA000012003F00BF92846F2BD002800D17047F8B5A0F10804012003F0DEF8DFF8AC5445
:200BC0002A6994421ED3636803F00300012819D0D808C0000119DE0729D4266813F00303B5
:200BE00000F0E280301873421C1994420AD36B699C4200F0CA80F308202B67D2A668E768F6
:200C0000BC4201D103F086B8B442FBD0D4F804C04FEADC0C4FEACC0CBCEBC30FF2D1BE4214
:200C200043D12A68012606FA03F39A432A608C42E8D24A68D307E5D5930700F15481AB6948
:200C4000994240F0B580E9684018E860AC6140F00101616069698C4202D100216961A960FC
:200C6000E969814280F0A080DFF8FC03006808B9FFF76AF8A869002800F09680E968292996
:200C80000BD305F2BC121368984203D35468E318984202D39268002AF5D1E869884280F0AB
:200CA00083804FF0FF30E8617EE05B0005EB830303F1280C664501D09642A3D328339F421D
:200CC00001D097429ED3F760BE60B0E7A669E368A34205D0A768974294D3FB609F601DE033
:200CE00004F214073B6833B904F110073B68ABB101E067463B6803F2140CDCF800E0BEF1A0
:200D0000000FF6D103F1100CDCF800E0BEF1000FEFD19742FFF476AF00223A60002E86D08A
:200D2000E26905EB820202F230121768BC4208D113607BB96A680123E669B3409A436A60E2
:200D400075E72A699642FFF45DAF3269A2420CBF33617361002B3FF46AAF2A699342FFF449
:200D600051AF9E6122692AB12E69B242FFF44AAF1A6193616269002A3FF459AF2E69B2426D
:200D8000FFF440AF5A61936151E70A7902F00302032A7FF44CAFA8604A68520852004A6065
:200DA00040F0010161600051012003F007F8F1BD6B69994204D1A9684018A8606C61EFE796
:200DC000D208D2001018D308202B24D28E68CF68B9423FF417AFB1423FF414AFBE4205D143
:200DE000296801229A409143296073E0590005EB810101F12802964203D02A699642FFF4C5
:200E000001AF28318F4203D029698F42FFF4FAAEF760BE605EE08B69CA688A4207D08E68B5
:200E20002F69BE42FFF4EEAEF26096601EE001F21406326832B901F110063268B2B101E0CD
:200E40003E46326802F21407D7F800C0BCF1000FF6D102F11007D7F800C0BCF1000FEFD13E
:200E60002F69BE42FFF4CEAE0027376093B3CE6905EB860606F230163768B9420BD132606E
:200E800016468EB96A680123C96903FA01F122EA010169601EE02E69B342FFF4B3AE1E695C
:200EA0008E420CBF1A615A61A2B12E69B242FFF4A9AE93610B692BB12E69B342FFF4A2AE26
:200EC00013619A61496929B12B699942FFF49AAE51618A6140F001016160005169698C42EC
:200EE00008D1A86060E7520852004A6040F0010161600051C10820291BD24A0005EB820273
:200F000002F2280213461028FFF47CAE012606FA01F02968014204BF0843286004D09368B4
:200F200028698342FFF46EAE9460DC60A360E2603AE7010A08BF002223D0B1F5803F28BF83
:200F40001F221ED2A1F58072120C02F008029140A1F580531B0C03F004039940A1F580462E
:200F6000360C06F00206C2F10E02D21A921BB14002EBD131CA1D20FA02F202F0010202EB1E
:200F8000410205EB820101F23011E261002363612361012606FA02F36E681E4207D143EA62
:200FA000060068600C60A161E460A4602CE009681F2A0EBF00225208C2F1190200FA02F2E2
:200FC00000E019464B68DB08DB0083420ED0D30F01EB830303F1100652003368002BF0D187
:200FE00028698642FFF40EAE3460DCE788682A699142FFF407AE9042FFF404AEC4608C600D
:20100000A060E1600020A061286A401E28627FF4CBAED5F8C40118B94FF0FF302862C3E604
:2010200080680028FCD1F7E738B5002460B101FB00F441EA0002120C120405D0B4FBF0F01E
:20104000884218BF4FF0FF342046FFF786FC050008D015F8040C10F0030003D021462846FA
:2010600002F0BAFE284632BDB47E00207C6000204100090E7F3915D4D1F11F0114D4400018
:2010800007D2C00140F00040C84048BF6FF000407047C00140F00040C8404CBF4FF000401E
:2010A000404270470020704700424FF0004058BFC04370474FF6FF70704780B50B000100E2
:2010C000180002F096FE4FF6FF7002BD80B50B000100180002F083FE4FF6FF7002BD80B58B
:2010E00002F0AEFE80B202BD30B583B00C00150000AA01A902F0E4FE002801D1002007E0FF
:201100002B00220000990198C0B202F056FF80B23EBD30B583B00C00150000AA01A902F0EB
:20112000CFFE002801D1002007E02B00220000990198C0B202F06BFF80B23EBD2DE9F04F12
:2011400085B080460D4616461F001CBF00203860444600E0641C2078A0F109010529F9D31C
:201160002028F7D02D2801D02B2802D114F8019B01E04FF02B09002E03D4012E01D0252EC0
:2011800004DB0DB1C5F80080002067E0012E0BDB102E16D12078302813D1607840F02000D8
:2011A00078280ED1A41C0CE02078302818BF0A2607D1607840F02000782808BF1026F1D0AF
:2011C000082603942078302803D114F8010F3028FBD04FF0000A02940FF28C008DF8040052
:2011E00009E0CDF800A09DF80410401A5FFA80FB06FB0ABA641C2178A1F141001A2838BFE0
:20120000203132460FF2600002F02EFF0028E8D10398A042B5D00298201A0FF27401715C8B
:20122000401A13D4012807DABAEB0B0004D3B0FBF6F00099884209D002F042FF2221016038
:201240000FB1012038604FF0FF3A04E0B9F12D0F08BFCAF1000A05B12C60504605B0BDE815
:20126000F08F00236AE70000303132333435363738396162636465666768696A6B6C6D6EC5
:201280006F707172737475767778797A0000000000002115110E0D0C0B0B0A0A090909091C
:2012A000090808080808080807070707070707070707070707000000DFF86403006850F0AC
:2012C0000100DFF85C130860DFF858030068DFF858130840DFF84C130860DFF84403006817
:2012E000DFF848130840DFF838130860DFF83003006830F48020DFF828130860DFF824033C
:20130000006830F4FE00DFF81C130860DFF82003002101607047DFF80813096831F4803169
:20132000DFF8FC221160DFF8F812096831F48021DFF8EC221160B0F5803F03D0B0F5802F4E
:2013400009D011E0DFF8D802006850F48030DFF8D012086008E0DFF8C802006850F4A020A0
:20136000DFF8BC120860FFE7704780B50020009000200021312000F031F901000098401C3D
:201380000090C9B2002903D10098B0F5A06FF1D1312000F023F9002801D0012000E00020C0
:2013A000C0B202BD0022DFF87C321B681A0032F47C1208430243DFF86C0202607047DFF83F
:2013C0007412C0B2086070470021DFF8582212681100890889000143DFF848020160704762
:2013E000DFF84002006810F00C0070470021DFF834221268110031F0F0010143DFF824027D
:20140000016070470021DFF81C221268110031F4E0610143DFF80C02016070470021814A60
:201420001268110031F4605151EAC0017D4801607047824900220A70804900220A70C0B234
:20144000012802D0042804D007E07C480121017003E07A4805210170FFE770477749096849
:2014600008437649086070477549C0B208607047F0B5002500260021002700220023002453
:201480005FF0000CDFF89CE1DEF800E01EF00C0E7546002D04D0042D05D0082D06D03DE0D5
:2014A000684901603CE06849016039E05D49096811F47011890C891C5A4A126812F4803721
:2014C000002F03D1614A5143016026E05A4A126812F48032584B1B6813F00F035B1C002AB1
:2014E00006D1594AB2FBF3F201FB02F1016014E0514A1268C2F30312541C4F4A1268C2F385
:20150000032212F1020C504AB2FBF4F20CFB02F2B2FBF3F201FB02F1016001E049490160B7
:201520004049096811F0F0052D090FF234116E5C0168F14041603B49096811F4E0652D0AC4
:201540000FF21C116E5C4168F14081603549096811F46055ED0A0FF208116E5C4168F1407A
:20156000C1603049096811F44045AD0B0FF200116E5CC168B1FBF6F10161F0BDC9B20029D3
:2015800005D03349096808433149086005E03049096831EA00002E4908607047C9B2002938
:2015A00005D02C49096808432A49086005E02949096831EA0000274908607047C9B2002934
:2015C00005D02549096808432349086005E02249096831EA000020490860704710B40022EE
:2015E00000230021C0B24409E4B22200012A02D10B490B6806E0022A02D110490B6801E0D9
:2016000016490B68C0B210F01F0201209040034201D0012100E000210800C0B210BC70473E
:2016200000100240041002400000FFF8FFFFF6FE08100240600042422C10024020100240EB
:201640003C04424200127A00001BB70000093D0014100240181002401C100240241002406E
:201660000000000001020304010203040607080902040608F0B400220026002400250023CC
:20168000002791F803C01CF00F0C624691F803C05FEACC6C01D58B781A430B781B0621D070
:2016A0000368002406E0CD78482D02D10125A5400561641C082C14D20125A5400E882E400E
:2016C000AE42F6D1A5000F2616FA05F7BB4312FA05F52B43CD78282DE5D10125A5404561FA
:2016E000E7E703600B884FF48074A34226D34368002420E0012514F10806B5400E882E4010
:20170000AE4217D1A5000F2616FA05F7BB4312FA05F52B43CD78282D04D1012514F10806F1
:20172000B5404561CD78482D04D1012514F10806B5400561641C082CDCD34360F0BC704782
:201740000022806880B2084201D0012200E000221000C0B2704789B20161704789B24161A3
:20176000704770B400220024002300252D4E36683300C0F30346350086B2320010F44016BF
:20178000B6F5401F08D133F07063264C246834F07064244D2C600FE0C40205D50324AC40DB
:2017A000A34353F0706307E0440DE4B2240112FA04F4A34353F07063C9B2002905D0400D74
:2017C000C0B2000112FA00F003431648036070BC704710B400220F2311F00304E4B2A40056
:2017E000A3401A00C9B28B100F4C54F8233033EA0202C9B28B100C4C44F82320C9B28A10B9
:20180000094B53F82220C0B211F00303DBB29B0098401043C9B28910034A42F8210010BC93
:2018200070470000040001400800014010B4002203881A0012F441520B884C8823438C885E
:201840002343CC8823430C8923434C8923438C892343CC8923431A430280828B4FF2FF735D
:201860001A408283098A018210BC7047C9B2002904D0018851F04001018004E001884FF6BA
:20188000BF72114001807047818170478089704700220089084201D0012200E0002210001A
:2018A000C0B270472DE9F04FA1B017461C4601AD6860A9600020E86211AE4FF00A096FF041
:2018C000004802E0E86A401CE862387818B9E86A21B0BDE8F08F252807D100206861A86107
:2018E000E86128626862A8620CE017F8011BA8686A689047A8600028E4D14FF0FF30E7E750
:2019000040F0010017F8011F2029F9D023290DD02B2904D02D2906D030290AD00CE040F089
:20192000020080B2EEE740F00400FAE740F00800F7E740F01000F4E72A290DD12268111D6F
:20194000216011686963002904D54942696340F0040080B27F1C10E00021696307E0696BCF
:20196000414503D009FB0121303969637F1C3A78A2F13001C9B20A29F1D339782E291CBF4D
:201980004FF0FF3129631BD117F8011F2A2906D12268111D2160116829637F1C10E000211D
:2019A000296307E0296B414503D009FB0121303929637F1C3A78A2F13001C9B20A29F1D329
:2019C000288739780FF6D83002F080FB08B117F8010B8DF83E009DF83E00682804D13878AE
:2019E00068280AD1622005E06C2806D138786C2803D171208DF83E007F1C11A828613A78AF
:201A00001046253825D01C3877D0001F022874D9133800F09E8009386FD0801E00F03681CF
:201A2000401E00F0DF80401E022866D9001F00F0D980401F36D0401E00F08B80401E23D0BB
:201A4000C01E0CD0801E00F08480C01E00F0818024E16869411C69612521815528E12168C0
:201A6000081D20600868E8602A6B002A08D4002102F0FAFA00281ABFE968401A286B01E047
:201A8000FAF7AEFBA86113E12168081D206008680021CDE9000111A8E860782100A800F007
:201AA00097F905E19DF83E0062281FD068280DD06A2812D06C2802D071280ED07428216881
:201AC000081D20600868E96A0160F1E0E86A2268111D216011680880EAE0E86AC117236861
:201AE0001A1D22601A68C2E90001E1E0E86A2268111D216011680870DAE02068C01D20F093
:201B000007002060034603F108002060D3E90001CDE90001002904D56869411C69612D21BD
:201B20000DE0288F810704D56869411C69612B2105E0C00704D56869411C696120218155C8
:201B4000686911A94018E860114600A800F0CFF9AEE09DF83E006C280FD0712801D06A28D3
:201B60000BD12068C01D20F007002060034603F108002060D3E9000104E02168081D2060F9
:201B800008680021CDE900019DF83E0068280CD0622806D0742801D07A280CD1DDE90001AB
:201BA00006E0DDE90001C0B202E0DDE9000180B20021CDE9000195F83800000760D5DDE98C
:201BC000000109B900285BD042F02000782857D16869411C6961302181556869411C6961BE
:201BE00082554DE09DF83E0062280CD0682810D06A281AD06C2824D0712816D0742820D029
:201C00007A280CD01DE02168081D206091F900001BE02168081D2060B1F9000015E0216840
:201C2000081D20600868002110E02068C01D20F007002060034603F108002060D3E9000100
:201C400004E02168081D20600868C117CDE90001DDE9000100290EDB288F810704D56869B1
:201C6000411C69612B210AE0C00709D56869411C6961202103E06869411C69612D2181552A
:201C8000686911A94018E860114607E76869411C69612268111D21601168DEE66869411C38
:201CA0006961252181551AB16869411C696182557F1C686B6969401A296A401AA969401AB1
:201CC000696A401AE969401AA96AA0EB010A95F83800400711D420208DF84000BAF1010FD1
:201CE0000BDBD346012210A900A800F03FFC00287FF403AEBBF1010BF4D16A6911A900A838
:201D000000F034FC00287FF4F8AD30208DF84000D5F820B0BBF1010F0ADB012210A900A88C
:201D200000F024FC00287FF4E8ADBBF1010BF4D1AA69E96800A800F019FC00287FF4DDADB0
:201D400030208DF84000D5F824B0BBF1010F0ADB012210A900A800F009FC00287FF4CDAD9E
:201D6000BBF1010BF4D1EA69A869E968411800A800F0FCFB00287FF4C0AD30208DF840002C
:201D8000D5F828B0BBF1010F0ADB012210A900A800F0ECFB00287FF4B0ADBBF1010BF4D12D
:201DA00095F8380040077FF590AD20208DF84000BAF1010FFFF689AD012210A900A800F007
:201DC000D5FB00287FF499ADBAF1010AF4D17CE52DE9FA4786B00546686900909DF8180090
:201DE0006F2808BF082705D040F02000782814BF0A2710273C24D5E90001064689469DF887
:201E00001820642A01D0692A04D1002902DA764269EB4909B9F1000F0DD166B9686B50B9CE
:201E2000082F3FD195F83C0000073BD5641E00983021215436E0A4F101084446F817CDE998
:201E4000047030464946DDE9042302F055F9CDE90201B246DDE90223DDE90401A0FB02696F
:201E60005046801B3030C0B23A2803D39DF8181051390818009908F80100DDE90269B9F14B
:201E8000000F00D126B12869009961188842D2D3082F07D195F83C00000703D50098205CAE
:201EA0003028C3D1C4F13C00E861009961182961696B884207DA081A6862A88F4FF6EF7119
:201EC0000840A88710E000290ED595F83C1001F01401102908D1A96BAA69891A6A6A891A5D
:201EE0000C1A012CA8BF6C6208B0BDE8F0872DE9F24F8EB0054604AFD5E90001CDE902017B
:201F00009DF8380040F020008DF8000061280BD0686B002848BF062005D405D19DF800004F
:201F2000672801D1012068636968C1F30A5040F2FF72904225D0012819DA284602F06AF92C
:201F4000012814DB002400209DF80010612940D12A69511C29613021117029694A1C2A6106
:201F60009DF83820612A0CBF782258222DE040F2FE316A6861F31E526A60441A4FF0FF3070
:201F8000E2E7080301D1286870B10320E8619DF838006138C0B21A2811D30FF210610322E9
:201FA0002869FAF7DBF89EE10320E8619DF838006138C0B21A2805D30FF2F851EFE70FF2CE
:201FC000E851ECE70FF2E851E9E70A70A969891CA96110B90026B0467BE19DF80000612851
:201FE00040F09780686B00284CBF2126461C36B2771CD5E900ABDDE902010022002302F007
:202000002BF93ABF8BF00040CDE902A0CDE902ABA4F104088DF810200DF11109012F33DB81
:20202000DDE902010022002302F02EF92CD21C2102A802F041F9DDE9020102F0C9F90446A1
:20204000FF1F012F09DB02F0EFF902460B46DDE9020102F001FACDE9020109F20700072142
:20206000012C0BDB491E5EBF04F00F0200F8012D2411F5D502E0002200F8012D491EFAD53F
:2020800000F20709012FCBDA0DF11100A9EB00010DF11107B142B8BF0E4636B2002E31D4D6
:2020A0003046884206DA04A941184978082928BF0F2100D2002104AA821800E0761E401EE4
:2020C00012F801398B42F9D00F2904D104A941184A78521C4A70002803D504AF761C08F1EB
:2020E000040836B2701E0DD4C1190A783032D2B23A2A03D39DF838303A3B9A1801F80129BA
:20210000401EF2D5686B002840F1E380701E6863DFE0DDE902010022002302F09DF805D287
:20212000DDE9020181F00041CDE9020124B247F2975060436D4990FBF1F80FFA88F8C8F166
:2021400007040027DFF8A891012C19DBDDE902ABE00707D5504659463A464B46FDF7FEF8B6
:2021600082468B466410384649463A464B46FDF7F5F807468946002CEAD1CDE902AB21E0EC
:2021800064429246DFF86CB114D0E00707D5504659463A464B46FDF7E1F882468B46641006
:2021A000384649463A464B46FDF7D8F807468946002CEAD1DDE9020152465B4602F00CFA40
:2021C000CDE902019DF8000066280CBF08F10A000620696B4618142EA8BF132630208DF846
:2021E00010000DF11104444F012E2FDBDDE9020102F004F904F1080104220A23B0FBF3F455
:2022000003FB1400303001F8010DB4FBF3F003FB1043303301F8013D521EEED101F108049B
:20222000083E012EE0DBDDE9020102F0E7F802F005F902460B46DDE9020102F00DF9002268
:202240003B46FDF78BF8CDE90201CFE70DF11100201A0DF111079DF81110302906D1401E74
:20226000A8F1010817F8011F3029F8D09DF80010662904BF0FFA88F808F1010103D0652990
:202280000CBF012100216A6B8E1836B2B042B8BF064636B2002E1CD43146814204DAC85DD5
:2022A000352828BF392000D23020CA19521E00E0761E491E12F801398342F9D0392802D12B
:2022C000C85D401CC855002903D57F1E761C08F101080FFA88F0009033B23A469DF83810DB
:2022E000284600F00BF80FB0BDE8F08FA0860100000024400000F03F84D797412DE9F04364
:2023000085B00546894617461E46BDF93040D5F83480012E02DA01260FF29C2749F02000B7
:2023200066280AD0672840F086806FF003018C42C0F28780444580F28480641C66280CD09D
:2023400095F83C00000702D44645B8BFB04624B2B8EB040848BF4FF000082869E96924B253
:20236000012C25DA4A1C30230B54B8F1010F03DA95F83C10090702D52E211154521CEA6156
:2023800018EB040FB8BFC8F1000424B26142A962A044B045B8BF464636B22E623246394624
:2023A000EB691818F9F7DAFEA8EB0600E862C6E00818A64218DA32463946F9F7CFFEE96948
:2023C0007118E961A01BA862B8F1010F03DA95F83C00000705D528692E220A54286A401CF8
:2023E0002862C5F82C80AAE022463946F9F7B6FEE8692018E861361BB8F1010F03DA95F88F
:202400003C10090704D5411CE96129692E22425436B2B045B8BF464636B23246E119E869DD
:202420002B69C018F9F79AFEE8693018E861A8EB0600A86283E0B9F1610F16D14FF0700907
:2024400018E0464504DA95F83C10090758BFB046B8F1010848BF4FF00008B9F1670F14BF32
:202460004FF045094FF0650904E0B9F1410F08BF4FF05009E9694A1C286917F8013B0B54F2
:20248000B8F1010F03DA95F83C10090702D52E211154521CEA61B8F1010F11DB761E36B258
:2024A000B045B8BF464636B232463946EB691818F9F754FEE8693018E861A8EB0600A862FA
:2024C000E8692969471807F8019B002C5CBF2B2007F8010B03D52D2007F8010B6442002686
:2024E0000DF1080824B2012C0EDB0A22214600A802F095F9019808F8010B009C761C24B27E
:20250000012CF2DA022E06DA49F02000652804BF302007F8010B1EB9302007F8010B09E093
:20252000012E07DB761E02A8305C303007F8010B012EF7DAE86929694018381A286295F8B1
:202540003C0000F0140010280DD1A869E9690818A96A0818296A0818E96A0818A96B88426B
:20256000BCBF081A686205B0BDE8F08370B504460D4616460020002E10D015F8011BE0686A
:20258000A2689047E060002802D14FF0FF3070BD206B401C20630020761EEED170BD00007A
:2025A000686A6C747A4C00006E616E004E414E00696E6600494E46003000000062F30F22B9
:2025C00062F31F4200B5130096469446103928BFA0E80C50FAD85FEA417C28BF0CC048BF21
:2025E00040F8042BC90728BF20F8022B48BF00F8012B00BD72B6704762B67047EFF3108070
:2026000072B6704780F310887047B0FA80F0704790FAA0F0704730BF704720BF704700003B
:2026200080B502F01DF9FEF747FE5FF48030FEF772FEFEF79AFEC0B20128FAD1C0B201282D
:2026400025D10020FEF7D2FE0020FEF7E7FE4FF48060FEF7D7FE022002F05CFA102002F02C
:2026600069FA5FF480115FF48030FEF79BFE0120FEF7A5FE3920FEF7B1FF0028FAD00220B7
:20268000FEF7A2FEFEF7ACFE0828FBD101BDFEE700B585B000A8FEF7EBFE019805B000BDEC
:2026A00080B50B48006850F08070094908600948002101600848006850F0010006490860BD
:2026C000FFF7E6FF02F04FFB01BD024800687047FCED00E0041000E0001000E010B4020049
:2026E00010324B1E002109E0026000244460002404810024C46010301032491C89B29BB29B
:202700009942F1D30021016000214160002101810021C16010BC704710B504006A4800688B
:20272000002803D145F21E7020801AE067480088002803D145F21D70208012E06348018881
:2027400061480068FFF7CAFF5E485F49096801605C485E49098881805A480021C180002088
:20276000208010BD41894289012A1AD30268554B1B6813604268534B1A60524AD2884389BB
:20278000D21A504BDA804F4A928843899A184D4B9A800022428100228281002202600022C5
:2027A0004260080080B27047018100214181002181810021016000214160704770B4448912
:2027C000002C0AD100200880002A01D00020106046F292501880002026E045686C682E89AF
:2027E0000E80002A01D0E9681160296841604168002904D1002101600021418102E04189A4
:20280000491E41812F48006828602E4805602D488088401C2B4988802A48C088401E29496E
:20282000C88000201880200070BC7047F0B4049D059C46890789BE4203D346F293502080BF
:202840003DE0204EB688002E03D145F21D70208035E01C4E36681B4FD6F800C0C7F800C0B5
:20286000184FBF887F1EDFF85CC0ACF80470154FFF887F1CDFF84CC0ACF806704789002F80
:2028800004D106604660012343810DE0DB0605D403681E6000233360066002E043683360A3
:2028A000466043895B1C438183894789BB4201D24389838171603281F56000202080F0BCAA
:2028C00070470000D8840020CC320108C432010800B583B000AB01AA00210020FAF7EFFE62
:2028E000BDF800100029F5D1DFF8980300780128F0D100F0FEF8EDE710B58AB00400DFF8BC
:20290000880300210160DFF884030021016000F02DF8DFF87C030078132803D346F273200B
:20292000208021E0089403200790002006900020059000200490DFF85C0300680390DFF879
:20294000580300680290DFF8540300680190DFF84003007800900023DFF844230FF25431F2
:20296000DFF84003FAF76EFD0AB010BD00200BE080B2DFF8341311EBC00100220A60002294
:202980008A800022CA80401CC849098880B28842EED3704730B492B2042A29D1BA4A126881
:2029A0008A1A521EC24CA24209D30021C164002101650021C16147F27E20188076E0C1643B
:2029C000511C0165C16CB94A1288B1FBF2F402FB141189B2B44A12EBC1018A88002A32D16F
:2029E0000022426100228261086001228A8054E000291ED092B2082A15D1826C8C18A24A53
:202A00001268A21A521E8A4201D2C46403E09E4A12688918C164C16C9B4A1268891A0165A9
:202A2000C16C8164CEE7984A12688A18C2640165C8E70021C164002101650021C16147F24D
:202A40007E20188032E00A6805E0946984614261606190610022002A1CD0D46C8A4D2D68BC
:202A6000641B1465146D056DAC420AD25469002C01D05269EFE700244461826150610022D7
:202A8000E9E79469002CE0D100248461426190610860DFE78A88521C8A80CA888C88A242ED
:202AA00001D28A88CA80C1610020188030BC7047C16900291CD0002202650A68824206D195
:202AC00042690A60002A08D00023936105E0826943695361002B00D09A61002242610022BB
:202AE00082610022C2610022C2648888401E888070472DE9F0410024FFF780FD0400FFF761
:202B0000E4FD050060480068401C5F4908605E48006866490988B0FBF1F201FB120080B237
:202B2000614911EBC000D0F80080002600E0B846F6B2002E40F09780B8F1000F00F091800D
:202B4000D8F8147098F8360000280BD0022809D009D3042806D01CD3062803D042D3072843
:202B600056D0E4E7E3E7D8F84C0047490968401AC8F8500044480068D8F84C10884206D152
:202B8000002088F836004046FAF745FC00E00126CDE7D8F84C003C490968401AC8F8500070
:202BA00039480068D8F84C10884219D10020C8F85C000020A8F86000FFF787FDC8F8400076
:202BC0004046FAF724FA4046FAF725FC002088F83600032088F83500002088F8340000E066
:202BE0000126A4E7D8F84C0027490968401AC8F8500025480068D8F84C10884206D10420F6
:202C000088F836004046FFF753FF00E001268EE7D8F84C001C490968401AC8F850001A48F6
:202C20000068D8F84C10884219D10020C8F85C000020A8F86000FFF748FDC8F8400040462F
:202C4000FAF7E5F94046FFF733FF042088F83600032088F83500002088F8340000E001266A
:202C600065E7012664E7FFF730FD401B07490968814201D2054908602000FFF7C3FCBDE891
:202C8000F081000039880020A4860020A8860020D8320108E4320108E0320108DC320108E6
:202CA000D128010858740020F8790020EC3201080100FFFF75432F4F532D49494920546901
:202CC000636B205461736B007047574800685749096811EB8000001F554908607047704795
:202CE0007047704710B40400019812EB8000001F5FF080720260001F0460001F4D4A02602B
:202D0000001F5FF012320260001F5FF003320260001F5FF002320260001F0360001F016094
:202D2000001F5FF011310160001F5FF010310160001F5FF009310160001F5FF00831016061
:202D4000001F5FF007310160001F5FF006310160001F5FF005310160001F5FF0043101605D
:202D600010BC704738B5FFF7B0FC02003248006832490968884217D02F480068D0F8940085
:202D8000101A2D490968C1F890002B480068D0E9264529480068D0F89000002120186941A6
:202DA000254B1B68C3E9260124480068C0F8942021480068D0F8B80021490968884205D240
:202DC0001D4800681E490968C0F8B8101C480021016031BD704710B50024FFF70FFC040055
:202DE00018480078401C174908702000FFF70AFCF9F735FEF9F7FEFE10BD401E12490860AE
:202E0000124800680002000A104908601048006850F005000E4908600D48006850F0020060
:202E20000B49086070470000BC320108B832010884860020B1D90008BC860020C0860020B1
:202E4000988600203888002014E000E020ED00E010E000E0002004E01F49002241F82020BC
:202E6000401C0028F8D0704710B500241A4801E02034001D01680029FAD00068FFF7C5FB38
:202E800004192000C0B210BDC0B24209C0B210F01F010120D1F11F018840D2B20E4951F878
:202EA00022100843D2B20C4941F822007047C0B24209C0B210F01F010120D1F11F01884090
:202EC000D2B2054951F8221031EA0000D2B2024941F822007047000088860020024900220E
:202EE0000A80002101807047A2870020024900220A80002101807047A4870020034900229D
:202F00000A8000210180704700000000A687002000B589B0A6490968002908D0A5490968D3
:202F2000A34A1268B1FBF2F1A34A116006E0A14909680A22B1FBF2F19F4A11609F499E4A17
:202F400012680A60994900220A609D4900220A6000210AE089B29B4A12EBC102002393808C
:202F60000023D38000231360491C974A128889B29142EFD395490968002903D147F2463199
:202F800001802DE092490968924A1268914203D247F24631018023E08F490978132903D3BA
:202FA00046F2732101801BE008900320079000200690002005900020049085480068039090
:202FC0008648006802908148006801908248007800900023824A0FF210218248FAF732FA8D
:202FE00009B000BD10B4022280F82A2089B2012905D1416A6D4A1268511881610DE0016AF7
:20300000002905D1416A694A12685118816104E0016A664A12685118816181696A4A128892
:20302000B1FBF2F302FB131189B2664A12EBC1010A68002A07D1002202610022426108600E
:20304000012088802EE08269584B1B68D21AC2610B6805E05A6942610361106158610023AA
:20306000002B1CD09A69514C2468121BDA61DA69C469A2420AD21A69002A01D01B69EFE79D
:2030800000220261436118610023E9E75A69002AE0D100224261036158610860DFE78888DD
:2030A000401C8880C8888A88904201D28888C88010BC70478169444A1288B1FBF2F302FB2A
:2030C000131189B23F4A12EBC1010A68824206D102690A60002A08D00023536105E04269FE
:2030E00003691361002B00D05A61012280F82A2000220261002242618888401E88807047DE
:20310000F0B583B00BE0FFF7E0FA041B00A8F9F74CFE2B480068A04201D22948046000AB0B
:2031200001AA00210020FAF7CAFA050000A8F9F70CFEFFF7CAFA04001C480068401C1B49FD
:2031400008601A48006820490988B0FBF1F201FB120080B21B4911EBC0000668002700E0E0
:203160000127FFB2002FCED1002EF9D035690F480068B169884216D13000FFF79BFF308D0C
:20318000022804D101213000FFF72CFF02E0032086F82A00B2681000002802D0F168300063
:2031A00090472E00DDE70127DBE70000B0860020F8320108D4320108B4860020B88600200C
:2031C000AC860020607A00200C330108FC32010804330108D0320108F4320108003301086E
:2031E000013101081875002075432F4F532D4949492054696D6572205461736B0000000082
:203200000FF210100FF2A00108000FF2A00108000FF29C0108000FF29C0108000FF2980153
:2032200008000FF2980108000FF2940108000FF2940108000FF2900108000FF29001080074
:203240000FF28C0108000FF28C0108000FF2880108000FF2880108000FF2840108000FF28F
:20326000840108000FF2800108000FF2800108000FF27C0108000FF27C0108000FF2780127
:2032800008000FF2780108000FF2740108000FF2740108000FF2700108000FF270010800B4
:2032A0000FF26C0108007047AC5800200C0000007D000000F4010000A05A00207D000000A8
:2032C000F40100006400000040060000F83B002040000000E803000010000000945C0020B1
:2032E0000C0000007D000000F40100000D00000068000000120000000A000000885E0020B9
:203300000C0000007D000000F40100000D00000068000000E00E00001748FF2101700020BC
:2033200080F309881548016881F3088814481549016062B6FEE772B6EFF3098028B12038E3
:2033400080E8F00F10490968086000B50F4880475DF804EB0E480F490A7802700A480E4972
:203360000A680260106890E8F00F203080F309884EF0040E62B6704722ED00E084860020FE
:2033800004ED00E000000010BC860020652D01083A8800203B880020C086002038B5040033
:2033A00001212020FEF7FAF8E4B2012C40D200230122E4B20520C14900FB04108178E4B246
:2033C0000520BE4D00FB04504078FCF791FA00230122E4B20520B94900FB04100179E4B216
:2033E0000520B64D00FB0450C078FCF781FA0022E4B20520B14900FB04108178E4B2052016
:20340000AE4B00FB04304078FCF7F3FA0022E4B20520AA4900FB04100179E4B20520A74BE6
:2034200000FB0430C078FCF7E4FA4FF6FF7000E0002032BD10B584B00400E4B2012C80F081
:2034400082800122E4B205209C4900FB04100179E4B20520994B00FB0430C078FCF7C9FA62
:2034600002A80190002000906423002200210020F9F737FA0122E4B20520904900FB041090
:203480008178E4B205208D4B00FB04304078FCF7B0FA02A80190002000904FF41673002243
:2034A00000210020F9F71DFA0022E4B20520834900FB04108178E4B20520804B00FB04305E
:2034C0004078FCF796FA02A80190002000906423002200210020F9F704FA0122E4B2052010
:2034E000764900FB04108178E4B20520734B00FB04304078FCF77DFA02A801900020009050
:203500004FF4FA73002200210020F9F7EAF90022E4B20520694900FB04108178E4B2052073
:20352000664B00FB04304078FCF763FA02A80190002000906423002200210020F9F7D1F914
:203540004FF6FF7000E0002004B010BD10B584B00400E4B2012C80F082800022E4B2052027
:20356000564900FB04100179E4B20520534B00FB0430C078FCF73DFA02A80190002000904E
:203580006423002200210020F9F7ABF90122E4B205204A4900FB04108178E4B20520474BE7
:2035A00000FB04304078FCF724FA02A80190002000904FF41673002200210020F9F791F97F
:2035C0000022E4B205203D4900FB04108178E4B205203A4B00FB04304078FCF70AFA02A8B8
:2035E0000190002000906423002200210020F9F778F90122E4B20520304900FB04108178E0
:20360000E4B205202D4B00FB04304078FCF7F1F902A80190002000904FF4FA7300220021D5
:203620000020F9F75EF90022E4B20520234900FB04108178E4B20520204B00FB04304078C5
:20364000FCF7D7F902A80190002000906423002200210020F9F745F94FF6FF7000E00020F0
:2036600004B010BD10B50400E4B2012C25D2C9B2012911D112480078002804D02000C0B25F
:20368000FFF7D8FE19E0F4F717F9212815D12000C0B2FFF7CFFE10E009480078002804D031
:2036A0002000C0B2FFF752FF07E0F4F705F9212803D12000C0B2FFF749FF10BD7809002006
:2036C0001F88002080B52E484FF6FF71018001F05DFB4FF6FF7001F0B9FC02F01FF901BDD7
:2036E00080B501F068FB01BD80B5254800884FF6FF71884214D0234800680090FFF7F0FFAE
:2037000022481F49098801801D480088002803D11C48006801F041FB19484FF6FF7101804C
:2037200001BD38B504000D004FF41B7220211848F6F7FEF9F4F7A5FA114800884FF6FF7158
:20374000884201D0002011E0A4B2002C0DD1A02200210D48F6F7ECF90B48286009490860BE
:20376000074804804FF6FF7000E0002032BD80B506480088002801D101F024FB01BD000000
:203780001C870020EC850020387700201E8700200852002070B58EB004001600E4B2102C78
:2037A00001D300203AE23000DFF89014FBF79CFD05D930005FF08041F8F798FC01D200202F
:2037C0002CE2E4B20C20DFF8781400FB04104068DFF87014884205D101214FF40060FDF74B
:2037E000DDFE2DE0E4B20C20DFF8541400FB04104068B0F1804F04D101210120FDF7DEFED1
:203800001EE0E4B20C20DFF8381400FB04104068DFF83414884204D101210220FDF7CEFE4C
:203820000EE0E4B20C20DFF8181400FB04104068DFF81814884203D101210420FDF7BEFE87
:2038400001210C20FDF7AAFEE4B2002C1FD0022C3DD02CD3042C59D049D3062C72D063D374
:20386000082C00F08B807BD30A2C00F0A380C0F093800C2C00F0BA80C0F0AA800E2C00F059
:20388000D380C0F0C2800F2C00F0DD80EAE04FF48070ADF8000018208DF8030003208DF851
:2038A000020000A9DFF8A803FDF7E4FEDAE04FF40070ADF8000018208DF8030003208DF88B
:2038C000020000A9DFF88803FDF7D4FECAE04FF48060ADF8000018208DF8030003208DF83B
:2038E000020000A9DFF86803FDF7C4FEBAE04FF40060ADF8000018208DF8030003208DF8DB
:20390000020000A9D248FDF7B5FEABE00120ADF8000018208DF8030003208DF8020000A9D7
:20392000CB48FDF7A7FE9DE00220ADF8000018208DF8030003208DF8020000A9C448FDF784
:2039400099FE8FE00420ADF8000018208DF8030003208DF8020000A9BD48FDF78BFE81E0A2
:203960000820ADF8000018208DF8030003208DF8020000A9B648FDF77DFE73E04020ADF8A2
:20398000000018208DF8030003208DF8020000A9AF48FDF76FFE65E08020ADF800001820FA
:2039A0008DF8030003208DF8020000A9A848FDF761FE57E00120ADF8000018208DF803002C
:2039C00003208DF8020000A9A248FDF753FE49E00220ADF8000018208DF8030003208DF80D
:2039E000020000A99B48FDF745FE3BE04FF48050ADF8000018208DF8030003208DF80200C5
:203A000000A99548FDF736FE2CE04FF40050ADF8000018208DF8030003208DF8020000A9A1
:203A20008D48FDF727FE1DE04FF48040ADF8000018208DF8030003208DF8020000A9864812
:203A4000FDF718FE0EE04FF40040ADF8000018208DF8030003208DF8020000A97E48FDF779
:203A600009FEFFE74FF418757C48007800280CD130007B49F8F73AFB15D27A483100F5F76A
:203A8000D9FFFDF7F5FA05000DE030007449F8F72DFB08D24FF47A7572483100F5F7CAFFC9
:203AA000FDF7E6FA2D1A08A8FDF7E2FC4FF47A70ADF818004720ADF814000020ADF81A0080
:203AC0000020ADF8160005A9E4B20C205C4A00FB0420406802F04AF8E4B20C20584900FB9C
:203AE0000410007A01281DD16020ADF804000120ADF80600ADF80A500220ADF80C0001A9B0
:203B0000E4B20C204E4A00FB0420406802F049F80821E4B20C204A4A00FB0420406802F019
:203B20005FF970E0E4B20C20454900FB0410007A02281DD16020ADF804000120ADF80600F7
:203B4000ADF80A500220ADF80C0001A9E4B20C203B4A00FB0420406802F05FF80821E4B2D3
:203B60000C20374A00FB0420406802F042F94AE0E4B20C20324900FB0410007A03281DD19B
:203B80006020ADF804000120ADF80600ADF80A500220ADF80C0001A9E4B20C20284A00FB85
:203BA0000420406802F07CF80821E4B20C20244A00FB0420406802F026F924E0E4B20C20DC
:203BC0001F4900FB0410007A04281CD16020ADF804000120ADF80600ADF80A500220ADF820
:203BE0000C0001A9E4B20C20154A00FB0420406802F098F80821E4B20C20114A00FB042040
:203C0000406802F009F90121E4B20C200C4A00FB0420406802F0D6F84FF6FF700EB070BDA8
:203C200080B50121C0B20C22054B02FB0030406802F0AEF84FF6FF7002BD00000100C64254
:203C400008060020002C0140000400400008004000080140000C014000140140D9870020D2
:203C60000000C842000020410149C0B20860704720000E422248008850F01000204908805B
:203C800070471F4800884FF6EF7108401C490880704700201B49098808001B49098889B2A0
:203CA00080B250EA0140704710B50400FFF7E2FF200C1549088013480480FFF7E2FF10BD6B
:203CC00010B50400FFF7D6FF200C10F00F000F4908800F480480FFF7D4FF10BD08480088EC
:203CE0008006FBD57047064800884FF6F771084003490880024800880007FBD570470000B8
:203D0000042800401C28004018280040082800400C28004080B5012002F0A4B800BF0000EC
:203D200006490868002801D000207047044808600449C908C900091A01607047C8860020B0
:203D400040A9002040CA002010B5224C206890B1201D02F092F804F1080002F08EF804F111
:203D60000C0002F08AF804F1100002F086F804F1140002F082F810BD38B50446154D2868E3
:203D800090B9281D02F078F805F1080002F074F805F10C0002F070F805F1100002F06CF81F
:203DA00005F1140002F068F801202860052C04D205EB8400001D02F061F831BD052800D32D
:203DC000704780B5034901EB8000001D02F057F801BD0000CC7E00200022FBF785BF03E07E
:203DE0000B680370401C491C13005A1E002BF7D17047F8B505000C00170004208DF8000069
:203E000000F0A8FEBE080420B7FBF0F101FB1071002909D0761C07E02968200000F0AEFE4A
:203E20008DF80000241D2D1D3000461E80B2002803D09DF800000428EED000F096FEF1BD00
:203E400010B5002400E0641C042C36D214200FF2E40100FB0410C06814210FF2D80201FB84
:203E60000421096814220FF2CC0302FB043292685118491E884201D0002020E0601C042846
:203E80000FD214200FF2AC0100FB0410C06814210FF2A00201FB04214969884201D30020BF
:203EA0000DE014200FF28C0100FB0410007900F069F80028C7D1002001E04FF6FF7010BD38
:203EC00030B4002300E05B1C042B2FD214240FF2640504FB03542468A042F4D314240FF2EE
:203EE000540504FB0354E4688442ECD314240FF2440504FB0354248A002C01D1002016E0A8
:203F0000002906D014240FF22C0504FB035424790C60002A07D014210FF2180401FB034146
:203F20000968401A10604FF6FF7000E0002030BC70470000000000000200000000000100EC
:203F4000FFFF0000FFFF0000000001000300000000000100FFFF0100FFFF00000000001053
:203F60000100000000000800FFFF0710000000000000003004000000100000000F000030A0
:203F8000FFFF000038B504000020002510E0EDB22421344A01FB05210978E4B28C4206D1BD
:203FA000EDB224202F4900FB0510406980476D1CEDB2042DEBD380B232BD2DE9F0410400A3
:203FC0000D0016001F0000205FF0000817E05FFA88F82421234A01FB08210978E4B28C429C
:203FE0000BD13A00310028005FFA88F82423DFF874C003FB08C3DB68984718F101085FFAD1
:2040000088F8B8F1040FE2D380B2BDE8F0812DE9F04104000D0016001F0000205FF0000863
:2040200017E05FFA88F824210E4A01FB08210978E4B28C420BD13A00310028005FFA88F8C1
:204040002423DFF820C003FB08C31B69984718F101085FFA88F8B8F1040FE2D380B2BDE803
:20406000F081000044050408C9B2830706D0521E22D310F8013B9942F7D11FE0083A13D32C
:2040800002F1040241EA012141EA014150F8043B121F21BF4B40A3F1013C2CEA030C1CF048
:2040A000803FF3D0C9B2001F083210F8013B521E28BF91EA030FF8D818BF0120401E7047A5
:2040C000014801F0DDBE0000CC8600200278C9B28A421AB11CBF10F8012FF9E718BF002023
:2040E0007047000013F0004C03D55B42524263F100039CEA210C15D11B4229D109424CD102
:204100002AB18446B0FBF2F002FB10C2704701F0B9BEFCD30022002370470B000200002186
:204120000020704710B5644603D34942404261F10001FFF7E1FF640004D34942404261F193
:204140000001244203D55B42524263F1000310BD904271EB030CE0D370B5B1FA81F4B3FAE9
:2041600083F52C1BA340C4F1200532FA05F63343A2405FF00046E64002E05B085FEA3202C7
:20418000841A71EB030524BF204629467641F4D302000B003000002170BD012AB9D970B57A
:2041A000140C20D0B1FA81F4B2FA82F5C4F120046419B4F12006D6D3B2405FF00044F44029
:2041C000002502E052085FEA3303C61A71EB020E24BF3046714664416D41F3D302000B007D
:2041E0002000290070BD0C46B1FBF2F102FB11452D0445EA1045B5FBF2F402FB145580B232
:2042000040EA0545B5FBF2F002FB105240EA044070BD000070B4416801F0004201210D4B24
:2042200044681C40446001D104686CB104684568E60F46EA4505456064000460491EEC022D
:20424000F4D544682340436043681A434260084670BC7047FFFF0F004FF4001C1CEB410F45
:2042600094BF1CEB430F09E041EA030C50EA4C0C52EA0C0C03D2994208BF9042704714BFB6
:204280008B428242704700004FF4001C1CEB410F94BF1CEB430F09E041EA030C50EA4C0CBF
:2042A00052EA0C0C03D28B4208BF8242704714BF994290427047000070B504460D46606805
:2042C000C0F30A5040F2FF71884209D16068000302D12068002801D0022070BD012070BDCF
:2042E00030B92046FFF796FF012801DB002070BD012D0EDB40F2FF71091A8D4209D3606843
:20430000002847BF00202F4900202F49C4E90001E4E74142A942616806DA2C4A114040198F
:2043200041EA0050606049E001F0004162681203120B42F480126260401E451905F135007A
:20434000352803D361600020206070BD002215F11F0F05DA20352268606820600020606060
:20436000684213D0521E9241D243C0F1200325689D4055EAD2722568C540666806FA03F341
:204380002B432360636823FA00F06060606808436060B2F1004F03D80AD12078C00707D5DE
:2043A0002068401C2060206810B96068401CB9E76068884202D12068002897D04FF0FF309A
:2043C00070BD00BF0000F0FF0000F07FFFFF0F80F446400D40EAC120490006D200F013F858
:2043E000004248BF6FF00040604700F00CF84FF0004188428CBF084640426047400D40EAB7
:20440000C12049000CD240F00040490DA1F58061491C05D4D1F11F0154BFC840C01770478E
:204420004FF0000070470000010040F10880F446404200F004F851F000416047010009D021
:20444000B0FA80F18840C91CC1F58461090501EBD02140057047000070B44FF0004591EAEF
:20446000030F44BF6B4001F018BD841A71EB030604D26E40001BB141121973414FF4001CE4
:204480001CEB410F34BF7CEB430684E00C0DA4EB1356362E7DDC012E43DC45EAC32343EA60
:2044A000525312BFD20292025B08240545EAC12141EA5051D2EBC020994125D407D1B0FAC3
:2044C00080F610FA06F164D00020203608E0B1FA81F6B140C6F1200220FA02F21143B04095
:2044E0004FEAF474B4EB465434F001064FEA74040AD8D6F50016760D04F00044F04061FAFD
:2045000006F25040F1404840C00A40EA415021F0004128BF5FEA500550F1000044EBD1219C
:2045200037E045EAC323DB0A45EAC121C90AB6F120050EDD42EA0242120CC5F1200603FA68
:2045400006F6EB4042EA06056D42984161F100010DE062FA06F5F240554063FA06FC82EA4C
:204560000C02F3405A406D42904161EB030111F4801F05D1641E620502D06D0040414941E3
:2045800021F48011430875F1004350F1000041EB045170BC70471CEB410F15D223F0004348
:2045A00052EA43060BD04FEA4C0CBCEB410F04D80C0D661E342EB7DDEBE7801A994150EA24
:2045C000410608BF0021E4E708BF1CEB430F28BF6FF00001DDE70000F0B540F2FF7581EA00
:2045E000030C0CF0004C15EA11541DBF15EA1357AC42AF42E5E0BC41C1F31301C3F3130386
:20460000801A994143F4801304D2641E4000494180185941C90241EA5051B1FBF3F603FBDE
:204620001611A2FB0675D7EBC020A94102D2761E80185941C90241EA5051B1FBF3FE03FBE3
:204640001E11A2FB0E75D7EBC020A94103D2AEF1010E80185941890241EA9051760546EA88
:204660008E2EB1FBF3F603FB1611A2FB0675D7EB8020A94102D2761E80185941C90241EAD0
:2046800050514EEA060EB1FBF3F603FB1611A2FB0675D7EBC020A94102D2761E8018594135
:2046A000C90241EA5051B1FBF3F703FB1711A2FB0735D3EBC020A94167F100070CBF0042DA
:2046C00047F0010766F3D5274FEA1E31B80814F5806412DDBD0775F1004250EB0E5051EBE1
:2046E000045111F5801F5CBF41EA0C01F0BD4CF07F6141F0E0410020F0BDBD076D0840EA22
:204700000E5041F48011D4F10104B4F120060ADAC4F120060200E04001FA06F3E14018438F
:20472000B24015430EE0342C13DCC6F1200445EA40056D0820FA06F2154321FA06F0A140D2
:204740000D43002175F1004250F1000051EB0C01F0BD00205FEA0C01F0BDCFB992185B4118
:20476000B3FA83F704BFB2FA82F6BF190B3FB7F120062FBF02FA06F3BB40C7F1200622FA63
:2047800006F638BF3343BA401CB1E419641E33E77F4231F00041B1FA81F404BFB0FA80F62A
:2047A000A4190B3CB4F120062FBF00FA06F1A140C4F1200620FA06F638BF3143A0403C1BD7
:2047C0001AE7AC421ABF05EA1357AF4212E050EA41061CBF52EA4306BFE750EA4107304656
:2047E00061461CBF41EA0551F0BD52EA430C08BFC143F0BD00204FF4001616EB410F98BFE5
:2048000016EB430F08BF16EB410F24BFC14305E016EB430F0CBF61464CEA0551F0BD91FBD7
:20482000F2F303FB1211C0E90031704780B5FDF7E1FE01BD80B5442803D21030C0B201F002
:2048400097FB01BD38B504000D000020442C06D2FDF7D4FEAC4941F82450FDF7D3FE31BD87
:2048600010B5002404E0A9492000FFF7EBFF641C442CF8D310BD80B5002000F02DF901BDC8
:2048800080B5012000F028F901BD80B5022000F023F901BD80B5032000F01EF901BD80B580
:2048A000042000F019F901BD80B5052000F014F901BD80B5062000F00FF901BD80B5072092
:2048C00000F00AF901BD80B5082000F005F901BD80B5092000F000F901BD80B50A2000F0CA
